:100000000C9476140C94A0140C94A0140C94A014CA
:100010000C94A0140C94A0140C94A0140C94A01490
:100020000C94A0140C94A0140C94A0140C94A01480
:100030000C94A0140C94B0200C94A0140C94A01454
:100040000C94A0140C94BDC40C9446C00C94A01441
:100050000C9489A10C947FA10C94A0140C94A0146E
:100060000C94A0140C94A0140C94A0140C94A01440
:100070000C94A0140C94A0140C94A0140C94A01430
:100080000C9426750C94A0140C94A0144E414E4967
:100090004E495459494E46CDCCCC3D0AD7233C1746
:1000A000B7D13877CC2B329595E6241FB14F0A0093
:1000B0000020410000C84200401C4620BCBE4CCA83
:1000C0001B0E5AAEC59D7400407A10F35A00A07200
:1000D0004E18090010A5D4E80000E8764817000083
:1000E000E40B54020000CA9A3B000000E1F5050051
:1000F0000080969800000040420F000000A086019A
:10010000000000102700000000E803000000006469
:1001100000000000000A00000000000100000000D4
:10012000002C76D888DC674F0823DFC1DFAE59E1A9
:10013000B1B796E5E3E453C63AE651997696E8E618
:10014000C28426EB898C9B62ED407C6FFCEFBC9CEB
:100150009F40F2BAA56FA5F490055A2AF75C936BFD
:100160006CF9676DC11BFCE0E40D47FEF520E6B5B8
:1001700000D0ED902E0300943577050080841E0892
:100180000000204E0A000000C80C333333330F98B0
:100190006E12831141EF8D2114893BE65516CFFE77
:1001A000E6DB18D1844B381BF77C1D901DA4BBE403
:1001B00024203284725E228100C9F124ECA1E53D45
:1001C0002741425300504C410042656400456E6334
:1001D0006C6F73757265002568753A2530326875E5
:1001E0000025303268753A253032687500202020AD
:1001F000202020200020202020003FFFF038007029
:1002000030FC3020FC102078102030102C00D02E34
:1002100031D02F7BD02F7BD02E31D02C00D020306E
:100220001020781020FC1030FC303800703FFFF0B8
:100230003FFFF03800703186302387102787902FDA
:1002400087D02F03D0203010207810207810203055
:10025000102F03D02F87D027879023871031863027
:100260003800703FFFF0041040020820020820040C
:100270001040082080104100104100082080041028
:10028000400000001FFFF81FFFF86E6F7469666979
:10029000636174696F6E200063616E63656C00500A
:1002A00072696E742041626F727465640044697390
:1002B0006D6973730055492041626F727465640003
:1002C000706175736500526573756D6500554920E1
:1002D00050617573650050617573696E672E2E2EBF
:1002E00000726573756D65006E6F74696669636130
:1002F00074696F6E200050726F6265205A204F66DD
:10030000667365740046696C2E204469612E004551
:1003100020696E206D6D5E33002008204661637495
:10032000002008204D6178002008204D696E004FA4
:100330006666004F6E004175746F74656D7000568F
:1003400054726176204D696E00566D696E00566D6F
:100350006178204500566D6178205A00566D6178AD
:10036000205900566D6178205800416D6178204514
:1003700000416D6178205A00416D6178205900413B
:100380006D6178205800412D54726176656C004192
:100390002D5265747261637400416363656C00562D
:1003A000652D4A65726B00565A2D4A65726B005670
:1003B000592D4A65726B0056582D4A65726B005074
:1003C000726F6265205A204F6666736574005072C2
:1003D0006F62652059204F66667365740050726FB6
:1003E00062652058204F66667365740045207374FB
:1003F0006570732F6D6D005A2053746570732F6D87
:100400006D00592053746570732F6D6D0058205323
:10041000746570732F6D6D00416476616E63656401
:100420002053657474696E6773003F0043616E63A7
:10043000656C00496E6974004D34323800496E694C
:100440007469616C697A6520454550524F4D00468C
:10045000696C616D656E740054656D706572617470
:100460007572650053746570732F6D6D0050726FF7
:100470006265204F666673657473004A65726B002F
:10048000416363656C65726174696F6E0056656C7B
:100490006F636974790053657420486F6D65204FF0
:1004A00066667365747300436F6E66696775726123
:1004B00074696F6E0053746F770053572D4D6F64DE
:1004C00065004465706C6F790053656C662D5465EA
:1004D000737400526573657400426564004E6F7AF0
:1004E0007A6C650046616E20537065656400436FE9
:1004F0006E66696775726174696F6E0052657374B8
:100500006F72652044656661756C7473004C6F6131
:10051000642053657474696E67730053746F7265F9
:100520002053657474696E67730050726568656105
:1005300074202420436F6E6600424C546F756368CC
:100540000050726F6265205A204F666673657400B2
:10055000416476616E6365642053657474696E6787
:1005600073004D61696E004D3139305335350A479E
:1005700032380A4732390A4D3430300A4D3130347E
:10058000533231350A4732380A4D3130395332311E
:10059000350A4D34323053310A47315831303059F1
:1005A00031303046353030300A47315A300A4D3517
:1005B00030300A4D31313720536574205A204F6650
:1005C00066736574004D313036533132380A4D331D
:1005D00030334338533231354530550A4D3530309C
:1005E0000A4D313137205049442054756E652044FE
:1005F0006F6E65004D3139305335350A4D31303429
:10060000533231350A4732380A4732394C310A47BA
:100610003120583130305931303046353030300AA1
:1006200047315A30004D3530300A4D313137205383
:10063000657474696E67732053746F7265640050DB
:1006400072657020666F72205A2041646A757374F7
:100650000053746F72652053657474696E6773001C
:100660005049442054756E65005365747570004D93
:1006700061696E003F004261636B0053746F7000EC
:10068000436F6E66696775726174696F6E00546559
:100690006D7065726174757265004D6F74696F6E0F
:1006A00000486F7374205374617274004C657665F2
:1006B0006C696E6720546F6F6C7300526573756D53
:1006C00065205072696E740054756E650053746FC6
:1006D00070205072696E740050617573652050729D
:1006E000696E7400496E666F2053637265656E00B3
:1006F0002100486F74656E6420746F6F20636F6CA7
:1007000064004261636B0050726F63656564004D05
:100710006F74696F6E0044697361626C6520537415
:10072000657070657273004D3834004F6666004F17
:100730006E00426564204C6576656C696E67004C9E
:100740006576656C20426564004732394E0041751C
:10075000746F20486F6D6500473238004D61696ED7
:100760000050726568656174202420456E640050F5
:100770007265686561742024204265640054656D6B
:10078000706572617475726500C501C101436F6F58
:100790006C646F776E005072656865617420240028
:1007A00046616E20537065656400426564004E6F5B
:1007B0007A7A6C65004D61696E0050726F626520D7
:1007C0005A204F666673657400466C6F7700466109
:1007D0006E20537065656400426564004E6F7A7ADE
:1007E0006C65005370656564004D61696E00486F0B
:1007F0006D696E67204661696C6564006F70656E37
:1008000000545249474745524544003A20007A5F18
:100810006D696E00795F6D696E00785F6D696E005D
:100820005265706F7274696E6720656E6473746F61
:1008300070207374617475730A0020746F6F206C7C
:100840006F6E6720657874727573696F6E20707251
:100850006576656E7465640A0020636F6C6420655C
:100860007874727573696F6E2070726576656E74D8
:1008700065640A00486F6D65202573257325732014
:100880004669727374005761726E696E673A2048E8
:100890006F6D696E672042756D702044697669736B
:1008A0006F72203C20310A000202040000000000A8
:1008B000000000000000000000964300005C4300C0
:1008C000009643000000410000004100000040008D
:1008D0000000010000000100008000555555000097
:1008E00000400033333300AAAA2A004992240000B2
:1008F000002000C7711C0099991900D145170055B7
:100900005515003BB11300244912001111110000CC
:100910000010000F0F0F00E3380E0043790D00CCDC
:10092000CC0C00C3300C00E8A20B0064210B00AA21
:10093000AA0A00703D0A009DD80900427B09009276
:10094000240900DCD3080088880800104208000051
:10095000000800F0C1070087870700755007007185
:100960001C07003EEB0600A1BC060069900600666D
:10097000660600703E06006118060017F405007454
:10098000D105005BB00500B290050062720500550C
:1009900055050078390500B81E0500050505004E0F
:1009A000EC040087D40400A1BD040090A704004912
:1009B000920400C17D0400EE690400C7560400449F
:1009C0004404005C320400082104004110040000CB
:1009D0000004003FF00300F8E0030026D20300C348
:1009E000C30300CCB503003AA803000A9B030038F8
:1009F0008E0300C08103009F750300D0690300507F
:100A00005E03001D53030034480300913D0300338F
:100A100033030016290300381F0300971503003025
:100A20000C0300030303000BFA020049F10200BAB1
:100A3000E802005CE002002DD802002DD00200592F
:100A4000C80200B0C0020031B90200DAB10200AA47
:100A5000AA0200A0A30200BC9C0200FA9502005C5E
:100A60008F0200DF88020082820200457C0200279C
:100A700076020027700200436A02007C640200D004
:100A80005E02003F590200C8530200FFFDFCFAF865
:100A9000F6F4F2F0EEECEAE9E7E5E3E1E0DEDCDAD9
:100AA000D9D7D5D4D2D0CFCDCBCAC8C7C5C3C2C081
:100AB000BFBDBCBAB9B7B6B4B3B2B0AFADACAAA9FA
:100AC000A8A6A5A4A2A1A09E9D9C9A99989795944A
:100AD0009392908F8E8D8B8A89888786848382817A
:100AE000807F7E7D7B7A797877767574737271708A
:100AF0006F6E6D6C6B6A696867666564636261607E
:100B00005F5E5D5C5B5A5958585756555453525165
:100B100050504F4E4D4C4B4A4A4948474646454433
:100B200043424241403F3E3E3D3C3B3B3A393838F0
:100B300037363535343332323130302F2E2E2D2C9E
:100B40002B2B2A2929282727262525242323222140
:100B50002120201F1E1E1D1C1C1B1B1A19191818D2
:100B6000171616151514131312121111100F0F0E5C
:100B70000E0D0D0C0C0B0A0A0909080807070606DA
:100B8000050504040303020201000000009643006F
:100B9000005C4300009643000000000000000000DD
:100BA00000000053657474696E67732053746F722C
:100BB000656400454550524F4D20496E6974696126
:100BC0006C697A65640A0000803B4400803B440005
:100BD000002041000096420000A0420000A0420018
:100BE00000C8430000BE42D0070000D007000064E8
:100BF0000000004B000000434F4D4D554E4943410E
:100C000054494F4E0044525952554E004552524F8E
:100C1000525300494E464F004543484F00486F74B9
:100C2000656E642049646C652054696D656F7574E8
:100C300000486F74656E642049646C652054696D6A
:100C4000656F75740A002121204B494C4C2063616B
:100C50007573656420627920746F6F206D756368A9
:100C600020696E6163746976652074696D65202DF5
:100C70002063757272656E7420636F6D6D616E6452
:100C80003A200053544F505045442E200050726972
:100C90006E7465722073746F70706564206475651E
:100CA00020746F206572726F72732E2046697820EF
:100CB000746865206572726F7220616E642075734E
:100CC00065204D39393920746F20726573746172F3
:100CD000742E202854656D7065726174757265207C
:100CE00069732072657365742E205365742069746E
:100CF0002061667465722072657374617274696EC6
:100D000067290A004E6F20436865636B73756D2019
:100D100077697468206C696E65206E756D626572A6
:100D20002C204C617374204C696E653A2000636816
:100D300065636B73756D206D69736D617463682C89
:100D4000204C617374204C696E653A20004C696ECA
:100D500065204E756D626572206973206E6F742018
:100D60004C617374204C696E65204E756D626572BE
:100D70002B312C204C617374204C696E653A200035
:100D80004D3131300053657269616C207374617448
:100D90007573206D69736D617463680A00776169AA
:100DA000740A00506C656173652052657365740048
:100DB0005052494E5445522048414C544544002518
:100DC000533A20255300706F7765726F6666004B4B
:100DD000494C4C45442E20005072696E7465722057
:100DE00068616C7465642E206B696C6C28292063C3
:100DF000616C6C6564210A0053544F505045442E79
:100E000020005072696E7465722073746F70706523
:100E1000642064756520746F206572726F72732E22
:100E20002046697820746865206572726F7220614F
:100E30006E6420757365204D39393920746F2072C6
:100E40006573746172742E202854656D70657261CB
:100E5000747572652069732072657365742E2053F2
:100E6000657420697420616674657220726573749C
:100E7000617274696E67290A006563686F3A00459C
:100E800072726F723A0042696C696E656172204CD1
:100E90006576656C696E6720477269643A0A00215D
:100EA000212053544F502063616C6C65642062654F
:100EB0006361757365206F6620424C546F7563687B
:100EC000206572726F72202D207265737461727466
:100ED0002077697468204D3939390A00212120535F
:100EE000544F502063616C6C65642062656361756A
:100EF0007365206F6620424C546F7563682065727D
:100F0000726F72202D20726573746172742077691C
:100F10007468204D3939390A002F2F616374696F65
:100F20006E3A0073746172740050726F62696E671A
:100F300020506F696E740025532025692F256900A4
:100F40002E0A002F0050726F62696E67206D657304
:100F50006820706F696E74200020284452595255E1
:100F60004E2900473239204175746F204265642054
:100F70004C6576656C696E67003F20284C2C522CBE
:100F8000462C4229206F7574206F6620626F756E43
:100F900064732E0A003F2856296572626F736520BC
:100FA0006C6576656C20696D706C61757369626CD7
:100FB000652028302D34292E0A00426164205A20F1
:100FC00076616C75650A004E6F2062696C696E65AA
:100FD000617220677269640A0020496E76616C69EB
:100FE000642065787472756465722000536C656561
:100FF000702E2E2E005A2050726F62652050617341
:1010000074204265640A005A2050726F6265205055
:1010100061737420426564004732384C3000205AB6
:101020003A200020593A200042656420583A2000B6
:101030004D65736820706F696E74206F7574206FD2
:10104000662072616E67650A004D302053746F70C0
:10105000004D312053746F7000436F6E74696E756C
:101060006500436C69636B20746F20526573756D06
:10107000652E2E2E004E6F204D6F76652E00256951
:10108000730025696D20256973002569682025692D
:101090006D2025697300256964202569682025690C
:1010A0006D202569730025697920256964202569EB
:1010B000682025696D20256973005072696E74205F
:1010C00074696D653A20006F6B006F666600180CDE
:1010D000130C0C0C050CF70B44454255473A004DD8
:1010E000696E69205375506552204F46462E002088
:1010F0004500204D39322058004649524D57415243
:10110000455F4E414D453A4D61726C696E20322EFD
:10111000302E375F4457372E3320544D3344204D03
:10112000534D4442422028417072203234203230E4
:1011300032312032313A32343A34322920534F5549
:101140005243455F434F44455F55524C3A6874746F
:1011500070733A2F2F6769746875622E636F6D2FF5
:10116000496E73616E6974794175746F6D617469EC
:101170006F6E2F4D61726C696E2F747265652F43AF
:101180007265616C6974794477696E5F322E3020C4
:1011900050524F544F434F4C5F56455253494F4E58
:1011A0003A312E30204D414348494E455F54595005
:1011B000453A4D696E692053755065522045585423
:1011C00052554445525F434F554E543A3120555580
:1011D00049443A63656465326132662D3431613267
:1011E0002D343734382D396231322D63353563363D
:1011F000326633363766660A002F2F004D3134359C
:1012000020533C696E6465783E206F7574206F666C
:101210002072616E67652028302D31290A00205424
:1012200000205200416363656C65726174696F6E82
:101230003A2050005741524E494E4721204C6F777B
:10124000205A204A65726B206D6179206C6561645B
:1012500020746F20756E77616E746564207061759F
:101260007365732E0A004D32303620580020580026
:1012700020204D61783A2000200020204D696E3AF0
:101280002000536F667420656E6473746F70733AD8
:10129000200046523A0020466C6F773A20003A20F0
:1012A0000020536572766F2000206F7574206F6682
:1012B0002072616E67650A00536572766F20005078
:1012C000726F6265204F6666736574205A005072B3
:1012D0006F6265204F6666736574205A0020643A19
:1012E0000020693A0020703A00496E76616C6964AA
:1012F0002065787472756465720A0020643A002073
:10130000693A0020703A0064697300656E004329F1
:101310000A0061626C656420286D696E2074656DD9
:10132000702000436F6C6420657874727564657317
:101330002061726520004F4646004F4E00426564B2
:10134000204C6576656C696E6720004661696C6546
:101350006420746F20656E61626C65204265642054
:101360004C6576656C696E670A00496E76616C69DA
:1013700064206D6573682E0A004D34323120696E29
:10138000636F727265637420706172616D657465FC
:10139000722075736167650A004D65736820706F10
:1013A000696E74206F7574206F662072616E676558
:1013B0000A004F666673657473204170706C6965CE
:1013C00064004572723A20546F6F2066617221008A
:1013D000546F6F206661722066726F6D2072656651
:1013E0006572656E636520706F696E740A004545AD
:1013F00050524F4D204F4B0A00290A0020746F2095
:10140000003F5A206F7574206F662072616E6765A9
:10141000202800290A0020746F20003F59206F7592
:1014200074206F662072616E676520282D00290A7E
:101430000020746F20003F58206F7574206F662065
:1014400072616E676520282D00205A0020590050D7
:10145000726F6265204F6666736574205800496E2E
:1014600076616C69642065787472756465720A00CF
:101470002042002050006F6B0020573A00436F6FEE
:101480006C696E672E2E2E0048656174696E672E3A
:101490002E2E00452025530020573A004265642037
:1014A000436F6F6C696E672E2E2E00426564204874
:1014B000656174696E672E2E2E0023646566696E01
:1014C000652044454641554C545F00626564004BBD
:1014D0006420004B6920004B70200050494420419B
:1014E00075746F74756E652066696E69736865647E
:1014F000212050757420746865206C617374204BD2
:10150000702C204B6920616E64204B6420636F6EE9
:101510007374616E74732066726F6D2062656C6F98
:101520007720696E746F20436F6E666967757261AC
:1015300074696F6E2E680A00504944204175746FBB
:1015400074756E65206661696C6564212074696DCF
:10155000656F75740A00504944204175746F747545
:101560006E65206661696C6564212054656D7065E7
:1015700072617475726520746F6F20686967680A9C
:1015800000204B643A2000204B693A2000204B7029
:101590003A200020436C61737369632050494420F2
:1015A0000A00204E6F206F76657273686F6F740A41
:1015B000002054753A2000204B753A2000206D61C0
:1015C000783A2000206D696E3A200020643A2000AD
:1015D00020626961733A2000504944204175746F5C
:1015E00074756E652073746172740A0050494420EA
:1015F0004175746F74756E65206661696C656421F0
:101600002054656D706572617475726520746F6FBA
:1016100020686967680A00504944204175746F74F6
:10162000756E6500504944204175746F74756E6520
:10163000206661696C65642120426164206865618F
:101640007465722069640A004572723A2075746686
:101650003820666F6E74206E6F7420696E697469CD
:10166000616C697A65642E004572723A2075746601
:101670003820666F6E74206E6F7420696E697469AD
:10168000616C697A65642E004572723A20757466E1
:101690003820666F6E74206E6F7420696E6974698D
:1016A000616C697A65642E00000C0F00FE0702254C
:1016B00003BB017FFE08FE08FE0508080600004087
:1016C000F0C88888987810050808060000C0F888D7
:1016D00088888888F80505050600012030F8302044
:1016E0000508080600002070F820202020E00509E9
:1016F000090600FF2070A8A8B88888702007050593
:10170000070001D86C366CD80509090600FFF8A857
:101710008888888888A8F8050A0A0600FE205050A4
:10172000505088A8A8887003030306000340A04017
:10173000FFFFFFFFFFFFFFFFFFFFFFFFFFFFFFFFB9
:10174000FFFFFFFFFFFF0000000605FF0107070680
:10175000020080808080800080030303060105A0D2
:10176000A0A005060606000050F85050F8500509E4
:10177000090600FF2070A8A07028A87020050707A0
:10178000060000C8C810204098980507070600000A
:1017900040A0A040A8906801030306020580808055
:1017A0000309090601FF204040808080404020035B
:1017B00009090601FF8040402020204040800507A5
:1017C0000706000020A8702070A820050505060067
:1017D000012020F820200203030601FFC0408005FD
:1017E0000101060003F8020202060100C0C005075D
:1017F000070600000810102040408005070706007B
:1018000000708898A8C8887003070706010040C0C8
:1018100040404040E005070706000070880810209F
:1018200040F8050707060000F80810300888700522
:10183000070706000010305090F810100507070643
:101840000000F880F00808887005070706000030DF
:101850004080F0888870050707060000F80810101F
:10186000202020050707060000708888708888708F
:1018700005070706000070888878081060020505D3
:10188000060100C0C000C0C00206060601FFC0C0BD
:1018900000C040800305050601012040804020056E
:1018A0000303060002F800F8030505060101804065
:1018B00020408005070706000070881020200020C7
:1018C0000507070600007088B8A8B88070050707EC
:1018D000060000708888F8888888050707060000D9
:1018E000F04848704848F0050707060000708880F7
:1018F00080808870050707060000F048484848487F
:10190000F0050707060000F88080F08080F80507E2
:1019100007060000F88080F0808080050707060039
:101920000070888080988870050707060000888806
:1019300088F8888888030707060100E04040404097
:1019400040E00507070600003810101010906005F1
:1019500007070600008890A0C0A09088050707062A
:101960000000808080808080F805070706000088DE
:10197000D8A8888888880507070600008888C8A82E
:10198000988888050707060000708888888888700E
:10199000050707060000F08888F0808080050707AB
:1019A00006000070888888A8906805070706000070
:1019B000F08888F0A09088050707060000708880EE
:1019C00070088870050707060000F82020202020F6
:1019D0002005070706000088888888888870050722
:1019E00007060000888888885050200507070600F1
:1019F0000088888888A8A8500507070600008888FE
:101A0000502050888805070706000088885020204D
:101A10002020050707060000F80810204080F80382
:101A200009090601FFE080808080808080E0050752
:101A30000706000080404020101008030909060135
:101A4000FFE020202020202020E0050303060005E1
:101A50002050880501010600FEF803030306010576
:101A60008040200505050600007008788878050785
:101A7000070600008080F0888888F00505050600CC
:101A800000708080887005070706000008087888C5
:101A90008888780505050600007088F080700507C5
:101AA00007060000304840E04040400507070600B8
:101AB000FE70888888780870050707060000808017
:101AC000F0888888880307070601004000C040406E
:101AD00040E00409090601FE1000301010101090BB
:101AE0006005070706000080808890E09088030763
:101AF00007060100C04040404040E00505050600E3
:101B000000D0A8A8A8A8050505060000B0C88888C8
:101B10008805050506000070888888700507070697
:101B200000FEF0888888F080800507070600FE78B0
:101B3000888888780808050505060000B0C88080F8
:101B40008005050506000078807008F00507070687
:101B500000002020F8202020180505050600008838
:101B60008888986805050506000088888850200543
:101B700005050600008888A8A85005050506000090
:101B800088502050880507070600FE888888502066
:101B90004080050505060000F8102040F8030909FB
:101BA0000601FF20404040804040402001090906D6
:101BB00002FF808080808080808080030909060188
:101BC000FF80404040204040408005030306000263
:101BD00048A890FF24F4D43050C38E20C2A24017EE
:101BE000828B7011127A910D816CD90AA861E1087B
:101BF000C7586607615143061E4B5D05C145A704E2
:101C00001A411104093D9803713931034036DB0252
:101C100065339102D4305402802E1D02632CEE01F4
:101C2000752AC501B028A001102781018F25640104
:101C30002B244B01E0223401AC211F018D200D012A
:101C4000801FFC00841EED00971DDF00B81CD20031
:101C5000E61BC600201BBC00641AB200B219A80023
:101C60000A19A0006A189900D117910040178B003B
:101C7000B516840031167E00B31579003A1573004D
:101C8000C7146F0058146A00EE13660088136300CF
:101C900025135E00C7125B006C125700151254002A
:101CA000C111510070114F0021114B00D610490095
:101CB0008D1047004610440002104200C00F400043
:101CC000800F3E00420F3C00060F3B00CB0E380059
:101CD000930E37005C0E3500270E3400F30D3200F2
:101CE000C10D3100900D3000600D2E00320D2D0021
:101CF000050D2C00D90C2B00AE0C2900850C2900F9
:101D00005C0C2700350C27000E0C2600E80B240085
:101D1000C40B2400A00B23007D0B23005A0B2100D1
:101D2000390B2100180B2000F80A1F00D90A1E00E9
:101D3000BB0A1E009D0A1D00800A1D00630A1C00CC
:101D4000470A1B002C0A1B00110A1A00F7091A0087
:101D5000DD091900C4091900AB091900920917001F
:101D60007B091800630917004C0916003609160094
:101D7000200916000A091500F5081500E0081400EE
:101D8000CC081400B8081400A4081400900813002C
:101D90007D0812006B081300580812004608120054
:101DA0003408110023081100120811000108110065
:101DB000F0071000E0071000D0071000C007100067
:101DC000B0070F00A107100091070E0083070F0056
:101DD00074070F0065070E0057070E0049070E0035
:101DE0003B070D002E070E0020070D0013070D0006
:101DF00006070D00F9060C00ED060D00E0060C00CC
:101E0000D4060C00C8060C00BC060C00B0060C0082
:101E1000A4060B0099060C008D060B0082060B0031
:101E200077060B006C060B0061060A0057060B00D4
:101E30004C060A0042060A0038060A002E060A006E
:101E400024060A001A060A001006090007060A00FE
:101E5000FD050900F4050900EB050900E20509008C
:101E6000D9050900D0050900C7050900BE0509000C
:101E7000B5050800AD050800A50509009C0508008A
:101E8000940508008C050800840508007C050800FE
:101E9000740508006C050700650508005D0507006E
:101EA000560508004E0507004705070040050800D5
:101EB00038050700310507002A050700230507003C
:101EC0001C050600160507000F050700080506009B
:101ED00002050700FB040600F5040700EE040600F7
:101EE000E8040600E2040700DB040600D50406004F
:101EF000CF040600C9040600C3040600BD040600A2
:101F0000B7040600B1040500AC040600A6040600F0
:101F1000A00405009B04060095040500900406003B
:101F20008A04050085040500800406007A04050083
:101F300075040500700405006B04050066040500C7
:101F4000610405005C040500570405005204050007
:101F50004D04050048040500430405003E04040048
:101F60003A04050035040500300404002C04050083
:101F700027040400230405001E0404001A040400BE
:101F800016040500110404000D04040009040500F2
:101F90000404040000040400FC030400F80304002B
:101FA000F4030400F0030400EC030400E80304005D
:101FB000E4030400E0030400DC030400D80304008D
:101FC000D4030400D0030400CC030400C8030300BE
:101FD000C503030024F404D9201BC40C5C0E980430
:101FE000C4095F0265077101F405F900FB04B30041
:101FF00048048700C10369005803550003034500E6
:10200000BE023A008402310053022A002902250050
:1020100004022000E4011C00C8011900AF011700F0
:102020009801140084011300710110006101100077
:1020300051010E0043010D0036010B002B010B0076
:1020400020010B00150109000C0109000301080023
:10205000FB000800F3000800EB000700E4000600A6
:10206000DE000600D8000600D2000600CC00050005
:10207000C7000500C2000500BD000400B90004004F
:10208000B5000400B1000400AD000400A900040084
:10209000A5000300A20003009F0004009B000300B2
:1020A00098000300950002009300030090000300D5
:1020B0008D0002008B0003008800020086000200F1
:1020C00084000300810002007F0002007D00020006
:1020D0007B00020079000200770001007600020018
:1020E0007400020072000100710002006F00020023
:1020F0006D0001006C0002006A000100690002002E
:102100006700010066000100650001006400020034
:102110006200010061000100600001005F00020038
:102120005D0001005C0001005B0001005A0001003D
:10213000590001005800010057000100560001003D
:10214000550001005400010053000000530001003D
:102150005200010051000100500001004F00010039
:102160004E0000004E0001004D0001004C00010037
:102170004B0000004B0001004A0001004900010033
:102180004800000048000100470001004600000030
:102190004600010045000000450001004400010028
:1021A0004300000043000100420000004200010023
:1021B0004100000041000100400001003F0000001C
:1021C0003F0001003E0000003E0001003D00000015
:1021D0003D0001003C0000003C0000003C0001000C
:1021E0003B0000003B0001003A0000003A00010003
:1021F00039000000390001003800000038000000FC
:1022000038000100370000003700010036000000F0
:1022100036000000360001003500000035000000E7
:1022200035000100340000003400000034000100DB
:1022300033000000330000003300010032000000D2
:1022400032000000320001003100000031000000C7
:1022500031000100300000003000000030000100BB
:102260002F0000002F0000002F0000002F000100B1
:102270002E0000002E0000002E0001002D000000A6
:102280002D0000002D0000002D0001002C0000009A
:102290002C0000002C0000002C0001002B0000008E
:1022A0002B0000002B0000002B0001002A00000082
:1022B0002A0000002A0000002A0001002900000076
:1022C0002900000029000000290000002900010069
:1022D000280000002800000028000000280000005E
:1022E0002800010027000000270000002700000050
:1022F0002700000027000100260000002600000043
:102300002600000026000000260001002500000035
:102310002500000025000000250000002500000029
:10232000250001002400000024000000240000001B
:10233000240000002400010023000000230000000E
:102340002300000023000000230000002300000001
:1023500023000100220000002200000022000000F3
:1023600022000000220000002200010021000000E5
:1023700021000000210000002100000021000000D9
:1023800021000000210001002000000020000000CA
:1023900020000000200000002000000020000000BD
:1023A00020000000200001001F0000001F000000AE
:1023B0001F0000001F0000001F0000001F000000A1
:1023C0001F0001001E0000001E0000001E00000093
:1023D0001E0000003930000033250000871900007E
:1023E000B00F0000DB080000BD0400007402000014
:1023F0003F01000020436F756E7420583A0042651B
:102400006400453100626564002C20737973746543
:102410006D2073746F707065642120486561746508
:10242000725F49443A200048656174696E672046CE
:1024300061696C65640048656174696E67206661F6
:10244000696C6564004D3131322053687574646F76
:10245000776E001000C90210012C014001220170AA
:10246000011801B0010E01F00104015002FA00B0A0
:1024700002F0003003E600D003DC009004D20070CC
:1024800005C800A006BE000008B400B009AA00D02C
:102490000BA000600E960060118C000015820020D9
:1024A000197800C01D6E00A0226400B0275A009069
:1024B0002C500000314600E0343C001038320090CF
:1024C0003A2800603C1E00A03D1400803E0A002017
:1024D0003F0000544845524D414C2052554E415703
:1024E000415900546865726D616C2052756E617758
:1024F0006179004572723A204D415854454D500063
:102500004D415854454D5020747269676765726536
:1025100064004572723A204D494E54454D50004D6D
:10252000494E54454D502074726967676572656401
:1025300000202F002042403A0020403A006001F481
:10254000017001EA019001E001B001D601D001CC97
:10255000010002C2013002B8016002AE019002A483
:1025600001D0029A012003900170038601C0037C10
:102570000130047201A004680120055E01B0055419
:102580000160064A0120074001F0073601F0082CDF
:1025900001100A2201500B1801C00C0E01500E044C
:1025A000013010FA002012F0005014E600C016DCD2
:1025B000007019D200501CC800501FBE007022B419
:1025C00000B025AA00F028A000202C9600302F8C07
:1025D0000010328200A0347800F0366E00E03864DB
:1025E00000803A5A00403B5500E03B5000F03C462A
:1025F00000C03D3C00603E3200E03E2800303F1EFF
:1026000000503F1900703F1400A03F0A00C03F0077
:1026100000D03FF6FFE03FECFF2020506C616E6E73
:10262000657242756666657242797465733A200018
:102630002046726565204D656D6F72793A200043C2
:102640006F6D70696C65643A20417072203234207D
:10265000323032310A00204C61737420557064614D
:102660007465643A20323032312D30342D313820C7
:102670007C20417574686F723A2054696E794D619F
:102680006368696E657333440A00322E302E375FFB
:102690004457372E330A004D61726C696E00205327
:1026A0006F6674776172652052657365740A0020E5
:1026B0005761746368646F672052657365740A00BC
:1026C0002042726F776E206F757420526573657447
:1026D0000A002045787465726E616C2052657365DE
:1026E000740A00506F77657255700A0073746172D6
:1026F000740A00456E6473746F707300255320254F
:102700006320256320256320256300205A3A00209A
:10271000593A0020583A00656E6473746F707320E4
:102720006869743A2000000000010200090A0000F4
:102730000000040308070000000000000000000083
:10274000000000000000004D6F76652025736D6D60
:10275000004D6F766520302E316D6D004D6F7665C2
:1027600020316D6D004D6F76652031306D6D004DFF
:102770006F76652041786973004578747275646579
:1027800072004D6F7665205A004D6F7665205900B6
:102790004D6F7665205800FFFFFF50726F62696EC3
:1027A00067204661696C65640A0050726F62696EE9
:1027B00067204661696C656400205A3A2000205900
:1027C0003A200042656420583A200073686F770011
:1027D000627574746F6E0070726F6D70745F0065F7
:1027E0006E6400626567696E00220A00556E6B6E4A
:1027F0006F776E20636F6D6D616E643A2022004DBD
:10280000696E692053755065522052656164792E56
:10281000005072696E74696E672E2E2E00507269B8
:102820006E74205061757365640020453A00205A2B
:102830003A0020593A00583A004572726F72207778
:10284000726974696E6720746F20454550524F4D10
:10285000210A0020746F6F206C6F6E67206578749A
:10286000727573696F6E2070726576656E746564DB
:102870000A0020636F6C6420657874727573696FE9
:102880006E2070726576656E7465640A00526573B9
:10289000656E643A200000002200250028002B000D
:1028A00000002100240027002A0002020202020286
:1028B00002020404040404040404030303030303E2
:1028C00003030101010101010101010204081020BB
:1028D00040800102040810204080010204081020FA
:1028E0004080804020100804020180D811241FBEBF
:1028F000CFEFD0E4DEBFCDBF12E0A0E0B1E0E8EB67
:10290000F5ED01E00BBF02C007900D92A832B107B0
:10291000D9F724E1A8E2B2E001C01D92AA3AB207B9
:10292000E1F714E1C6E7D4E104C02197FE010E945B
:1029300082E8C537D107C9F70E941FD90C94DAEA9B
:102940000C9400009F92AF92BF92CF92DF92EF92D1
:10295000FF920F931F93CF93DF9300D000D01F926D
:10296000CDB7DEB7EBE8FAE00027BB27462F572F9D
:10297000A82FAA2341F4A52F542FB85FAA2319F436
:10298000A52F5527B85FA03138F45295A295452F51
:102990004F70507FA42BBC5FA03428F4550FAA1FA2
:1029A000550FAA1FBE5FA03818F4550FAA1FB39584
:1029B000550FAA1FEA0FF01F449151E0AA27B85003
:1029C00081F1C8F0B0FF02C0440F551FB1FF04C031
:1029D000440F551F440F551FB2FF06C05295429534
:1029E000142F1F70407F512BB3FF1BC0A52F542FF6
:1029F00044270C941115B195B0FF02C05595479529
:102A0000B1FF04C05595479555954795B2FF05C050
:102A10005295407F4295452B5F70B3FF02C0452F12
:102A20005527DD24CC24BB24B2E0649FD018C10814
:102A3000B00AB00B749FC018B108B00B849FB018D7
:102A4000B109659FC018B108B00B759FB018B109E6
:102A5000859FB0196A9FB018B1097A9FB0194D9D32
:102A6000A12C99243327992722275D9DA00C911C26
:102A7000301F901F201FAD9D900C311D901F201FF7
:102A80004C9DA00C911C301F901F201F5C9D900C32
:102A9000311D901F201FAC9D300D911D201F4B9D9F
:102AA000900C311D901F201F5B9D300D911D201F2C
:102AB000AB9D900D211D4B9F300D911D201F5B9FE5
:102AC000900D211DAB9F200DB1E0BB24CC24DD2453
:102AD000639FD018C108B00AB00B739FC018B1082B
:102AE000B00B839FB018B109699FC018B108B00B33
:102AF000799FB018B109899FB019629FB018B109C8
:102B0000729FB019D61AC70AB80A20F0B1E03B0F7D
:102B1000901F201F1124792F632F90E0822F0F9098
:102B20000F900F900F900F90DF91CF911F910F9109
:102B3000FF90EF90DF90CF90BF90AF909F9008955F
:102B4000CF92DF92EF92FF9280918002882309F466
:102B500057C0C0907C02D0907D02E0907E02F09041
:102B60007F0220E030E0A901C701B6010E9495E193
:102B7000882309F445C020E030E040E05FE3C7016E
:102B8000B6010E94FBE19B01AC010E94FBE12BED31
:102B90003FE049E450E40E94FBE19B01AC0160E0AE
:102BA00070E080E89FE30E940FE96B017C01C09216
:102BB0007702D0927802E0927902F0927A026091E4
:102BC000240170912501072E000C880B990B0E949F
:102BD0009CE12AE037ED43E25CE30E94FBE1A701C0
:102BE00096010E94FBE160936E0170936F018093E8
:102BF000700190937101FF90EF90DF90CF90089556
:102C0000C12CD12C80E8E82E8FE3F82ED0CFCF92C4
:102C1000DF92EF92FF92FC01C080D180E280F380CE
:102C200020E030E0A901C701B6010E9495E187FFCD
:102C300068C0C701B601905820E030E040E251E49E
:102C40000E94FBE120E030E040EA50E40E948CE882
:102C500020E030E040E251E40E940FE90E9481E967
:102C60009B0160E22031F7E23F0730F0C90160E1EB
:102C700077E20E945AE8605D6093AA0B283E83E0E9
:102C8000380708F445C0C90168EE73E00E945AE8AD
:102C9000CB016AE070E00E945AE8805D8093AB0B44
:102CA00080E22436310558F0C90164E670E00E94E4
:102CB0005AE8CB016AE070E00E945AE8805D809398
:102CC000AC0B80E22A30310558F0EAE0F0E0C901AF
:102CD000BF010E945AE8CB01BF010E945AE8805D03
:102CE0008093AD0BC9016AE070E00E945AE8805DF4
:102CF0008093AE0B8AEA9BE0FF90EF90DF90CF903D
:102D0000089520E030E040E251E4C701B60198CFD9
:102D100080E2C4CF8F929F92AF92BF92CF92DF9208
:102D2000EF92FF92FC01C080D180E280F38020E02E
:102D300030E040E251E4C701B6010E94FBE120E02F
:102D400030E040E251E40E94FBE14B015C0120E0F5
:102D500030E0A901C701B6010E9495E120E030E012
:102D600040EA50E487FF04C020E030E040EA50EC45
:102D7000C501B4010E948CE820E030E040E251E45B
:102D80000E940FE90E9481E99B018BE237FF05C099
:102D900022273327261B370B8DE28093A90BC9010D
:102DA00068EE73E00E946EE8CB01EAE0F0E0BF015C
:102DB0000E946EE8805D8093AA0BC90164E670E012
:102DC0000E946EE8CB01BF010E946EE8805D809397
:102DD000AB0BC901BF010E946EE8282FCB01BF01D8
:102DE0000E946EE8805D8093AC0B8EE28093AD0B09
:102DF000205D2093AE0B89EA9BE0FF90EF90DF907F
:102E0000CF90BF90AF909F908F9008958F929F9298
:102E1000AF92BF92CF92DF92EF92FF92CF93FC01DD
:102E2000C080D180E280F38020E030E040E251E4D5
:102E3000C701B6010E94FBE120E030E048EC52E41B
:102E40000E94FBE14B015C0120E030E040E251ECEC
:102E5000C701B6010E9495E1181654F420E030E055
:102E600048EC52E4C701B6010E940FEA87FD86C014
:102E700020E030E0A901C701B6010E9495E187FF7B
:102E80006EC060E070E080EA90ECA50194010E94C1
:102E90008CE820E030E040E251E40E940FE90E941B
:102EA00081E96B017C01F7FC5FC020E137E240E083
:102EB00050E00E94FFE7CA01B9012AE030E040E09B
:102EC00050E00E94FFE7605D6093A90BC701B60167
:102ED00028EE33E040E050E00E94FFE79AE0892EC0
:102EE000912CA12CB12CCA01B901A50194010E9419
:102EF000FFE7605D6093AA0BC701B60124E630E0EE
:102F000040E050E00E94FFE7CA01B901A501940129
:102F10000E94FFE7605D6093AB0B8EE28093AC0B89
:102F2000C701B601A50194010E94FFE7C62FCA019F
:102F3000B901A50194010E94FFE7605D6093AD0BAC
:102F4000C05DC093AE0B89EA9BE0CF91FF90EF90FC
:102F5000DF90CF90BF90AF909F908F90089560E0EA
:102F600070E080EA90E491CFF094E094D094C09423
:102F7000C11CD11CE11CF11C6DE2A6CF20E030E0A9
:102F8000A901C701B6010E9495E187FF6AC060E010
:102F900070E080EA90ECA50194010E948CE820E0AA
:102FA00030E040E251E40E940FE90E9481E94B01C8
:102FB0005C0120E030E0A901C701B6010E940FEAE0
:102FC00087FD0BC020E030E040E251E4C701B601CC
:102FD0000E9495E160E287FD13C0B7FC47C0C501C0
:102FE000B40128EE33E040E050E00E94FFE7CA0160
:102FF000B9012AE030E040E050E00E94FFE7605D68
:103000006093AA0BC501B40124E630E040E050E033
:103010000E94FFE78AE0C82ED12CE12CF12CCA01D6
:10302000B901A70196010E94FFE7605D6093AB0BB9
:103030008EE28093AC0BC501B401A70196010E94FA
:10304000FFE7C62FCA01B901A70196010E94FFE759
:10305000605D6093AD0BC05DC093AE0B8AEA9BE0F0
:1030600074CF60E070E080EA90E495CFB094A094D3
:1030700090948094811C911CA11CB11C6DE2C0CF66
:103080009C0197FF26C0EE27FF27E81BF90B2D397F
:103090008FEF38070CF05DC08DE28093AB0BCF0152
:1030A00064E670E00E946EE8CB012AE030E0B901EE
:1030B0000E946EE8805D8093AC0BCF01B9010E9445
:1030C0006EE8CB01B9010E946EE8805D8093AD0B84
:1030D0002AC0283E83E03807B4F1C90168EE73E0E6
:1030E0000E946EE8CB01EAE0F0E0BF010E946EE8CA
:1030F000805D8093AB0BC90164E670E00E946EE8CE
:10310000CB01BF010E946EE8805D8093AC0BC901CA
:10311000BF010E946EE8CB01BF010E946EE8805D96
:103120008093AD0BF901CF016AE070E00E946EE878
:10313000805D8093AE0B8BEA9BE008958DE237FDB6
:10314000C5CF80E2C3CFF90180E2243631050CF00F
:10315000A4CF80E28093AB0B8093AC0BEA30F105F7
:103160006CF38DE237FF80E28093AC0BCF016AE015
:1031700070E00E946EE8605D6093AD0BD4CF9C015F
:1031800097FD2DC080E2243631055CF0C90164E66C
:1031900070E00E946EE8CB016AE070E00E946EE889
:1031A000805D8093AC0B80E22A3031055CF0EAE070
:1031B000F0E0C901BF010E946EE8CB01BF010E948F
:1031C0006EE8805D8093AD0BC9016AE070E00E94FB
:1031D0006EE8805D8093AE0B8CEA9BE0089531959C
:1031E000219531098DE2DDCF24E6829FC0011124B3
:1031F00081589F4F6FEF70E00E946EE8262F81E3A9
:10320000643609F080E28093AB0B90E22A3040F004
:103210003AE0822F632F0E9440E80E9440E8905DD0
:103220009093AC0B822F6AE00E9440E8905D9093EF
:10323000AD0B85E28093AE0B8BEA9BE00895609125
:10324000240170912501072E000C880B990B0E9418
:103250009CE12AE037ED43E25CE30E94FBE1209130
:103260007702309178024091790250917A020E945F
:10327000FBE160936E0170936F01809370019093F6
:10328000710108958091B60B811104C08091890B62
:1032900080930C0C0895CF93DF93EC01CB01BA011E
:1032A0000E949CE129EC38EC48EC5EE30E940FE9B7
:1032B00020E030E040E05FE30E948CE80E9488E973
:1032C0006883DF91CF9108950E949CE129EC38EC4E
:1032D00048EC5EE30E940FE920E030E040E05FE36D
:1032E0000E948CE80E9488E9862F0C94F418E091E3
:1032F000B60B86E0E802F0011124E958F44F809102
:10330000890B90E0958384830895CF93DF9300D059
:1033100000D0CDB7DEB70E9488E90E949AE16983A8
:103320007A838B839C83CE0101960E9407160F90AF
:103330000F900F900F90DF91CF9108958F929F92F1
:10334000AF92BF92CF92DF92EF92FF92CF936B0139
:103350007C0120E030E0A9010E9495E187FD9FC03B
:103360006DEB77E386E095E3A70196010E948CE878
:103370006B017C0120E030E040E251E40E94FBE17F
:1033800020E030E048EC52E40E94FBE14B015C019C
:1033900020E030E0A901C701B6010E9495E120E0DC
:1033A00030E040EA50E487FF04C020E030E040EA2B
:1033B00050ECC501B4010E948CE820E030E040E20E
:1033C00051E40E940FE90E9481E96B017C018BE2CC
:1033D000F7FE09C0F094E094D094C094C11CD11CB5
:1033E000E11CF11C8DE28093A80BC701B60120E11E
:1033F00037E240E050E00E94FFE78AE0882E912CFF
:10340000A12CB12CCA01B901A50194010E94FFE7CA
:10341000605D6093A90BC701B60128EE33E040E080
:1034200050E00E94FFE7CA01B901A50194010E9482
:10343000FFE7605D6093AA0BC701B60124E630E0A8
:1034400040E050E00E94FFE7CA01B901A5019401E4
:103450000E94FFE7605D6093AB0B8EE28093AC0B44
:10346000C701B601A50194010E94FFE7C62FCA015A
:10347000B901A50194010E94FFE7605D6093AD0B67
:10348000C05DC093AE0B88EA9BE0CF91FF90EF90B8
:10349000DF90CF90BF90AF909F908F9008956DEB8D
:1034A00077E386E095EB60CF8F929F92AF92BF92C9
:1034B000CF92DF92EF92FF926B017C0120E030E02F
:1034C000A9010E9495E187FD6BC06DEB77E386E073
:1034D00095E3A70196010E948CE86B017C0120E036
:1034E00030E040E251E40E94FBE120E030E040E2C5
:1034F00051E40E94FBE14B015C0120E030E0A901B6
:10350000C701B6010E9495E120E030E040EA50E4B6
:1035100087FF04C020E030E040EA50ECC501B40170
:103520000E948CE820E030E040E251E40E940FE984
:103530000E9481E99B018BE237FF05C022273327D8
:10354000261B370B8DE28093AA0BC90164E670E05D
:103550000E946EE8CB01EAE0F0E0BF010E946EE855
:10356000805D8093AB0BC901BF010E946EE8282FDC
:10357000CB01BF010E946EE8805D8093AC0B8EE2B0
:103580008093AD0B205D2093AE0B8AEA9BE0FF9009
:10359000EF90DF90CF90BF90AF909F908F90089565
:1035A0006DEB77E386E095EB94CF8F929F92AF928D
:1035B000BF92CF92DF92EF92FF92CF936B017C018B
:1035C00020E030E0A9010E9495E187FDAAC06DEBE3
:1035D00077E386E095E3A70196010E948CE86B01F2
:1035E0007C0120E030E0A9010E9495E187FF9EC0A8
:1035F000C701B601905820E030E040E251E40E945B
:10360000FBE120E030E040E251E40E94FBE120E0F9
:1036100030E040EA50E40E948CE820E030E040E2F4
:1036200051E40E940FE90E9481E96B017C0180E274
:103630008093A80B60E280E1C81687E2D806E10417
:10364000F1048CF0C701B60120E137E240E050E020
:103650000E94FFE7CA01B9012AE030E040E050E0F3
:103660000E94FFE7605D6093A90B60E288EEC816D8
:1036700083E0D806E104F1048CF0C701B60128EE1E
:1036800033E040E050E00E94FFE7CA01B9012AE0C0
:1036900030E040E050E00E94FFE7605D6093AA0BDD
:1036A00060E284E6C816D104E104F1048CF0C7019D
:1036B000B60124E630E040E050E00E94FFE7CA0196
:1036C000B9012AE030E040E050E00E94FFE7605D91
:1036D0006093AB0B8AE0882E912CA12CB12CC701F2
:1036E000B601A50194010E94FFE7C62FCA01B901E6
:1036F000A50194010E94FFE7605D6093AC0B8EE230
:103700008093AD0BC05DC093AE0B88EA9BE0CF9178
:10371000FF90EF90DF90CF90BF90AF909F908F90F1
:1037200008956DEB77E386E095EB55CF20E030E030
:1037300040E251E4C701B60162CFCF92DF92EF922F
:10374000FF92CF93DF9300D000D0CDB7DEB76B01EF
:103750007C0120E030E0A9010E9495E187FD1BC0BB
:103760006DEB77E386E095E3A70196010E948CE874
:1037700069837A838B839C83CE0101960E9407160E
:103780000F900F900F900F90DF91CF91FF90EF90DF
:10379000DF90CF9008956DEB77E386E095EBE4CF73
:1037A000CF92DF92EF92FF926B017C0120E030E03C
:1037B000A9010E9495E187FD26C06DEB77E386E0C5
:1037C00095E3A70196010E948CE86B017C0120E043
:1037D00030E0A9010E9495E120E030E040E05FE3A5
:1037E00087FF04C020E030E040E05FEBC701B60196
:1037F0000E948CE80E9481E9CB01FF90EF90DF905E
:10380000CF900C94BF186DEB77E386E095EBD9CFA2
:10381000CF93DF93EC01CB01BA010E949CE120E041
:1038200030E040E251E40E940FE920E030E0A901DD
:103830000E948CE8688379838A839B83DF91CF9190
:103840000895CF93DF93EC01CB01BA010E949CE174
:1038500020E030E040E251E40E940FE920E030E057
:10386000A9010E948CE8688379838A839B83DF9116
:10387000CF9108950E949CE120E030E040E251E4C5
:103880000E940FE920E030E0A9010E948CE80C942E
:10389000D51A0E949CE120E030E040E251E40E9411
:1038A0000FE920E030E0A9010E948CE80C94541A42
:1038B000CF93DF93EC01CB01BA010E949CE120E0A1
:1038C00030E048EC52E40E940FE920E030E0A9012A
:1038D0000E948CE8688379838A839B83DF91CF91F0
:1038E0000895CF93DF93EC01CB01BA010E949CE1D4
:1038F00020E030E048EC52E40E940FE920E030E0A4
:10390000A9010E948CE8688379838A839B83DF9175
:10391000CF9108950E949CE120E030E048EC52E411
:103920000E940FE920E030E0A9010E948CE80C948D
:103930009E19CF93DF93EC01CB01BA010E949CE169
:1039400020E030E0A9010E948CE8688379838A83B3
:103950009B83DF91CF910895CF93DF93EC01CB014F
:10396000BA010E949CE120E030E0A9010E948CE8AD
:10397000688379838A839B83DF91CF9108950E9426
:103980009CE120E030E0A9010E948CE80C94D01B5F
:10399000CF93DF93EC01CB01BA010E949CE12AE0B6
:1039A00037ED43E25DE30E940FE920E030E0A9013A
:1039B0000E948CE80E9488E9688379838A839B83CC
:1039C000DF91CF9108950E949CE12AE037ED43E218
:1039D0005DE30E940FE920E030E0A9010E948CE83D
:1039E0000C948519CF93DF93EC01CB01BA010E94AF
:1039F0009CE12AE037ED43E25DE30E940FE920E01D
:103A000030E0A9010E948CE8688379838A839B83D4
:103A1000DF91CF9108950E949CE12AE037ED43E2C7
:103A20005DE30E940FE920E030E0A9010E948CE8EC
:103A30000C949D1B0E949CE120E030E0A9010E94B3
:103A40008CE80C949D1BCF92DF92EF92FF92CF9364
:103A5000DF9300D000D0CDB7DEB70E949CE120E01C
:103A600030E048EC52E40E940FE920E030E0A90188
:103A70000E948CE86B017C0120E030E0A9010E94EB
:103A800095E12DEB37E346E055E387FF04C02DEBCE
:103A900037E346E055EBC701B6010E948CE8698325
:103AA0007A838B839C83CE0101960E9406170F9028
:103AB0000F900F900F90DF91CF91FF90EF90DF90DC
:103AC000CF900895CF93DF93EC01CB01BA010E9410
:103AD0009CE120E030E0A9010E948CE80E9481E98D
:103AE00079836883DF91CF9108950E949CE120E063
:103AF00030E0A9010E948CE80E9481E9CB010C947E
:103B0000BF18CF93DF93EC01CB01BA010E949CE177
:103B100020E030E04AE754E40E940FE920E030E082
:103B2000A9010E948CE8688379838A839B83DF9153
:103B3000CF9108958091561390915713891B8F70E0
:103B400039F481E09091C50B913019F080E008952F
:103B500081E00895FC0184910895FC01808108951D
:103B600090917B0281E089270C9451724091F5027B
:103B700021E042276CE070E00C946CB54091F502B6
:103B800021E0422764E070E00C946CB54091F502AE
:103B900021E0422761E070E00C946CB54091F502A1
:103BA00021E0422762E070E00C946CB54091F50290
:103BB00021E0422761E070E00C946CB54091F50281
:103BC00021E0422768E070E00C946CB54091F5026A
:103BD00021E042276CE070E00C946CB541E061E0BC
:103BE00070E00C946CB54091F50221E042270C94F2
:103BF0006CB562E070E00C94E8BE6CE070E00C9490
:103C0000E8BE64E070E00C94E8BE61E070E00C9403
:103C1000E8BE61E070E00C94E8BE6CE070E00C94EB
:103C2000E8BE0C945CBF0C945CBFCF93DF93809193
:103C3000561390915713891B80958F7019F40E9429
:103C4000C47DF5CF809156138F5F8F70A09156136E
:103C50009BE5A99FD0011124FD01E05EF34FEF0128
:103C600019929A95E9F798E09083AB5CB34F90E195
:103C7000E8E5F3E101900D929A95E1F72091561352
:103C800090915713291303C094E690935313809394
:103C90005613DF91CF910C944073CF92DF92EF9245
:103CA000FF920F931F93C12CD12C76018C0120EE33
:103CB0003BE04CED5BE068ED7BE084ED9BE00E9437
:103CC000C4B41F910F91FF90EF90DF90CF900895B3
:103CD0008F929F92AF92BF92EF92FF920F931F939A
:103CE000CF93DF93EC018B01E42EF22E80916813C9
:103CF000909169138C179D0709F43EC020915502DD
:103D000027FD1092550228E5C130D20709F03FC0C7
:103D1000895D9D4571F40E9450BF6E517B4F8F4F5E
:103D20009F4F60937A0470937B0480937C049093FC
:103D30007D04D0936913C093681330E020E00093B2
:103D4000970B1093980B2093990B30939A0BE0925A
:103D5000900BF092910BC95DDD4521F410928F0B11
:103D60001092790482E08093650181E08093A70B33
:103D70001092780410928E0BDF91CF911F910F91CA
:103D8000FF90EF90BF90AF909F908F9008952DE59A
:103D9000C93DD20771F68150984519F0C9EDDDE5AE
:103DA000C8CF0E9450BF80907A0490907B04A0906E
:103DB0007C04B0907D04681979098A099B0997FFF2
:103DC000EDCF8091B90B8770873041F7CAE8DFE407
:103DD000B0CF20E040E070E060E081E190E20C9440
:103DE000681E80911D0C811114C080917201909108
:103DF0007301019720910A1330910B13281739078B
:103E000044F420E040E070E060E086E190E20C9451
:103E1000681E0C94E91E21E020938F0BFC01808129
:103E20009181A281B3818093120190931301A09399
:103E30001401B093150120E040E070E060E0809153
:103E4000870B9091880B0C94681ECF93DF9300D062
:103E500000D0CDB7DEB78DEC9CECACECBCE3898335
:103E60009A83AB83BC83CE0101960E940B1F0F90F7
:103E70000F900F900F90DF91CF910895CF93DF9324
:103E800000D000D0CDB7DEB78DEC9CECACECBDE340
:103E900089839A83AB83BC83CE0101960E940B1F5A
:103EA0000F900F900F900F90DF91CF910895CF93C7
:103EB000DF9300D000D0CDB7DEB780E090E0A0E87F
:103EC000BFE389839A83AB83BC83CE0101960E94B2
:103ED0000B1F0F900F900F900F90DF91CF910895CF
:103EE000CF93DF9300D000D0CDB7DEB780E090E075
:103EF000A0E2B1E489839A83AB83BC83CE010196AF
:103F00000E940B1F0F900F900F900F90DF91CF9199
:103F10000895CF92DF92EF92FF92CF93C82F0E9425
:103F200050BF6B017C0124EA30E74DE75FE360910D
:103F300012017091130180911401909115010E945A
:103F400095E187FD18C08AEF90E0A0E0B0E08C0D0D
:103F50009D1DAE1DBF1D8093290490932A04A0933C
:103F60002B04B0932C04C0931001CF91FF90EF90DD
:103F7000DF90CF90089580E090E0DC01E8CFCF9310
:103F8000DF9300D000D0CDB7DEB784EF91E0A0E0A2
:103F9000B0E089839A83AB83BC83BE016F5F7F4FA0
:103FA00088E70E949B740F900F900F900F90DF9105
:103FB000CF910895CF93C82FCB010E9491768BE0CB
:103FC00098E00E9491768CEF97E0CC2311F081E08D
:103FD00098E00E9491768AE0CF910C94E575CF939A
:103FE000DF93CDB7DEB720E24F8158856E818D819A
:103FF0000E94B4B9DF91CF9108956FEF8091890B42
:104000000C94FCBF6AEF7EE382E00C9467D66FEFFE
:104010007EE381E00C9467D664E07FE380E00C945B
:1040200067D669E07FE383E00C9467D6EF92FF9256
:104030000F931F9380EFE82E86E0F82E02EF16E034
:1040400024E23DE349EE5EE162E077E087E097E05D
:104050000E9401C11F910F91FF90EF900895EF9280
:10406000FF920F931F9384E7E82E86E0F82E0DEC65
:1040700016E024E23DE344E35AE566E776E08BE7A9
:1040800096E00E9401C11F910F91FF90EF9008955B
:10409000EF92FF920F931F938AE2E82E84E0F82EAE
:1040A0000DE314E030E020E042EC57E56CE274E010
:1040B00083E394E00E9401C11F910F91FF90EF9064
:1040C000089580916501882341F060917E0470918C
:1040D0007F0441E081E00C9457B90895CF92DF92BC
:1040E000EF92FF92CF93DF9300D000D0CDB7DEB731
:1040F0006B017C0120E030E0A9010E9495E187FD81
:104100001BC06DEB77E386E095E3A70196010E9463
:104110008CE869837A838B839C83CE0101960E940D
:104120009FBA0F900F900F900F90DF91CF91FF905B
:10413000EF90DF90CF9008956DEB77E386E095EBFD
:10414000E4CF0E949CE120E030E04AE754E40E9482
:104150000FE920E030E0A9010E948CE80C946E2069
:104160000F930FB70F9300916E000F930B7F009387
:104170006E0000916F000D7F00936F000F930BB7DF
:104180000F930CB70F921F922F933F934F935F9310
:104190006F937F938F939F93AF93BF93EF93FF930F
:1041A00011240E944CCCFF91EF91BF91AF919F9150
:1041B0008F917F916F915F914F913F912F911F90C0
:1041C0000F900CBF0F910BBF0F910260F8940093FA
:1041D0006F000F9100936E000F910FBF0F91189514
:1041E000EF92FF920F931F93E092F602F092F70284
:1041F0000093F8021093F902609315057093160569
:10420000809317059FEFFF27621B730B840B30F41D
:10421000809570956195790B890B99279093B504DA
:10422000A6E06A9F0092A904512DEE277A9F500DB7
:10423000E11D8A9FE00D5093AA04E093AB04AFE028
:104240006A9F0092AD04512DEE277A9F500DE11D1B
:104250008A9FE00D5093AE04E093AF04AAE06A9FFA
:104260000092B104512DEE277A9F500DE11D8A9FD7
:10427000E00D5093B204E093B3041F910F91FF90AF
:10428000EF900895000000000000000080913D05BF
:1042900080FF27C0459A8FEF8093110580913D05DF
:1042A000869580FF21C0479A8FEF809312058091F9
:1042B0003D058695869580FF1AC02A988FEF8093DA
:1042C000130580913D0586958695869580FF12C0E1
:1042D000289A8FEF80931405000000000000000072
:1042E0000895459881E0D8CF479881E0DECF2A9A9B
:1042F00081E0E5CF289881E0EDCF833B21E0920774
:1043000014F083EB91E090930D1380930C130C94B5
:104310005CBFAF92BF92CF92DF92EF92FF920F936A
:104320001F93CF93DF93C1EDD1E104EF1BE081EE4A
:10433000A82E81E1B82EC12CD12C7601C3946991AD
:104340007991899199910E949AE1288939894A89BC
:104350005B890E94FBE10E9488E9F80161937193F7
:10436000819391938F01C616D706E806F90610F4DB
:104370006B017C01AC16BD0611F76FEF7FEFCB012F
:10438000A70196010E94DDE72093040C3093050CF1
:104390004093060C5093070CDF91CF911F910F9122
:1043A000FF90EF90DF90CF90BF90AF9008950F9364
:1043B0001F93CF93DF9305EE11E1CDE0DCE0F80130
:1043C00021913191419151918F0160E070E080E83D
:1043D0009FE30E940FE96993799389939993FCE095
:1043E000CD31DF0761F70E9426B5DF91CF911F9194
:1043F0000F910C9489210C94D7210C94D7210C9403
:10440000D7210C94D7210C9489210C9489210C94E8
:1044100089210C94892190915613809157139813F8
:1044200006C080911E0C90911F0C892B19F00E94E0
:10443000C47DF1CF0895909156138091571398132E
:1044400008C080911E0C90911F0C892B11F40C94C4
:1044500081730E94C47DEFCFCF93DF9320917B02C5
:10446000222379F0EC010E9464709B01AC01688505
:1044700079858A859B850E948BE8688779878A87FA
:104480009B87DF91CF910895CF93DF9320917B029B
:10449000222379F0EC010E9464709B01AC016885D5
:1044A00079858A859B850E948CE8688779878A87C9
:1044B0009B87DF91CF910895CF9383E50E94107081
:1044C000882331F00E94B16F9093230180932201E1
:1044D00082E40E941070882331F00E94B16F9093A3
:1044E00021018093200186E40E94DF6F8823B9F0C8
:1044F0000E94B56F60931C0170931D0180931E0193
:1045000090931F01C1E020E030E0A9010E9495E1F5
:10451000811101C0C0E0C0933805CF91089560E0DB
:1045200070E0CB01E7CF2F923F924F925F926F9254
:104530007F928F929F92AF92BF92CF92DF92EF9233
:10454000FF920F931F93CF93DF93CDB7DEB76C9796
:104550000FB6F894DEBF0FBECDBF8C015B015A834E
:104560004983FC01EA5BFF4F208131814281538105
:1045700029873A874B875C87CA01B9010E949AE173
:104580006B017C01D5012D913D914D915C910E9473
:10459000FBE10E94F8E82B013C01E981FA812081CE
:1045A000318142815381C701B6010E94FBE10E9423
:1045B000F8E84B015C01C301B2010E9488E9698BF4
:1045C0007A8B8B8B9C8B683771058105910540F444
:1045D00028E730E040E050E0298B3A8B4B8B5C8B36
:1045E000C501B4010E9488E96D877E878F87988B0B
:1045F000683771058105910540F448E750E060E0B7
:1046000070E04D875E876F87788BF801EE5AFF4F19
:104610004080518062807380C301B2010E949CE19E
:1046200069837A838B839C8369897A898B899C8946
:104630000E949AE16D8B7E8B8F8B988F20E030E00B
:10464000A90169817A818B819C810E9495E18823EF
:1046500009F4E1C1A7019601C701B6010E94FBE17F
:104660004B015C012D893E894F89588DCA01B901E2
:104670000E94FBE19B01AC01C501B4010E948BE8E3
:104680004B015C0129813A814B815C81CA01B901EE
:104690000E948CE89B01AC01C501B4010E940FE9A6
:1046A0000E94F8E80E9488E96D837E838F83988753
:1046B00066277727CB0164197509860997090E9437
:1046C0009CE14B015C016D857E858F8598890E94F8
:1046D0009AE12B013C0120E030E0A901C501B401C1
:1046E0000E9495E1882309F49AC1A3019201C301B4
:1046F000B2010E94FBE1698F7A8F8B8F9C8FA7019B
:104700009601C701B6010E94FBE19B01AC01698DD6
:104710007A8D8B8D9C8D0E948BE86B017C01A501AD
:104720009401C501B4010E948CE89B01AC01C70152
:10473000B6010E940FE90E94B7E9D80195968D90C5
:104740009D90AD90BC909897750164012D813E813C
:104750004F815885C21AD30AE40AF50A0E9488E9F3
:10476000C61AD70AE80AF90AF7FE8EC02D893E89D3
:104770004F89588DCA01B9010E94FBE16B017C0190
:1047800029813A814B815C81CA01B9010E948CE880
:1047900069877A878B879C8720E030E0A90169814F
:1047A0007A818B819C810E9495E1882309F43BC129
:1047B000C501B4010E949AE129853A854B855C8543
:1047C0000E94FBE1A70196010E948BE86D837E8326
:1047D0008F839887A3019201C301B2010E94FBE17C
:1047E0009B01AC016D817E818F8198850E948CE850
:1047F0002B013C0120E030E040E850E469817A81FF
:104800008B819C810E94FBE19B01AC01C301B20141
:104810000E940FE90E94F8E82B013C0120E030E003
:10482000A9010E940FEA18161CF0412C512C3201EC
:10483000C301B2010E9488E96D837E838F839887CC
:1048400086169706A806B90620F48D829E82AF824E
:10485000B8866D817E818F8198850E949AE1298535
:104860003A854B855C850E94FBE1A70196010E9479
:104870008CE80E944DEA0E9488E969877A878B87D5
:104880009C87C12CD12C760169857A858B859C8586
:1048900029893A894B895C89621B730B840B950BC0
:1048A0000E949AE129813A814B815C810E940FE943
:1048B00020E034E244EF59E40E94FBE10E9488E9E1
:1048C0004B015C0169857A858B859C852D853E85AC
:1048D0004F855889621B730B840B950B0E949AE1DC
:1048E00029813A814B815C810E940FE920E034E20A
:1048F00044EF59E40E94FBE10E9488E92B013C014E
:104900003FE683169104A104B10408F090C0F401BD
:10491000EE0FFF1FEE0FFF1FE153F74F85919591AB
:10492000A591B4918983292E3A2EBD8B4FE644166A
:1049300051046104710408F083C0F201EE0FFF1FFF
:10494000EE0FFF1FE153F74F45915591659174911B
:104950009A01CB014D815E816F817885D80199964E
:104960004D935D936D937C939C974C0D5D1D6E1DD7
:104970007F1DF80145A756A767A770ABE65BFF4F01
:1049800049895A896B897C89408351836283738307
:10499000D5968D929D92AD92BC92D897F80141AE7A
:1049A00052AE63AE74AEFD9649814083218232825D
:1049B0005D89538334962083318382839383698511
:1049C0007A858B859C85D1966D937D938D939C93F1
:1049D000D4973D962D853E854F8558892083318318
:1049E000428353836C960FB6F894DEBF0FBECDBFE3
:1049F000DF91CF911F910F91FF90EF90DF90CF90BB
:104A0000BF90AF909F908F907F906F905F904F90EE
:104A10003F902F90089560E070E0CB0141CE60E0C0
:104A200070E0CB0188CE60E070E0CB01F3CEC50131
:104A3000B4010E94A2146983272E382E9D8B76CF55
:104A4000C301B2010E94A2149B0184CF90916F0018
:104A500081E091FD02C080E0089590916F009D7FFC
:104A600090936F0008950E9426251092080C1092D2
:104A7000090C10920A0C10920B0C81110C944073CB
:104A800008950F931F938091561390915713891B8C
:104A90008F7009F449C090915313992361F08330CA
:104AA00040F48FEF890F29F08093531390E080E05A
:104AB00038C010925313809157132BE5829FC00189
:104AC0001124805E934FFC01208120FDEFCF4091A7
:104AD000080C5091090C60910A0C70910B0CE95A6A
:104AE000FF4F0081118122813381401B510B620BEA
:104AF000730B4093080C5093090C60930A0C70934D
:104B00000B0C209157132F5F2F702093541330916B
:104B1000571320915513321304C02091541320933E
:104B200055131F910F9108950E943325BFCFFC01AB
:104B300020813181428153816091F1117091F21194
:104B40008091F3119091F4110E94FBE10E9414EA0C
:104B50006093641370936513809366139093671347
:104B6000909156138091571398130C94151E0E9420
:104B70000B220E9426254091641350916513609189
:104B80006613709167134093320550933305609319
:104B900034057093350581110C94407308954F923C
:104BA0005F926F927F928F929F92AF92BF92CF92BD
:104BB000DF92EF92FF920F931F93CF93DF93EC015D
:104BC0008B015A01F9012091F1113091F2114091BC
:104BD000F3115091F41160817181828193810E945F
:104BE000FBE10E9414EA6B017C012091ED113091F0
:104BF000EE114091EF115091F011F501608171813A
:104C0000828193810E94FBE10E9414EA4B015C01C6
:104C10002091E9113091EA114091EB115091EC1182
:104C2000F80160817181828193810E94FBE10E9481
:104C300014EA2B013C012091E5113091E6114091DD
:104C4000E7115091E811688179818A819B810E94E6
:104C5000FBE10E9414EA60935813709359138093F8
:104C60005A1390935B1340925C1350925D136092C1
:104C70005E1370925F138092601390926113A09202
:104C80006213B0926313C0926413D0926513E092E2
:104C90006613F092671390915613809157139817EB
:104CA00091F0DF91CF911F910F91FF90EF90DF90E6
:104CB000CF90BF90AF909F908F907F906F905F90BC
:104CC0004F900C94151E0E940B220E9426254091A5
:104CD000601350916113609162137091631300919E
:104CE0005C1310915D1320915E1330915F13C0909F
:104CF0005813D0905913E0905A13F0905B13C09260
:104D00002605D0922705E0922805F0922905009308
:104D10002A0510932B0520932C0530932D054093E5
:104D20002E0550932F056093300570933105409107
:104D300064135091651360916613709167134093EB
:104D400032055093330560933405709335058823FD
:104D500091F0DF91CF911F910F91FF90EF90DF9035
:104D6000CF90BF90AF909F908F907F906F905F900B
:104D70004F900C944073DF91CF911F910F91FF9052
:104D8000EF90DF90CF90BF90AF909F908F907F90EB
:104D90006F905F904F900895CF92DF92EF92FF92C5
:104DA000CF93DF93C82F0E94262594E0C99FE0018E
:104DB0001124FE01EA5DFA4FC080D180E280F380C9
:104DC00081110E944073C35FD34FC701B6010E9497
:104DD0009CE1288139814A815B810E94FBE1DF915E
:104DE000CF91FF90EF90DF90CF900895CF92DF9218
:104DF000EF92FF92CF93DF93C82F0E94262594E075
:104E0000C99FE0011124FE01E65EFA4FC080D18007
:104E1000E280F38081110E944073C35FD34FC701CA
:104E2000B6010E949CE1288139814A815B810E9400
:104E3000FBE1DF91CF91FF90EF90DF90CF9008954D
:104E4000CF93DF9324E0829FC0011124EC01CA5369
:104E5000D44FFC01E05CFA4F85599D4FDC012D9148
:104E60003D914D915C9160817181828193810E941D
:104E70008CE8688379838A839B83DF91CF9108953F
:104E800080FF04C090919B0490FD8E7F81FF05C040
:104E900090919B04969590FD8D7F82FF06C0909126
:104EA0009B049695969590FD8B7F08952F923F9247
:104EB0004F925F926F927F928F929F92AF92BF922A
:104EC000CF92DF92EF92FF920F931F93CF93DF93D6
:104ED000CDB7DEB7A6970FB6F894DEBF0FBECDBF35
:104EE00080912601882309F4CDC080919B04C82EAF
:104EF000D12CF12CE12C80FF3CC0809028019090B7
:104F00002901A0902A01B0902B0120915B023091E1
:104F10005C0240915D0250915E02C501B4010E94A5
:104F20000FEA181644F480925B0290925C02A09201
:104F30005D02B0925E028090340190903501A090A5
:104F40003601B090370120915B0230915C024091B4
:104F50005D0250915E02C501B4010E9495E187FF98
:104F600008C080925B0290925C02A0925D02B092B7
:104F70005E02D701C601B695A7959795879580FFE4
:104F80003CC080902C0190902D01A0902E01B090FB
:104F90002F0120915F023091600240916102509197
:104FA0006202C501B4010E940FEA181644F480920F
:104FB0005F0290926002A0926102B09262028090C1
:104FC000380190903901A0903A01B0903B012091B6
:104FD0005F02309160024091610250916202C5010E
:104FE000B4010E9495E187FF08C080925F02909211
:104FF0006002A0926102B092620292E0F694E7949D
:10500000D794C7949A95D1F7C0FE3CC0C0903001A8
:10501000D0903101E0903201F09033012091630291
:10502000309164024091650250916602C701B60159
:105030000E940FEA181644F4C0926302D0926402F0
:10504000E0926502F0926602C0903C01D0903D0172
:10505000E0903E01F0903F012091630230916402A4
:105060004091650250916602C701B6010E9495E128
:1050700087FF08C0C0926302D0926402E09265028A
:10508000F09266028091D01183FD7EC02091E00BEA
:105090003091E10B4091E20B5091E30B609167027C
:1050A000709168028091690290916A020E9495E174
:1050B000882309F469C010911D0C111161C0809101
:1050C000720190917301019720910A1330910B1393
:1050D000281739073CF40E94597C89E598E00E9422
:1050E000917611E02091E00B3091E10B4091E20BC1
:1050F0005091E30B609167027091680280916902A0
:1051000090916A020E948BE86B017C0120E030E004
:10511000A9010E940FEA87FF04C0F7FAF094F7F89C
:10512000F09420916E0130916F0140917001509187
:105130007101C701B6010E94FBE120E030E84BE3BA
:1051400054E40E940FEA1816ECF40E94597C8AE39A
:1051500098E00E9491768091670290916802A091F8
:105160006902B0916A028093E00B9093E10BA093E7
:10517000E20BB093E30B87E692E00E94972504C010
:1051800010E0B0CF1111E7CF2AE037ED43E25CE346
:10519000609118017091190180911A0190911B0181
:1051A0000E94FBE16B017C01609116017091170177
:1051B000072E000C880B990B0E949CE19B01AC010F
:1051C000C701B6010E94FBE1698B7A8B8B8B9C8BAC
:1051D00080917B02882309F46CC02091D40B30911C
:1051E000D50B4091D60B5091D70B60915B0270911B
:1051F0005C0280915D0290915E020E948BE86D8B53
:105200007E8B8F8B988F2091D80B3091D90B40914A
:10521000DA0B5091DB0B60915F027091600280911C
:105220006102909162020E948BE8698F7A8F8B8F66
:105230009C8F2091DC0B3091DD0B4091DE0B509167
:10524000DF0B60916302709164028091650290911E
:1052500066020E948BE86D8F7E8F8F8F98A32091BE
:10526000E00B3091E10B4091E20B5091E30B609128
:105270006702709168028091690290916A020E94AF
:105280008BE86B017C0120E030E0A9016D897E890B
:105290008F89988D0E9495E181110FC020E030E048
:1052A000A901698D7A8D8B8D9C8D0E9495E181116C
:1052B00004C0C12CD12C76012CC12D893E894F8987
:1052C000588DCA01B9010E94FBE14B015C01298D97
:1052D0003A8D4B8D5C8DCA01B9010E94FBE19B01A7
:1052E000AC01C501B4010E948CE84B015C012D8D1D
:1052F0003E8D4F8D58A1CA01B9010E94FBE19B016F
:10530000AC01C501B4010E948CE84B015C01A7010E
:105310009601C701B6010E94FBE19B01AC01C501EA
:10532000B4010E948CE80E944DEA4B015C012DEB18
:1053300037E346E855E30E9495E187FF0FC020E080
:1053400030E0A901C701B6010E940FEA46015701EA
:1053500087FF04C0B7FAB094B7F8B0942DEB37E3E9
:1053600046E855E3C501B4010E9495E187FDDEC022
:1053700020E030E040EA51E4C501B4010E940FE9A9
:105380000E9488E91B01672B19F422242394312CF5
:10539000B10190E080E00E949AE19B01AC0160E0E5
:1053A00070E080E89FE30E940FE92B013C01AC0113
:1053B0009B01C501B4010E94FBE14B015C01A3010B
:1053C00092016D897E898F89988D0E94FBE16D8B9A
:1053D0007E8B8F8B988FA3019201698D7A8D8B8D37
:1053E0009C8D0E94FBE1698F7A8F8B8F9C8FA3012C
:1053F00092016D8D7E8D8F8D98A10E94FBE16D8F46
:105400007E8F8F8F98A3A3019201C701B6010E94DE
:10541000FBE169A37AA38BA39CA380E1E4EDFBE00D
:105420008E010F5F1F4FD80101900D928A95E1F711
:105430000E9450BF2B013C0128EC420E511C611C04
:10544000711C0DA31EA381E0281A310809F45FC066
:105450000E9450BF8B019C010419150926093709C8
:1054600037FD86C02B013C0128EC420E511C611C0B
:10547000711C0E94C47D2D893E894F89588D698198
:105480007A818B819C810E948CE869837A838B83EB
:105490009C83298D3A8D4B8D5C8D6D817E818F81B2
:1054A00098850E948CE86D837E838F8398872D8DED
:1054B0003E8D4F8D58A169857A858B859C850E948C
:1054C0008CE869877A878B879C8729A13AA14BA1B1
:1054D0005CA16D857E858F8598890E948CE86D879B
:1054E0007E878F87988B750164018E010F5E1F4F39
:1054F0009E01235F3F4FAE01475F5F4FBE016B5F71
:105500007F4F8DA19EA10E94C4B481119CCF7501D3
:1055100064018E010F5E1F4F27E632E043E652E042
:105520006FE572E08BE592E00E94C4B480E1EBE5A8
:10553000F2E0A4EDBBE001900D928A95E1F7A6960A
:105540000FB6F894DEBF0FBECDBFDF91CF911F9194
:105550000F91FF90EF90DF90CF90BF90AF909F9012
:105560008F907F906F905F904F903F902F90089515
:105570000E94EEC780CF8091970490919804A091EB
:105580009904B0919A048093180190931901A09303
:105590001A01B0931B018091950490919604909309
:1055A00017018093160108958091180190911901B7
:1055B000A0911A01B0911B018093970490939804D5
:1055C000A0939904B0939A048091160190911701C9
:1055D000909396048093950484E690E0909317014D
:1055E0008093160108954F925F926F927F928F92EF
:1055F0009F92AF92BF92CF92DF92EF92FF920F9362
:105600001F93CF93DF93CDB7DEB72C970FB6F894E7
:10561000DEBF0FBECDBF2B013C0129873A874B87E8
:105620005C8747015801F601E080F1800281138117
:1056300020E030E0A901B701C8010E9495E188236C
:1056400009F488C05E2D4F2D302F212F852F942FE8
:10565000A32FB22F89839A83AB83BC8320E030E0F1
:10566000A901B701C8010E9495E1811108C0E0902D
:105670006601F09067010091680110916901C7010E
:10568000D8018D839E83AF83B887A5019401609173
:10569000DC0B7091DD0B8091DE0B9091DF0B0E9493
:1056A00095E187FF0CC08092DC0B9092DD0BA092FD
:1056B000DE0BB092DF0BCE0101960E944D1E409290
:1056C000D40B5092D50B6092D60B7092D70B898574
:1056D0009A85AB85BC858093D80B9093D90BA0930A
:1056E000DA0BB093DB0BCE0105960E944D1EA5018F
:1056F00094016091DC0B7091DD0B8091DE0B909139
:10570000DF0B0E940FEA181664F48092DC0B909273
:10571000DD0BA092DE0BB092DF0BCE0101960E9452
:105720004D1E0E940B222C960FB6F894DEBF0FBEC2
:10573000CDBFDF91CF911F910F91FF90EF90DF9040
:10574000CF90BF90AF909F908F907F906F905F9021
:105750004F90089550E040E030E820E477CFCF92BA
:10576000DF92EF92FF920F931F936A01E090DC0BA0
:10577000F090DD0B0091DE0B1091DF0BFB0120811F
:10578000318142815381FC016081718182819381E9
:105790000E94F32A1F910F91FF90EF90DF90CF901E
:1057A0000895CF92DF92EF92FF920F931F936B01B8
:1057B000FC01E080F18002811381E4EDFBE02481B3
:1057C00035814681578160817181828193810E94F8
:1057D000F32A1F910F91FF90EF90DF90CF900895E3
:1057E000AF92BF92CF92DF92EF92FF920F931F93EF
:1057F000CF93DF9300D000D0CDB7DEB7FC01E080BF
:10580000F18002811381611112C0A090DC0BB09075
:10581000DD0BC090DE0BD090DF0B9501A601B70128
:10582000C8010E9495E187FF02C07501860120E052
:1058300030E046E953E4B701C8010E9495E187FDD5
:1058400004C0E12CF12C06E913E4C701D8018983D7
:105850009A83AB83BC836DEC71E0CE0101960E940C
:10586000D12B0F900F900F900F90DF91CF911F9140
:105870000F91FF90EF90DF90CF90BF90AF90089581
:105880008F929F92AF92BF92CF92DF92EF92FF9250
:105890001F93CF93DF93CDB7DEB760970FB6F89421
:1058A000DEBF0FBECDBF182F80E00E94CC264B017B
:1058B0005C018092890490928A04A0928B04B09239
:1058C0008C0481E00E94CC266B017C01C0928D0487
:1058D000D0928E04E0928F04F092900482E00E94B5
:1058E000CC266093910470939204809393049093D8
:1058F00094041D861E861F86188A89829A82AB822E
:10590000BC82CD82DE82EF82F88669877A878B87B8
:105910009C8783E00E94CC266D877E878F87988B3B
:10592000CE0101960E942C221E3FD9F480E1FE0197
:105930003196A4EDBBE001900D928A95E1F7609657
:105940000FB6F894DEBF0FBECDBFDF91CF911F9190
:10595000FF90EF90DF90CF90BF90AF909F908F908F
:10596000089584E0189FF0011124DF01AC52B44F78
:1059700081E090E08C0F9D1FE80FF91F408151815D
:10598000628173814D935D936D937C931397D7CF11
:105990000C9426B5CF930E94D12B8091610BC82F18
:1059A000C47082FD0CC01092610B82E00E94402CFA
:1059B0000E94C82C81E0C11180E0CF9108950E941F
:1059C0009F7C882381F3F9CFCF93DF93CDB7DEB7E8
:1059D0002C970FB6F894DEBF0FBECDBF0E94A2B5C4
:1059E0000E9426259CE0E6E2F5E0DE01119601909A
:1059F0000D929A95E1F781110E944073CE010196B4
:105A00000E940CCC2C960FB6F894DEBF0FBECDBF13
:105A1000DF91CF9108952F923F924F925F926F92B4
:105A20007F928F929F92AF92BF92CF92DF92EF922E
:105A3000FF920F931F93CF93DF9300D01F92CDB7A8
:105A4000DEB78090D40B9090D50BA090D60BB09081
:105A5000D70B4090D80B5090D90B6090DA0B709018
:105A6000DB0BC090DC0BD090DD0BE090DE0BF090F8
:105A7000DF0B0E9489210E94A01507E91BE088E244
:105A800091E09B838A838BE8282E8BE0382E198245
:105A900089810E942027C8010E946E6EEA81FB81E5
:105AA0006193719381939193FB83EA83C1010E9477
:105AB0006E6EEA81FB816087718782879387F981A7
:105AC000FF5FF9830C5F1F4F84E0280E311CF33019
:105AD000F9F60E94E3720E94D721A501940160911A
:105AE000D40B7091D50B8091D60B9091D70B0E945F
:105AF00095E181111CC0A30192016091D80B7091B6
:105B0000D90B8091DA0B9091DB0B0E9495E181110A
:105B10000EC02091DC0B3091DD0B4091DE0B5091DB
:105B2000DF0BC701B6010E9495E18823B9F00F9001
:105B30000F900F90DF91CF911F910F91FF90EF90F9
:105B4000DF90CF90BF90AF909F908F907F906F909D
:105B50005F904F903F902F900C94E42C0F900F90FB
:105B60000F90DF91CF911F910F91FF90EF90DF90F9
:105B7000CF90BF90AF909F908F907F906F905F90ED
:105B80004F903F902F9008952F923F924F925F92A7
:105B90006F927F928F929F92AF92BF92CF92DF923D
:105BA000EF92FF920F931F93CF93DF93CDB7DEB7A2
:105BB000C358D1090FB6F894DEBF0FBECDBFCDB626
:105BC000DEB641E064E070E0CE0187589F4F0E944E
:105BD0006CB541E062E070E0CE0183589F4F0E94B7
:105BE0006CB543E050E0BE0167587F4F85ED91E012
:105BF0000E94B2EA892B31F181E08093A804909150
:105C0000A80481E089270FB6F894DEBE0FBECDBE92
:105C1000CD57DF4F0FB6F894DEBF0FBECDBFDF917B
:105C2000CF911F910F91FF90EF90DF90CF90BF9099
:105C3000AF909F908F907F906F905F904F903F902C
:105C40002F900895E9961CAE1DAE1EAE1FAEE997CB
:105C500010921C1310921B13CE018F579F4F0E945E
:105C6000EE1DADB6BEB6CF57DF4F0881C158D0404C
:105C700010E00D5F1F4F000F111F000F111F8DB798
:105C80009EB7801B910B0FB6F8949EBF0FBE8DBFC1
:105C9000EDB7FEB73196CE57DF4FF983E883C25890
:105CA000D040801B910B0FB6F8949EBF0FBE8DBFE6
:105CB000EDB7FEB731964F01801B910B0FB6F894EC
:105CC0009EBF0FBE8DBFEDB7FEB731967F01B80105
:105CD000CE57DF4F88819981C258D0400E94F31D72
:105CE0004091F50281E0482764E070E081EE91E1A7
:105CF0000E946CB5B801C4010E94F31DB801C70130
:105D00000E94F31D1091F502111153C0CF57DF4FC0
:105D10008881C158D04090E00296A1EDB1E170E0D9
:105D200060E030E020E043EF5BE0821793070CF483
:105D300098C0CE57DF4FE881F981C258D040E60FB6
:105D4000F71F40805180628073804D925D926D920A
:105D50007D92821793070CF48AC0F401E60FF71FB7
:105D6000208031800281E3812101602E7E2E5096B9
:105D70004D925D926D927C925397821793070CF42B
:105D800080C0F701E60FF71F208031800281E38198
:105D90002101602E7E2E90964D925D926D927C92A6
:105DA00093972F5F3F4F6C5F7F4F2430310509F091
:105DB000BCCF85E092E10E94BE1D89E092E10E9485
:105DC000BE1D8DE092E10E94BE1D81E192E10E9424
:105DD000BE1D85E192E10E94BE1D41E0412760E1C8
:105DE00070E084EE9BE00E946CB5CE018B589F4F13
:105DF0000E94BE1D0FB6F894BEBE0FBEADBE80E4BD
:105E000095E00E94E61DCE0183599F4F0E94C61D5A
:105E10008E010F5F1F4FC8010E94BE1DCE018B581F
:105E20009F4F0E94BE1DCE018B589F4F0E94BE1DEA
:105E3000C8010E94EE1DCE0183599F4F0E94EE1DA6
:105E4000E980AE968FADAE97E89E70011124F1E027
:105E5000EF1AF10800F1CE018B589F4F0E94BE1D32
:105E6000F6CFFA0145905590659074906ECFE3EEB1
:105E7000FBE045905590659074901201062DE72D3A
:105E800073CFE3EDFBE0459055906590749012015F
:105E9000062DE72D7DCF85E493E10E94E61D8AE083
:105EA000F82EFA94CE01FF2029F08B589F4F0E94C4
:105EB000BE1DF7CF81589F4F0E94EE1DCE01805826
:105EC0009F4F0E94EE1DC158DF4F8881CF57D040B1
:105ED000853009F083C1C058DF4F8881C058D04059
:105EE000853009F07BC18091F502811102C00E94CA
:105EF00051728DEE92E00E94DE1D85EE92E00E94CE
:105F0000DE1D4091F50281E0482764E670E081E8FB
:105F100092E00E946CB5C8010E94D61DCE01835943
:105F20009F4F0E94C61D4091F502FF24F3944F2518
:105F300064E070E0C8010E946CB58EE395E00E94B9
:105F4000D61D4091F5024F256CE070E087E79BE09D
:105F50000E946CB54091F5024F2564E170E0C801E4
:105F60000E946CB5F090F502F11038C089809A80DB
:105F7000AB80BC80A5019401C501B4010E948DEAEB
:105F800081112CC080920F1390921013A0921113C4
:105F9000B09212132CEA35EC47E25EE36D817E810C
:105FA0008F8198850E94FBE1609313137093141303
:105FB00080931513909316132CEA35EC47E25EE3B9
:105FC00069857A858B859C850E940FE960931713FC
:105FD000709318138093191390931A13C8010E9499
:105FE000CE1DC8010E94B61DF11038C089809A806C
:105FF000AB80BC80A5019401C501B4010E948DEA6B
:1060000081112CC080926B0B90926C0BA0926D0B47
:10601000B0926E0B2CEA35EC47E25EE36D817E8137
:106020008F8198850E94FBE160936F0B7093700BDA
:106030008093710B9093720B2CEA35EC47E25EE390
:1060400069857A858B859C850E940FE96093730B27
:106050007093740B8093750B9093760BC8010E941C
:10606000B61DC8010E94C61DC8010E94CE1D85E054
:10607000F80111928A95E9F7EE24E3944F2D4E250D
:1060800065E070E0C8010E946CB5C8010E94D61D91
:106090004091F5024E2560E270E0C8010E946CB5A7
:1060A000CE0183599F4F0E94D61D4091F5024E2587
:1060B00069E070E0C8010E946CB54091F5024111A1
:1060C0000FC08981809380028A819B81AC81BD81D0
:1060D00080937C0290937D02A0937E02B0937F0216
:1060E000FF24F3944F2560E270E0C8010E946CB574
:1060F0004091F5024F2560E470E0C8010E946CB544
:106100004091F5024F2560E170E0C8010E946CB536
:106110004091F5024F2560E170E0C8010E946CB526
:10612000C8010E94BE1D4091F5024F256CE070E051
:10613000C8010E946CB54091F5024F256CE670E0F5
:10614000C8010E946CB519821A821B821C821D82B2
:106150001E821F82188619861A861B861C86C80115
:106160000E94B61D4091F5024F2568E070E0C8011D
:106170000E946CB54091F5024F256CE070E0C801BB
:106180000E946CB5CE0181589F4F0E94C61DCE0162
:1061900083599F4F0E94BE1D8091D20B9091D30BCB
:1061A0008134934069F41092A80420911B1330911C
:1061B0001C13EF968EAD9FADEF972817390719F096
:1061C00081E08093A8048091F502811118CD80911F
:1061D000A804811114CD0E940B2D11CDC8010E947D
:1061E000DE1DCE0183599F4F0E94DE1DC158DF4F37
:1061F000E880CF57D040C058DF4F8881C058D0408A
:10620000E89E7001112481E0E81AF10808F483CEB9
:10621000CE018B589F4F0E94BE1DF5CF84E690E0C3
:106220009093D30B8093D20B10921C1310921B13DC
:106230000C94C42D80913C05811105C08091BA0B4E
:10624000882309F461C080918804329B57C0816023
:106250008093880480918804339B52C0826080932D
:10626000880480918804349B4DC0846080938804A6
:106270008091190580FF10C080913D0580FF0CC002
:106280008091880480FF08C08091610B81608093B9
:10629000610B80E00E942CCC80911905869580FFCF
:1062A00011C080913D05869580FF0CC080918804C7
:1062B00081FF08C08091610B82608093610B81E057
:1062C0000E942CCC809119058695869580FF1CC074
:1062D00080913D058695869580FF16C08091BA0B0A
:1062E000882391F08091880482FF0EC08091610B19
:1062F00084608093610B82E00C942CCC8E7FA8CFBD
:106300008D7FADCF8B7FB2CF0895CF93DF9300D039
:1063100000D0CDB7DEB784EF91E0A0E0B0E0898394
:106320009A83AB83BC83BE016F5F7F4F8CE30E9477
:106330009B7480E298E00E94917686B16AE178E0F1
:1063400082FB882780F90E94DA1F86B164E178E039
:1063500083FB882780F90E94DA1F86B16EE078E01F
:10636000829581700E94DA1F349909C00E94D57409
:106370000F900F900F900F90DF91CF9108950E9492
:10638000BA740F900F900F900F90DF91CF910895F6
:1063900080913C05811104C08091BA0B882331F0B3
:1063A00062E070E080E090E00C945D730895CF931C
:1063B000DF93CDB7DEB72C970FB6F894DEBF0FBED4
:1063C000CDBFA1EDB1E190E080E0FC01E951F44FD7
:1063D00045915591659174914D935D936D937D9326
:1063E000FC01E952F44F4591559165917491509695
:1063F0004D935D936D937C935397FC01E953F44F58
:10640000459155916591749190964D935D936D93DF
:106410007C939397049680319105B9F680E29EE4CF
:10642000A0E0B0E08093E1119093E211A093E3111A
:10643000B093E41180E090E8ABE3B4E480930512FC
:1064400090930612A0930712B093081280E090E098
:10645000AAE7B4E48093091290930A12A0930B1256
:10646000B0930C1280E090E0A6E9B3E480930D12A3
:1064700090930E12A0930F12B0931012109211125B
:1064800010921212109213121092141210921512EE
:1064900010921612109217121092181280E090E0CB
:1064A000A0E2B1E48093E40B9093E50BA093E60B9C
:1064B000B093E70B80E090E0A0EAB0E48093E80BB3
:1064C0009093E90BA093EA0BB093EB0B4AE959E9DF
:1064D00069E97EE34093EC0B5093ED0B6093EE0B78
:1064E0007093EF0B8093F00B9093F10BA093F20B52
:1064F000B093F30B109248051092490510924A058B
:1065000010924B05109244051092450510924605D5
:1065100010924705109240051092410510924205D5
:10652000109243050E949F728CE0E4E7F1E0DE01E7
:10653000119601900D928A95E1F789819A81AB813C
:10654000BC818093451390934613A0934713B09357
:1065500048138D819E81AF81B885809349139093B4
:106560004A13A0934B13B0934C1389859A85AB853E
:10657000BC8580934D1390934E13A0934F13B0930B
:10658000501384EB90E09093780B8093770B86E424
:1065900090E090937A0B8093790B10927C0B109281
:1065A0007B0B80EF90E090937E0B80937D0B8EE6CB
:1065B00090E09093800B80937F0B1092820B10924F
:1065C000810B86E696E6A6E8B1E480930F139093DC
:1065D0001013A0931113B09312138CE993E5A9E45F
:1065E000BEE38093131390931413A0931513B093E9
:1065F000161380EE95EBA5EAB3E4809317139093FE
:106600001813A0931913B0931A1383EC95E9ACE215
:10661000B4E480936B0B90936C0BA0936D0BB093D1
:106620006E0B80E29BE1A2E9B1E480936F0B909343
:10663000700BA093710BB093720B87EF9CEDABECDA
:10664000B5E48093730B9093740BA093750BB09388
:10665000760B1092800280E090E0A0EEBFE3809382
:106660007C0290937D02A0937E02B0937F021092F1
:106670003C0510923B050E94C8312C960FB6F89449
:10668000DEBF0FBECDBFDF91CF910C940B2D0C94CC
:10669000D7313F924F925F926F927F928F929F92EB
:1066A000AF92BF92CF92DF92EF92FF920F931F9320
:1066B000CF93DF9300D000D0CDB7DEB7382E80E087
:1066C00090E0A0E2B1E489839A83AB83BC83C0905D
:1066D0004D13D0904E13E0904F13F090501320E0E4
:1066E00030E0A901C701B6010E9495E187FF0CC007
:1066F000A701960160E070E080E291E40E948BE8DF
:1067000069837A838B839C8360E0CE0101960E942B
:10671000F02B4090D40B5090D50B6090D60B70901E
:10672000D70B8090D80B9090D90BA090DA0BB0903B
:10673000DB0B332089F10E94E27C19821A821B82D2
:106740001C82E090DC0BF090DD0B0091DE0B1091D1
:10675000DF0BCE0101966C01A5019401C301B201CA
:106760000E94F32A3092BA0B0E94C8310F900F900A
:106770000F900F90DF91CF911F910F91FF90EF90AD
:10678000DF90CF90BF90AF909F908F907F906F9051
:106790005F904F903F9008950E949F7CCECF2F92A4
:1067A0003F924F925F926F927F928F929F92AF92A1
:1067B000BF92DF92EF92FF920F931F93CF93DF93DD
:1067C000CDB7DEB764970FB6F894DEBF0FBECDBF6E
:1067D000D82E282E312CF101E956F84DF49082E0A4
:1067E000D81234C08091BA0B811103C081E00E949D
:1067F00049330E94E27C81115AC18BEC98E00E94DF
:106800006E6E20E030E0A9010E9495E18823F1F04E
:106810006F2DFF0C770B880B990B0E949CE12B01CD
:106820003C018BEC98E00E946E6E4B015C0120E015
:1068300030E040EA50E40E9495E187FF1BC0812CC4
:10684000912C90EAA92E90E4B92E14C06F2DFF0C64
:10685000770B880B990B0E949CE12B013C01C10135
:10686000880F991F880F991F8D53974F0E946E6E46
:106870004B015C01A3019201C501B4010E94FBE13F
:106880004B015C017101EE0CFF1CEE0CFF1CC701FB
:106890008954974F0E946E6E20E030E040EC5FE339
:1068A0000E94FBE1A30192010E94FBE1AB01BC014C
:1068B00000E010E098018D2D0E9479B892E0D91285
:1068C00030C10E949F7C20E030E0A901C501B401E5
:1068D0000E9495E100E010E020E431E4811118C04D
:1068E0008091B90B84608093B90B80919B04846084
:1068F00080939B04C7018555974F0E946E6E6093ED
:10690000DC0B7093DD0B8093DE0B9093DF0B3DC0AF
:10691000B501A40170588D2D0E9479B8E2E0DE1611
:1069200009F4C0C0A5019401C501B4010E948CE81E
:10693000698B7A8B8B8B9C8BF2E0DF12D0C000E0EE
:1069400010E020EC30E449895A896B897C898D2DCF
:106950000E9479B882E0D812F0C00E949F7C80919A
:10696000B90B84608093B90B80919B048460809301
:106970009B04C7018555974F0E946E6EF701EC523C
:10698000F44F608371838283938320914D13309100
:106990004E1340914F13509150136091DC0B709146
:1069A000DD0B8091DE0B9091DF0B0E948BE86093F2
:1069B000DC0B7093DD0B8093DE0B9093DF0BF70104
:1069C000E559FD4F10821182128213828D2D0E9493
:1069D00020270E94C82CF701EC52F44F808191814E
:1069E000A281B381F701E55AFD4F80839183A28391
:1069F000B38392E0D91609F48FC08CE0E0E8F1E0AF
:106A0000DE01119601900D928A95E1F7E1E0F0E048
:106A1000EC0FFD1FEE0DFF1D80809180A280B380E2
:106A200020E030E0A901C501B4010E9495E188236E
:106A3000F1F120E030E0A901C501B4010E940FEAA4
:106A400087FF04C0B7FAB094B7F8B094F701EC52DE
:106A5000F44F7F01A5019401C301B2010E94FBE143
:106A60009B01AC01F70160817181828193810E9459
:106A70008BE8F7016083718382839383F2E080E087
:106A800090E0A0E4B1E4DF1621F080E090E0A8E41B
:106A9000B2E48D879E87AF87B88BCE010D960E949A
:106AA0004D1E05C00E94E27C882309F43BCF64960A
:106AB0000FB6F894DEBF0FBECDBFDF91CF911F910F
:106AC0000F91FF90EF90DF90BF90AF909F908F90CD
:106AD0007F906F905F904F903F902F900895F101BD
:106AE000E855F74F6491611107C00E94597C86E810
:106AF00098E00E9491766AE070E090E080E00E9469
:106B00009AE19B01AC0160E070E088E492E40E94AD
:106B10000FE98B019C0117CF0E94746E8111C7CFC2
:106B20006CCF20E030E0A901C501B4010E9495E1DD
:106B300000E010E098018111EBCE81E090E0A0E050
:106B4000B0E00D2C04C0880F991FAA1FBB1F0A9428
:106B5000D2F72091B90B282B2093B90B20919B04DD
:106B6000822B80939B04C7018555974F0E946E6EC0
:106B7000F701EC52F44F60837183828393831FCFBC
:106B80008091610B882319F01092610B089540E009
:106B900070E060E08EEE97E00E942B7D0F931F93D4
:106BA0008091C50B813019F50E9450BF009184047B
:106BB000109185042091860430918704601B710B2D
:106BC000820B930B28EE33E040E050E00E94DDE7BB
:106BD000609180047091810480918204909183047B
:106BE000620F731F841F951F1F910F91089560916D
:106BF0005602709157028091580290915902D6CF57
:106C00001092C50B10928404109285041092860491
:106C10001092870410925602109257021092580256
:106C200010925902109280041092810410928204F2
:106C30001092830408958091C50B8130F1F0823069
:106C4000C9F40E94CE3560938004709381048093D0
:106C500082049093830481E08093C50B0E9450BF0F
:106C600060938404709385048093860490938704D2
:106C700081E008950E940036EECF80E008950E94E2
:106C800007B661E081EE92E00E949F760C941B367D
:106C90008091C50B8150823070F41092C50B0E9418
:106CA00050BF60935602709357028093580290939E
:106CB000590281E0089580E00895E0917904E6307A
:106CC00010F581E08E0F809379044091970B5091DD
:106CD000980B6091990B70919A0B9091900B809109
:106CE000910B28E0E29FF0011124E85BFB4F20911B
:106CF0006813309169133183208342835383648303
:106D00007583968387830895CF93DF93EC010E9468
:106D10005D3620E040E070E060E0CE01DF91CF9191
:106D20000C94681E20E040E070E060E089ED9DE595
:106D30000C94681E10920C0C0E940EC50C94923696
:106D4000E0917904EE2389F0E150E093790488E042
:106D5000E89FF0011124E85BFB4F6281738127817A
:106D60004681808191810C94681E0C9492369F928A
:106D7000AF92BF92CF92DF92EF92FF920F931F9349
:106D8000CF93DF930E94ADBBC091900B85E0A82EFE
:106D9000AC0ED6E0DC1B85E0F82EFC1A84E0E82E71
:106DA000EC1A83E0D82EDC1A82E0C82ECC1A81E0DF
:106DB000B82EBC1A9C2E9194C11158C08091920B90
:106DC0008823D1F180916501882359F081E0909169
:106DD000920B911180E024E049EE57E0692D0E946A
:106DE000B4B980910C0C8093890BC43009F0E1C0D8
:106DF0001092B60B8091920B843009F4C5C080913B
:106E00006501882391F011E08091920B843009F0A4
:106E100010E08091890B0E94F41800E09C014EEC78
:106E200057E06E2D812F0E94A36CCF5FCA11C4CF93
:106E300087E08093910B0EC080918D0B10928D0B8B
:106E4000882309F4BFCF0E94A0368091A70B882326
:106E500009F4B8CFDF91CF911F910F91FF90EF9080
:106E6000DF90CF90BF90AF909F900895C130C1F553
:106E70008091920B8130E9F0809165018823A1F027
:106E800011E08091920B813009F010E080911601A1
:106E9000909117010E94BF1800E09C0143EE57E05B
:106EA0006B2D812F0E94A36C80910C0C8093890B19
:106EB000BCCF80918D0B10928D0B8823E9F210E0EE
:106EC00000E027EE33E04AE050E066E171E083EE57
:106ED00097E00E946ABD8091A70B882369F2BACF20
:106EE000C23009F0C2C08091920B8230C9F080910B
:106EF00065018823C9F211E08091920B823009F07C
:106F000010E080910C1390910D130E94BF1800E0C7
:106F10009C014CED57E06C2D812F0E94A36C61CF3A
:106F200080918D0B10928D0B882309F30E9493BAE8
:106F300001E11EE123EB31E050E040E06CE073E161
:106F40008CED97E00E946ABD8091A70B882379F2AF
:106F500081CF80918D0B10928D0B882309F48DC009
:106F60000E9493BA0FEC1FEB2CE830E050E040E0B9
:106F700068E67BE088ED97E00E946ABD8091A70BF0
:106F8000882309F47AC066CF80918D0B10928D0B07
:106F9000882309F434CF0E9493BA62E479E18EEC3D
:106FA00097E00E9417BE8091A70B882309F427CF92
:106FB00051CFC53091F58091920B8530B9F0809119
:106FC0006501882309F431CF11E08091920B85305F
:106FD00009F010E080912401909125010E94BF18D2
:106FE00000E09C0149EC57E06F2D1CCF80918D0B88
:106FF00010928D0B882319F30FE119E127EE33E08E
:107000004AE050E064E271E089EC97E00E946ABDDA
:107010008091A70B882399F21DCFC63009F005CFC8
:107020008091920B863091F080916501882309F45C
:10703000FCCE81E09091920B963009F080E023E045
:107040004AEB57E06D2F0E94B4B9EFCE80918D0BC3
:1070500010928D0B882341F38AE89FE40E948436C6
:107060008091A70B882301F3F5CEC33009F0B9CE88
:107070008091920B833009F46CCF80916501882355
:1070800009F412CF11E08091920B833009F010E0E7
:107090008091680B9091690B0E94BF1800E09C01E1
:1070A00048ED57E06D2D38CF3F924F925F926F922F
:1070B0007F928F929F92AF92BF92CF92DF92EF9288
:1070C000FF920F931F93CF93DF93FF24F39480914C
:1070D0000C1390910D13892B09F4F12C0E94ADBB78
:1070E000C091900B5C2E95E0692E6C0E83E0E82E2B
:1070F000EC1A82E0982E9C1A81E0882E8C1A4C2E75
:1071000041942AE9C22E26E3D22E3DE8A32E37E091
:10711000B32E86E0782E7C1AC11193C08091920B19
:10712000882309F46EC080916501882359F081E0BD
:107130009091920B911180E024E045EB57E0642D93
:107140000E94B4B910E000E0D4E03C2E3518009362
:10715000890BCD131FC0F801EE0FFF1FE757F84F43
:10716000859194919093B80B8093B70B8091920B7B
:107170008C1709F414C180916501882359F081E0CE
:107180009091920B9D1380E023E046E957E0632D38
:107190000E94B4B98D2F0F5F1F4FD5E08530B9F62F
:1071A0008091680B9091690B892B19F4FF2009F4E9
:1071B00016C1C630E9F48091920B863009F400C103
:1071C000809165018823A1F0DF92CF92BF92AF92A8
:1071D0007F9281E09091920B963009F080E08F933E
:1071E0000E94EF1F0F900F900F900F900F900F9035
:1071F00087E0FF24F394CF5FC6118ECF8093910B6D
:107200000EC080918D0B10928D0B882309F48BCFCB
:107210000E94A0368091A70B882309F484CFDF91C8
:10722000CF911F910F91FF90EF90DF90CF90BF9083
:10723000AF909F908F907F906F905F904F903F9016
:107240000895C13009F05FC08091920B813009F43C
:107250003FC080916501882309F474CFD1E080910B
:10726000920B813009F0D0E080910C1390910D13B6
:107270000E94BF1800E09C014EEA57E0682D8D2F58
:107280000E94A36C80910C0C8093890BC33009F091
:1072900059CF1092B60B8091920B833009F46AC0DB
:1072A00080916501882309F44DCFD1E08091920B44
:1072B000833009F0D0E08091890B0E94F41800E03F
:1072C0009C0140EA57E06E2D8D2F0E94A36C3ACFAF
:1072D00080918D0B10928D0B882309F4BACF0E94F8
:1072E00093BA03E11EE123EB31E050E040E06CE0B3
:1072F00073E18EEA97E00E946ABD8091A70B882314
:1073000009F4A7CF8CCFC23009F0BCCF8091920B8B
:107310008230B9F080916501882309F413CFD1E060
:107320008091920B823009F0D0E08091680B9091AF
:10733000690B0E94BF1800E09C014AEA57E0692DE2
:107340009ECF80918D0B10928D0B882319F30E9494
:1073500093BA0FEC1FEB2CE830E050E040E068E619
:107360007BE08AEA97E00E946ABD8091A70B8823A0
:1073700089F255CF80918D0B10928D0B882309F4E3
:107380008FCF0E9493BA62E479E180EA97E00E948D
:1073900017BE8091A70B882309F482CF40CF80913C
:1073A0008D0B10928D0B882309F4E5CE81EF99E3C4
:1073B0000E9484368091A70B882309F4DCCE2FCF5E
:1073C00080918D0B10928D0B882309F4F9CE0E94C9
:1073D0009A368091A70B882309F4F2CE20CF86E05D
:1073E0000ACF4F925F926F927F928F929F92AF924D
:1073F000BF92CF92DF92EF92FF920F931F93CF93A2
:10740000DF930091890B0E94ADBBC091900B10E0FF
:10741000000F111F0757184F95E0592E5C0E2FE6ED
:10742000E22E27E0F22ED3E0DC1B3DEFC32E3FE13E
:10743000D32E41E6A42E47E0B42E82E0782E7C1AAB
:1074400056E9852E57E0952E81E0682E6C1A4C2E59
:107450004194C11137C08091920B8823B1F0809183
:107460006501882359F081E09091920B911180E0A1
:1074700024E04DE757E0642D0E94B4B9CF5F5C1261
:10748000E8CF84E08093910B0CC080918D0B10921B
:107490008D0B882321F30E94A0368091A70B8823AF
:1074A000F1F2DF91CF911F910F91FF90EF90DF905C
:1074B000CF90BF90AF909F908F907F906F905F9094
:1074C0004F900895C13059F5F801859194919093AA
:1074D000B80B8093B70B8091920B813081F0809133
:1074E0006501882359F21F929F928F926F9281E0DB
:1074F0009091920B913009F474C080E072C0809139
:107500008D0B10928D0B882351F38091890B682F7E
:107510000E94FCBF8091A70B882309F3C2CFC23021
:1075200009F042C0F801859194919093B80B809333
:10753000B70B8091920B8230D1F080916501882346
:1075400009F49CCFDF92CF92BF92AF927F9281E0FD
:107550009091920B923009F080E08F930E94EF1F80
:107560000F900F900F900F900F900F9087CF8091FA
:107570008D0B10928D0B882301F30E94FD1F8091CB
:10758000A70B8823D1F28DCF80918D0B10928D0B9C
:107590008823C1F06091890B8FEF0E94FCBF80911E
:1075A000A70B882379F07DCFC33009F067CFF801AE
:1075B000859194919093B80B8093B70B8091920B27
:1075C000833011F380916501882309F457CF1F920E
:1075D000FF92EF92DF9381E09091920B933009F04C
:1075E0008CCF8F930E94EF1F0F900F900F900F90F2
:1075F0000F9044CF2F923F924F925F926F927F9263
:107600008F929F92AF92BF92CF92DF92EF92FF92B2
:107610000F931F93CF93DF930E94ADBBC091900B4C
:107620006C2E85E0582E5C0E99E4C92E97E0D92E79
:1076300023E0E22E4E2C4C1A7724739438E5A32EC7
:1076400037E0B32E12E01C1B372C3C1A2C2E219451
:1076500047E2842E47E0942E84E0F82EFC1AC111F4
:107660007CC08091920B882309F456C080916501FB
:10767000882359F081E09091920B911180E024E0F1
:107680004CE557E0622D0E94B4B980919B0487704D
:10769000873009F0BAC020E030E0A9016091ED0226
:1076A0007091EE028091EF029091F0020E9495E1BC
:1076B000882309F4AAC0D5E0C43009F0A7C0D0914E
:1076C0007B028091920B843079F480918D0B109223
:1076D0008D0B882349F0D725E09265010E94B01DEB
:1076E0008091A70B811126C080916501882391F0BC
:1076F00081E09091920B943009F080E02FE237E026
:10770000D11102C02BE237E001E042E357E06F2DD8
:107710000E94A36CD5E08EC080918D0B10928D0BD2
:10772000882309F4A3CF0E94A0368091A70B882359
:1077300009F49CCFDF91CF911F910F91FF90EF90B3
:10774000DF90CF90BF90AF909F908F907F906F9081
:107750005F904F903F902F900895C13019F5809120
:10776000920B813081F080916501882309F48DCFDF
:1077700081E09091920B913009F080E023E04FE698
:1077800057E2632D80CF80918D0B10928D0B882353
:1077900051F386E49CE30E9484368091A70B8823F2
:1077A00011F3C8CFC23009F05BC09091920B9230B8
:1077B00071F080916501882309F467CF81E09230F0
:1077C00009F080E020E24EE457E0612F5CCF809129
:1077D0008D0B10928D0B882361F3B0924D05A09212
:1077E0004C058091A70B882321F3A4CF80918D0BAA
:1077F00010928D0B8823E1F1D0924D05C0924C057B
:107800008091A70B8823A1F195CFD4E0DC1312C09F
:107810009091920B9D17A9F080916501882351F0FA
:107820006C2F661981E09C1380E020E246E157E06E
:107830000E94B4B9CF5FC51112CFDF5FD093910B17
:1078400079CF80918D0B10928D0B882329F3909224
:107850004D0580924C058091A70B8823E9F26ACFF1
:10786000C33009F012CF9091920B933009F4BECF40
:1078700080916501882309F408CF81E0933009F0F5
:1078800080E020E24FE357E0642DFDCEDF92EF92DF
:10789000FF920F931F93CF93DF930E94ADBBC091D4
:1078A000900B85E0E82EEC0ED4E0DC1B13E01C1BF3
:1078B00002E00C1B81E0F82EFC1ADC2ED194C111E1
:1078C0002EC08091920B8823B1F0809165018823AE
:1078D00059F081E09091920B911180E024E04FE00B
:1078E00057E06D2D0E94B4B9CF5FCE11E8CF85E08F
:1078F0008093910B0CC080918D0B10928D0B88237F
:1079000021F30E94A0368091A70B8823F1F2DF912A
:10791000CF911F910F91FF90EF90DF900895C130AC
:1079200011F58091920B813079F080916501882367
:10793000D9F281E09091920B913009F080E023E040
:1079400040E957E26F2DCECF80918D0B10928D0BB9
:10795000882359F38CE090E20E9484368091A70B33
:10796000882319F3D4CFC23009F055C08091920B0F
:10797000823081F080916501882309F4B5CF81E0E0
:107980009091920B923009F080E023E049E857E2B1
:10799000602FA8CF80918D0B10928D0B882351F30F
:1079A00087E090E20E9484368091A70B882311F330
:1079B000AECF8091920B833081F080916501882356
:1079C00009F492CF81E09091920B933009F080E01E
:1079D00023E042E857E2612F85CF80918D0B109212
:1079E0008D0B882351F382E090E20E9484368091CF
:1079F000A70B882311F38BCF80918D0B10928D0BE9
:107A0000882391F081EF9EE10E9484368091A70B3C
:107A1000882351F07CCFC33061F2C43009F064CFC9
:107A20008091920B843041F380916501882309F4A1
:107A30005BCF81E09091920B943009F080E023E0DD
:107A400049E757E26D2F4ECF0C94A0362F923F920C
:107A50004F925F926F927F928F929F92AF92BF925E
:107A6000CF92DF92EF92FF921F93CF93DF93CDB728
:107A7000DEB72C970FB6F894DEBF0FBECDBF1C014A
:107A8000162F80918D0B10928D0B8823E1F01092B0
:107A90008F0B0E94A0362C960FB6F894DEBF0FBE57
:107AA000CDBFDF91CF911F91FF90EF90DF90CF90EE
:107AB000BF90AF909F908F907F906F905F904F900E
:107AC0003F902F9008958091970B9091980BA091E3
:107AD000990BB0919A0B8D839E83AF83B887892BC6
:107AE0008A2B8B2B09F460C080912601882309F42E
:107AF000BDC0809127018111B9C0613009F494C0E3
:107B0000623009F4A2C08090280190902901A090D1
:107B10002A01B0902B01C0903401D0903501E09043
:107B20003601F0903701612E712C6D817E818F813D
:107B300098850E949CE1209112013091130140919F
:107B40001401509115010E94FBE1D301AA0FBB1F44
:107B5000AA0FBB1FBC87AB87AC52B44FBA87A987AB
:107B60002D913D914D915C910E948CE82B013C013F
:107B70008D819E81AF81B885B7FF8FC0A50194012B
:107B8000C301B2010E9495E187FD7FC0EB85FC85B2
:107B9000EC52F44F4082518262827382812F0E94A4
:107BA000891F81E0809365011092970B1092980BCA
:107BB0001092990B10929A0B80916501882309F419
:107BC0006ACFF4E01F9FC0011124FC01EC52F44F76
:107BD0008A53944FDC012D913D914D915C916081D0
:107BE0007181828193810E948CE86B017C01C98242
:107BF000DA82EB82FC822DEC3CEC4CEC5DE3609194
:107C000012017091130180911401909115010E944D
:107C10000FEA87FD52C0CE0101960E948A16BC0170
:107C2000C1010E94246C37CF80902C0190902D01CF
:107C3000A0902E01B0902F01C0903801D090390152
:107C4000E0903A01F0903B016ECF8090300190902F
:107C50003101A0903201B0903301C0903C01D0902E
:107C60003D01E0903E01F0903F015DCF812C30E579
:107C7000932E33ECA32E37ECB32EC12C40E5D42E3B
:107C800043ECE42E47E4F42E4ECFA985BA858D92BD
:107C90009D92AD92BC92139781CFA7019601C3012B
:107CA000B2010E940FEA18160CF070CFE985FA8530
:107CB000C082D182E282F38271CF20E030E040E2E4
:107CC00051E4C701B6010E94FBE120E030E04AE741
:107CD00054E40E94FBE14B015C0120E030E0A9018B
:107CE000C701B6010E9495E120E030E040EA50E48F
:107CF00087FF04C020E030E040EA50ECC501B40149
:107D00000E948CE820E030E040E251E40E940FE95C
:107D10000E9481E96B017C01F7FC62C020EA36E831
:107D200041E050E00E94FFE7CA01B9012AE030E0DB
:107D300040E050E00E94FFE7605D6093A80BC70140
:107D4000B60120E137E240E050E00E94FFE78AE020
:107D5000882E912CA12CB12CCA01B901A501940146
:107D60000E94FFE7605D6093A90BC701B60128EE92
:107D700033E040E050E00E94FFE7CA01B901A501ED
:107D800094010E94FFE7605D6093AA0B8EE28093EE
:107D9000AB0BC701B60124E630E040E050E00E94A2
:107DA000FFE7CA01B901A50194010E94FFE7605DE8
:107DB0006093AC0BC701B601A50194010E94FFE7D7
:107DC000162FCA01B901A50194010E94FFE7605D69
:107DD0006093AD0B105D1093AE0B88EA9BE01FCF54
:107DE000F094E094D094C094C11CD11CE11CF11C0F
:107DF0006DE2A3CF62E082E897E20C94263D61E059
:107E000089E897E20C94263D60E080E997E20C94C3
:107E1000263DCF93DF9300D000D0CDB7DEB7809161
:107E20008D0B10928D0B882359F010928F0B0E94AE
:107E3000A0360F900F900F900F90DF91CF91089583
:107E40006091970B7091980B8091990B90919A0B80
:107E5000611571058105910561F10E949CE12091F8
:107E600012013091130140911401509115010E94AB
:107E7000FBE12091E00B3091E10B4091E20B50913E
:107E8000E30B0E948CE86093E00B7093E10B80930E
:107E9000E20B9093E30B83E00E94891F81E08093C3
:107EA00065011092970B1092980B1092990B1092FB
:107EB0009A0B80916501882309F4BBCF2091830B35
:107EC0003091840B4091850B5091860B6091E00BB3
:107ED0007091E10B8091E20B9091E30B0E948BE893
:107EE00069837A838B839C83CE0101960E948A16D4
:107EF000BC0189E797E20E94246C9BCF3F924F928E
:107F00005F926F927F928F929F92AF92BF92CF9229
:107F1000DF92EF92FF920F931F93CF93DF930E9414
:107F2000ADBBC091900B3C2E85E0482E4C0E95E2E7
:107F3000C92E96E0D92E01E516E0D4E0DC1B24EF33
:107F4000A22E25E0B22E3FE3E32E36E0F32E83E0AF
:107F5000782E7C1A45EC842E45E0942E82E0682E23
:107F60006C1A81E0582E5C1AC11139C08091920BB5
:107F70008823B9F080916501882361F0632D6195B4
:107F800081E09091920B911180E024E04FE656E061
:107F90000E94B4B9CF5FC411E7CF85E08093910B05
:107FA0000CC080918D0B10928D0B882319F30E94C9
:107FB000A0368091A70B8823E9F2DF91CF911F9122
:107FC0000F91FF90EF90DF90CF90BF90AF909F9078
:107FD0008F907F906F905F904F903F900895C13049
:107FE00041F58091920B813089F080916501882361
:107FF00089F21F9289E696E09F938F935F9281E0CA
:108000009091920B913061F180E02AC080918D0BAC
:1080100010928D0B882349F387E695E090934D05E8
:1080200080934C050E9492368091A70B8823E9F239
:10803000C4CFC23009F064C08091920B8230C9F085
:1080400080916501882309F4A5CF1F9280E696E010
:108050009F938F936F9281E09091920B9230A1F653
:108060008F930E94EF1F0F900F900F900F900F9023
:1080700091CF80918D0B10928D0B882309F39092F4
:108080004D0580924C050E9492368091A70B882363
:10809000B9F293CF8091920B833081F0809165018A
:1080A000882309F477CF1F92FF92EF927F9281E0AD
:1080B0009091920B933009F0A7CFD2CF80918D0B86
:1080C00010928D0B882351F3B0924D05A0924C0570
:1080D0000E9492368091A70B882301F36ECF809186
:1080E0008D0B10928D0B8823A1F0D0924D05C0927C
:1080F0004C050E9492368091A70B882351F05DCFEA
:10810000C33041F2C43009F045CF8091920B8430E6
:1081100031F380916501882309F43CCF1F921F93AE
:108120000F93DF9381E09091920B943009F06CCF24
:1081300097CF7F928F929F92AF92BF92CF92DF9212
:10814000EF92FF920F931F93CF93DF930E949A1D9C
:10815000182F0E94ADBBC091900B0C2F85E0782E9C
:108160007C0E85E0F82EFC1A86E0E82EEC1A84E0FE
:10817000D82EDC1A83E0C82ECC1A82E0982E9C1AE6
:1081800098E3A92E94E0B92E81E0882E8C1AC111B3
:108190004AC08091920B882361F180916501882308
:1081A00061F0602F619581E09091920B911180E0D8
:1081B00024E047EA54E00E94B4B9111193C1C530DC
:1081C00009F022C18091920B853009F4BBC08091E7
:1081D0006501882361F081E09091920B953009F060
:1081E00080E023E04DE654E06F2D0E94B4B9D7E063
:1081F0007AC180918D0B10928D0B882371F20E94B1
:10820000A0368091A70B882341F2DF91CF911F9177
:108210000F91FF90EF90DF90CF90BF90AF909F9025
:108220008F907F900895C13079F58091920B8130C5
:10823000D1F080916501882309F4BFCF1F9286E9B0
:1082400094E09F938F938F9281E09091920B913065
:1082500009F080E08F930E94EF1F0F900F900F9016
:108260000F900F90AACF80918D0B10928D0B8823C9
:1082700001F3B0924D05A0924C050E949236809178
:10828000A70B8823B1F2C1CFC23009F00EC1809193
:10829000920B8230A1F080916501882361F081E02A
:1082A0009091920B923009F080E023E04DE854E089
:1082B000692D0E94B4B9112309F499CF13C180919B
:1082C0008D0B10928D0B882331F38EEB93E40E947B
:1082D00084368091A70B8823F1F297CF8091920B7F
:1082E000833081F080916501882309F4F8C081E032
:1082F0009091920B933009F080E023E040E854E045
:108300006C2DD7CF80918D0B10928D0B882351F35C
:108310008EE895E40E9484368091A70B882311F3A0
:1083200074CF80918D0B10928D0B882309F4C8C0F7
:1083300087E898E40E9484368091A70B882309F48B
:10834000BFC063CF80918D0B10928D0B882309F4F1
:108350003ECF85E69AE40E9484368091A70B88235D
:1083600009F435CF52CF80918D0B10928D0B88235D
:1083700009F452C082EE9BE40E9484368091A70BE0
:10838000882309F449C041CF80918D0B10928D0B49
:10839000882309F4AFC081E19DE40E948436809176
:1083A000A70B882309F4A6C030CF80918D0B1092C3
:1083B0008D0B882309F44BC080E99EE40E9484362B
:1083C0008091A70B882309F442C01FCF80918D0BA9
:1083D00010928D0B882309F453C00E945D3620E073
:1083E00040E070E060E088E490E2DF91CF911F917F
:1083F0000F91FF90EF90DF90CF90BF90AF909F9044
:108400008F907F900C94681EC63009F0F0CE80915A
:10841000920B863009F4A7CF80916501882309F477
:10842000E6CE81E09091920B963009F080E023E057
:1084300044E654E06E2D0E94B4B9D7E081E08D0F80
:108440008C1315C08091920B8C1709F4AECF8091DC
:108450006501882361F06C2F601B81E09091920B85
:108460009C1380E023E04FE454E00E94B4B982E022
:108470008D0F8C1313C09091920B9C1709F4A6CF0B
:1084800080916501882351F06C2F601B81E09C1363
:1084900080E023E04DE354E00E94B4B9CF5FC71100
:1084A00076CEDD5FD093910BB0CEC33009F416CFFA
:1084B000C43009F082CE8091920B843009F431CF20
:1084C00080916501882359F081E09091920B94305E
:1084D00009F080E023E04BE754E06D2DEACE112354
:1084E00009F492CFD5E0DC13A9CF8091920B8D17C0
:1084F00009F44ACF80916501882309F49FCF6C2F3E
:10850000601B81E09091920B9C1380E023E048E592
:1085100054E00E94B4B992CF6F927F928F929F9253
:10852000AF92BF92CF92DF92EF92FF920F931F9381
:10853000CF93DF930E94ADBBC091900B6C2E85E072
:10854000782E7C0E90EFE92E94E7F92E2AEBC22EBE
:1085500024E0D22ED5E0DC1B3AEBA32E34E7B32E79
:1085600014E01C1B03E00C1B82E0982E9C1A81E097
:10857000882E8C1AC11136C08091920B8823B9F0D5
:1085800080916501882361F0662D619581E090916D
:10859000920B911180E024E04EEE54E00E94B4B9B9
:1085A000CF5FC711E7CF86E08093910B0CC080911D
:1085B0008D0B10928D0B882319F30E94A0368091A9
:1085C000A70B8823E9F2DF91CF911F910F91FF90C4
:1085D000EF90DF90CF90BF90AF909F908F907F9063
:1085E0006F900895C13029F58091920B8130A1F0F0
:1085F000809165018823A1F28BE095E79F938F938B
:1086000083ED94E09F938F938F9281E09091920BF2
:10861000913049F180E027C080918D0B10928D0B35
:10862000882331F30E940B758091A70B882301F3F7
:10863000CACFC23009F085C08091920B8230E9F038
:1086400080916501882309F4ABCF8FEB9FE19F9365
:108650008F9389EC94E09F938F939F9281E0909108
:10866000920B9230B9F68F930E94EF1F0F900F90EC
:108670000F900F900F900F9093CF80918D0B1092D1
:108680008D0B8823E9F20E94BF1F8091A70B8823DE
:10869000B9F299CF8091920B8330A9F08091650156
:1086A000882309F47DCF85ED94E79F938F9382EC27
:1086B00094E09F938F930F9381E09091920B93306E
:1086C00009F0A8CFD0CF80918D0B10928D0B88230D
:1086D00029F30E94D5748091A70B8823F9F273CFF8
:1086E0008091920B843099F080916501882309F480
:1086F00057CFBF92AF9285EB94E09F938F931F93D8
:1087000081E09091920B943009F084CFACCF8091AE
:108710008D0B10928D0B882339F30E94BA748091CF
:10872000A70B882309F34FCF80918D0B10928D0BEF
:10873000882399F00E94F0748091A70B882369F038
:1087400042CFC33009F4A6CFC43051F2C53009F08E
:1087500027CF8091920B853039F380916501882372
:1087600009F41ECFFF92EF92DF92CF92DF9381E068
:108770009091920B953009F04DCF75CF7F928F92EB
:108780009F92AF92BF92CF92DF92EF92FF920F93A0
:108790001F93CF93DF930E94ADBBC091900B65E018
:1087A000862E8C0ED6E0DC1B85E0D82EDC1A84E009
:1087B000C82ECC1A83E0B82EBC1A82E0A82EAC1AC0
:1087C00081E0982E9C1A7C2E7194C11134C0809146
:1087D000920B8823B1F080916501882359F081E0E4
:1087E0009091920B911180E024E048E154E0672DD4
:1087F0000E94B4B9CF5FC811E8CF87E08093910B96
:108800000CC080918D0B10928D0B882321F30E9458
:10881000A0368091A70B8823F1F2DF91CF911F91B1
:108820000F91FF90EF90DF90CF90BF90AF909F900F
:108830008F907F900895C130E9F58091920B81303F
:10884000E9F0809165018823A9F211E08091920BF3
:10885000813009F010E06091F5117091F61180916E
:10886000F7119091F8110E949D1B00E09C0143E6D6
:1088700053E0692D812F0E94A36CBCCF80918D0B9A
:1088800010928D0B8823E9F20E9493BAE12C1CE32D
:10889000F12E0CE116E420E030E040E85FE365EF04
:1088A00071E183E693E00E9403BC8091A70B8823CB
:1088B00041F2B3CFC23009F006C18091920B8230F1
:1088C000D9F080916501882309F494CF11E080915B
:1088D000920B823009F010E06091F9117091FA1159
:1088E0008091FB119091FC110E949D1B00E09C0166
:1088F0004CE553E06A2DBECF80918D0B10928D0B0D
:108900008823F9F20E9493BAE12C1CE3F12E0CE1CA
:1089100016E420E030E040E85FE369EF71E18CE5C8
:1089200093E00E9403BC8091A70B882351F275CF7E
:108930008091920B8330D9F080916501882309F4EE
:1089400059CF11E08091920B833009F010E06091D3
:10895000FD117091FE118091FF11909100120E9403
:108960009D1B00E09C0145E553E06B2D83CF80917A
:108970008D0B10928D0B8823F9F20E9493BAE12C93
:108980001CE3F12E0CE116E420E030E040E85FE368
:108990006DEF71E185E593E00E9403BC8091A70B28
:1089A000882351F23ACF8091920B8430D9F0809194
:1089B0006501882309F41ECF11E08091920B843069
:1089C00009F010E06091011270910212809103127F
:1089D000909104120E949D1B00E09C014EE453E024
:1089E0006C2D48CF80918D0B10928D0B8823F9F25E
:1089F0000E9493BAE12C1CE3F12E0CE116E420E076
:108A000030E040E85FE361E072E18EE493E00E94D1
:108A100003BC8091A70B882351F2FFCE8091920B6B
:108A20008530D9F080916501882309F4E3CE11E007
:108A30008091920B853009F010E0609111127091D5
:108A4000121280911312909114120E949D1B00E04B
:108A50009C0149E453E06D2D0DCF80918D0B109258
:108A60008D0B8823F9F20E9493BAE12C1CE3F12EBE
:108A70000CE116E420E030E0A90161E172E189E453
:108A800093E00E9403BC8091A70B882359F2C5CEC6
:108A900080918D0B10928D0B882329F10E9493BA3F
:108AA000E12C1CE3F12E0CE116E420E030E0A901FA
:108AB00065E172E18FE393E00E9403BC8091A70B14
:108AC000882389F0AACEC33009F432CFC43009F428
:108AD0006ACFC53009F4A2CFC63009F08BCE8091A1
:108AE000920B8630A9F280916501882309F482CE29
:108AF00011E08091920B863009F010E06091151220
:108B00007091161280911712909118120E949D1B5D
:108B100000E09C014FE353E06D2FACCE2F923F92CB
:108B20004F925F926F927F928F929F92AF92BF927D
:108B3000CF92DF92EF92FF920F931F93CF93DF9329
:108B4000CDB7DEB72C970FB6F894DEBF0FBECDBF02
:108B5000C090D511D090D611E090D711F090D811D7
:108B60008091D9119091DA11A091DB11B091DC11B3
:108B70008C159D05AE05BF0510F4D701C601C09048
:108B8000D111D090D211E090D311F090D411BC014A
:108B9000CD016C157D058E059F0510F4C701B6014A
:108BA0000E949AE12B013C010E94ADBB2091900BE9
:108BB0002B872E83822F8B5F8D8387E0922F821BE2
:108BC0008F8386E0821B888785E0821B898784E00B
:108BD000821B8A8783E0282E221A82E0382E321ADE
:108BE00091959C872B85211142C08091920B8823FF
:108BF000C9F080916501882359F081E09091920B32
:108C0000911180E024E048E154E06C850E94B4B901
:108C10008B858F5F8B879D819813E4CF88E080934D
:108C2000910B0CC080918D0B10928D0B882309F352
:108C30000E94A0368091A70B8823D9F22C960FB6FC
:108C4000F894DEBF0FBECDBFDF91CF911F910F9182
:108C5000FF90EF90DF90CF90BF90AF909F908F905C
:108C60007F906F905F904F903F902F9008958B85ED
:108C7000813009F089C08091920B8130F9F08091A8
:108C80006501882329F211E08091920B813009F06F
:108C900010E0609105127091061280910712909178
:108CA00008120E949D1B61E02E81621B00E09C0166
:108CB00049E953E0812F0E94A36CAACF80918D0BCC
:108CC00010928D0B8823D9F20E9493BA2AE037EDD7
:108CD00043E25DE3C301B2010E94FBE120E030E02A
:108CE000A9010E948CE84B015C0120E030E040E0EB
:108CF0005FE40E9495E187FD05C0812C912CA12C99
:108D00003FE4B32E2AE037ED43E25DE360910512C4
:108D10007091061280910712909108120E94FBE157
:108D200020E030E0A9010E948CE820E030E040E83B
:108D30005FE30E948BE80E9488E969837A838B83D2
:108D40009C83C501B4010E9481E97B018C0121E073
:108D5000E21AF10801091109912C812C25EDA22EAE
:108D600020E5B22EC980DA8021E030E040E050E01A
:108D700065E072E189E993E00E943ABB8091A70B1C
:108D8000882309F47CCF5ACF8B85823009F08EC1BD
:108D90008091920B8230D9F080916501882309F48B
:108DA00037CF11E08091920B823009F010E0609192
:108DB000091270910A1280910B1290910C120E946C
:108DC0009D1B00E09C014FE853E0632D73CF809121
:108DD0008D0B10928D0B8823F9F20E9493BA60914B
:108DE000DD117091DE118091DF119091E0110E94F0
:108DF0009AE17B018C0120E030E048EC52E469E02C
:108E000072E18FE893E00E9403BC8091A70B882356
:108E100019F214CF8091920B8330D9F080916501C3
:108E2000882309F4F5CE11E08091920B833009F08C
:108E300010E060910D1270910E1280910F129091BE
:108E400010120E949D1B00E09C0146E853E0622D39
:108E500031CF80918D0B10928D0B8823F9F20E94F7
:108E600093BA2AE037ED43E25DE3C301B2010E9409
:108E7000FBE120E030E0A9010E948CE84B015C019D
:108E800020E030E040E05FE40E9495E187FD05C00E
:108E9000812C912CA12C9FE4B92E2AE037ED43E2DE
:108EA0005DE360910D1270910E1280910F129091FE
:108EB00010120E94FBE120E030E0A9010E948CE842
:108EC00020E030E040E85FE30E948BE80E9488E900
:108ED00069837A838B839C83C501B4010E9481E9F5
:108EE0007B018C0121E0E21AF10801091109912CA2
:108EF000812C85EDA82E80E5B82EC980DA8021E08E
:108F000030E040E050E06DE072E186E893E00E94DE
:108F10003ABB8091A70B882309F480CF8FCE809134
:108F2000920B8430E9F080916501882309F470CEBA
:108F300011E08091920B843009F010E06091D11122
:108F40007091D2118091D3119091D4110E949AE125
:108F50000E94851900E09C014FE753E06A85AACE84
:108F600080918D0B10928D0B8823E9F20E9493BAA9
:108F700009E012E224E630E040E050E061ED71E10A
:108F80008FE793E00E94A0BC8091A70B882359F241
:108F900055CE8091920B8530E9F080916501882350
:108FA00009F436CE11E08091920B853009F010E083
:108FB0006091D5117091D6118091D7119091D811EF
:108FC0000E949AE10E94851900E09C0148E753E065
:108FD000698570CE80918D0B10928D0B8823E9F2FC
:108FE0000E9493BA07E012E224E630E040E050E04D
:108FF00065ED71E188E793E00E94A0BC8091A70B2A
:10900000882359F21BCE8091920B8630E9F0809133
:109010006501882309F4FCCD11E08091920B863024
:1090200009F010E06091D9117091DA118091DB1193
:109030009091DC110E949AE10E94851900E09C0148
:1090400041E753E0688536CE80918D0B10928D0BF1
:109050008823E9F20E9493BA05E012E22AE030E0A8
:1090600040E050E069ED71E181E793E00E94A0BC2F
:109070008091A70B882359F2E1CD80918D0B10923E
:109080008D0B882339F10E9493BA03E012E224E6A3
:1090900030E040E050E06DED71E18AE693E00E943F
:1090A000A0BC8091A70B8823A9F0C8CD2B852330C5
:1090B00009F4B0CE243009F432CF253009F469CF59
:1090C000263009F4A0CF273009F0A2CD8091920B71
:1090D000873099F280916501882309F499CD11E0D8
:1090E0008091920B873009F010E06091DD11709152
:1090F000DE118091DF119091E0110E949AE10E94AF
:10910000851900E09C014AE653E06F81D3CD3F9280
:109110004F925F926F927F928F929F92AF92BF9287
:10912000CF92DF92EF92FF920F931F93CF93DF9333
:109130000E94ADBBC091900BA5E04A2E4C0ED4E02E
:10914000DC1B83E0782E7C1A82E0682E6C1A81E0AA
:10915000582E5C1A3C2E3194C11138C08091920B6C
:109160008823B1F080916501882359F081E09091C6
:10917000920B911180E024E048E154E0632D0E94BD
:10918000B4B9CF5FC411E8CF85E08093910B0CC0D8
:1091900080918D0B10928D0B882321F30E94A036B5
:1091A0008091A70B8823F1F2DF91CF911F910F914E
:1091B000FF90EF90DF90CF90BF90AF909F908F90F7
:1091C0007F906F905F904F903F900895C13009F06D
:1091D0005BC08091920B8130E9F08091650188231A
:1091E00081F211E08091920B813009F010E06091E2
:1091F000E40B7091E50B8091E60B9091E70B0E94D8
:10920000D01B00E09C0147EB53E0652D812F0E94AD
:10921000A36CB7CF80918D0B10928D0B8823E9F250
:109220000E9493BA20E030E0A9016091E40B7091B4
:10923000E50B8091E60B9091E70B0E948CE820E013
:1092400030E040E85FE30E948BE80E9488E9912CBF
:10925000812CE9ECAE2EE0E5BE2E6B011DEDE12E7A
:1092600013E0F12E00E010E021E030E040E050E0BB
:1092700064EE7BE087EB93E00E943ABB8091A70B02
:10928000882309F4AACF90CFC23009F0F8C08091AA
:10929000920B8230D9F080916501882309F471CF57
:1092A00011E08091920B823009F010E06091E80BA0
:1092B0007091E90B8091EA0B9091EB0B0E94D01B0F
:1092C00000E09C014FEA53E0662DA0CF80918D0B0A
:1092D00010928D0B8823F9F20E9493BA20E030E0BF
:1092E000A9016091E80B7091E90B8091EA0B9091D4
:1092F000EB0B0E948CE820E030E040E85FE30E9446
:109300008BE80E9488E9912C812C49ECA42E40E541
:10931000B42E6B011DEDE12E13E0F12E00E010E004
:1093200021E030E040E050E068EE7BE08FEA93E03F
:109330000E943ABB8091A70B882309F4ACCF34CFAD
:109340008091920B8330D9F080916501882309F4D4
:1093500018CF11E08091920B833009F010E06091FA
:10936000EC0B7091ED0B8091EE0B9091EF0B0E9446
:109370009E1900E09C0147EA53E0672D47CF80919A
:109380008D0B10928D0B8823F9F20E9493BA20E086
:1093900030E048EC52E46091EC0B7091ED0B809161
:1093A000EE0B9091EF0B0E94FBE120E030E0A90171
:1093B0000E948CE820E030E040E251E40E948BE81B
:1093C0000E9488E9912C812C23ECA22E20E5B22E5C
:1093D0006B011EEAE12E12E8F12E01E010E02AE016
:1093E00030E040E050E06CEE7BE087EA93E00E94E2
:1093F0003ABB8091A70B882309F4A6CFD5CE8091E4
:109400008D0B10928D0B882309F444C00E9493BAEF
:1094100020E030E048EC52E46091F00B7091F10BE9
:109420008091F20B9091F30B0E94FBE120E030E081
:10943000A9010E948CE820E030E040E251E40E9463
:109440008BE80E9488E9912C812C83ECA82E80E582
:10945000B82E6B011EEAE12E12E8F12E01E010E0B9
:109460002AE030E040E050E060EF7BE08FE993E0FD
:109470000E943ABB8091A70B882361F095CEC33040
:1094800009F45ECFC43009F07CCE8091920B843019
:1094900009F4B5CF80916501882309F472CE11E0FB
:1094A0008091920B843009F010E06091F00B709184
:1094B000F10B8091F20B9091F30B0E949E1900E04A
:1094C0009C014FE953E06D2FA1CE4F925F926F92B6
:1094D0007F928F929F92AF92BF92CF92DF92EF9244
:1094E000FF920F931F93CF93DF930E94ADBBC09168
:1094F000900B65E0562E5C0ED3E0DC1B82E0782EEC
:109500007C1A81E0682E6C1A4C2E4194C11137C030
:109510008091920B8823B1F080916501882359F0E6
:1095200081E09091920B911180E024E048E154E0B9
:10953000642D0E94B4B9CF5FC511E8CF84E0809359
:10954000910B0CC080918D0B10928D0B882321F311
:109550000E94A0368091A70B8823F1F2DF91CF9172
:109560001F910F91FF90EF90DF90CF90BF90AF9041
:109570009F908F907F906F905F904F900895C13033
:1095800009F05FC08091920B8130E9F08091650114
:10959000882389F211E08091920B813009F010E06C
:1095A0006091451370914613809147139091481331
:1095B0000E94541A00E09C014DED53E0662D812F6E
:1095C0000E94A36CB8CF80918D0B10928D0B8823D5
:1095D000E9F220E030E040E251E4609145137091FF
:1095E000461380914713909148130E94FBE120E0BD
:1095F00030E0A9010E948CE820E030E84BE355E41C
:109600000E948CE80E9488E9912C812C4DEBA42EBD
:1096100040E5B42E6B0110E7E12E17E1F12E00E0DA
:1096200010E028E434EF4FEF5FEF65E473E18DED78
:1096300093E00E943ABB8091A70B882309F4A6CF40
:109640008DCFC23009F09BC08091920B8230D9F04F
:1096500080916501882309F46ECF11E08091920B0F
:10966000823009F010E06091491370914A138091A3
:109670004B1390914C130E94541A00E09C014EEC45
:1096800053E0672D9CCF80918D0B10928D0B88231A
:10969000F9F220E030E040E251E46091491370912A
:1096A0004A1380914B1390914C130E94FBE120E0F0
:1096B00030E0A9010E948CE820E030E849E055E460
:1096C0000E948CE80E9488E9912C812C2DEBA22E1F
:1096D00020E5B22E6B0110E3E12E11E1F12E00E046
:1096E00010E028E637EF4FEF5FEF69E473E18EECAF
:1096F00093E00E943ABB8091A70B882309F4A8CF7E
:109700002DCF80918D0B10928D0B882309F43FC0D3
:1097100020E030E04AE754E460914D1370914E131D
:1097200080914F13909150130E94FBE120E030E0B4
:10973000A9010E948CE820E030EA4CE056E40E9447
:109740008CE80E9488E9912C812C8DEEA82E80E572
:10975000B82E6B0110E5E12E16E4F12E00E010E0CA
:1097600028ED3CED4FEF5FEF6DE473E18FEB93E09D
:109770000E943ABB8091A70B882349F0EFCEC330FB
:1097800009F0D9CE8091920B833009F4BACF809141
:109790006501882309F4CFCE11E08091920B8330CC
:1097A00009F010E060914D1370914E1380914F13AA
:1097B000909150130E946E2000E09C014FEB53E00B
:1097C0006D2FFDCEBF92CF92DF92EF92FF920F935B
:1097D0001F93CF93DF930E94ADBBC091900B85E0A8
:1097E000C82ECC0ED4E0DC1B13E01C1B82E0F82E4C
:1097F000FC1A81E0E82EEC1ABC2EB194C11130C0E5
:109800008091920B8823B1F080916501882359F0F3
:1098100081E09091920B911180E024E048E154E0C6
:109820006B2D0E94B4B9CF5FCC11E8CF85E0809357
:10983000910B0CC080918D0B10928D0B882321F31E
:109840000E94A0368091A70B8823F1F2DF91CF917F
:109850001F910F91FF90EF90DF90CF90BF900895F0
:10986000C130B9F58091920B8130F1F080916501A2
:109870008823C9F2DD24D3948091920B813009F0C2
:10988000D12C6091E5117091E6118091E7119091D2
:10989000E8110E94D51A00E09C014DE054E06E2DC5
:1098A0008D2D0E94A36CBFCF80918D0B10928D0BDC
:1098B0008823E1F20E9493BA41E052E265EE71E141
:1098C0008DE094E00E9420BD8091A70B882371F267
:1098D000BDCFC23009F07FC08091920B8230E1F0A1
:1098E00080916501882309F49ECFDD24D394809173
:1098F000920B823009F0D12C6091E9117091EA113C
:109900008091EB119091EC110E94D51A00E09C011E
:1099100042E054E06F2DC4CF80918D0B10928D0BDF
:109920008823F1F20E9493BA4FEF51E269EE71E1A0
:1099300082E094E00E9420BD8091A70B882381F2F1
:1099400085CF8091920B8330E1F08091650188236F
:1099500009F469CFDD24D3948091920B833009F010
:10996000D12C6091ED117091EE118091EF119091D9
:10997000F0110E94D51A00E09C0147EF53E0612FDF
:109980008FCF80918D0B10928D0B8823F1F20E9466
:1099900093BA4DEF51E26DEE71E187EF93E00E94D3
:1099A00020BD8091A70B882381F250CF80918D0B31
:1099B00010928D0B8823C9F00E9493BA4BEF51E2AD
:1099C00061EF71E18CEE93E00E9420BD8091A70BC6
:1099D000882359F03BCFC33009F4B3CFC43009F02A
:1099E00022CF8091920B843009F380916501882306
:1099F00009F419CFDD24D3948091920B843009F0BF
:109A0000D12C6091F1117091F2118091F31190912C
:109A1000F4110E94D51A00E09C014CEE53E06D2F2A
:109A20003FCF2F923F924F925F926F927F928F9291
:109A30009F92AF92BF92CF92DF92EF92FF920F93DD
:109A40001F93CF93DF9300D000D000D0CDB7DEB707
:109A50000E94ADBB7090900B7E8285E0870D8D8358
:109A600084E0682E671823E0322E232C271882E02A
:109A7000582E571881E0482E4718711041C0809128
:109A8000920B8823C1F080916501882361F06E817B
:109A9000619581E09091920B911180E024E048E182
:109AA00054E00E94B4B973948D817812E6CF85E0BA
:109AB0008093910B0CC080918D0B10928D0B88239D
:109AC00011F30E94A0368091A70B8823E1F226961D
:109AD0000FB6F894DEBF0FBECDBFDF91CF911F91BF
:109AE0000F91FF90EF90DF90CF90BF90AF909F903D
:109AF0008F907F906F905F904F903F902F90089540
:109B000081E078122DC09091920B9130B9F0809144
:109B10006501882341F281E0913009F080E0909165
:109B2000380523E333E0911102C02FE233E001E076
:109B300046E353E0642D0E94A36CB5CF80918D0B5A
:109B400010928D0B882319F3809138058725809317
:109B50003805309265018091A70B8823C1F2B7CFF9
:109B600082E078129BC08091920B8230C1F080918C
:109B70006501882309F497CF11E08091920B823020
:109B800009F010E080912201909123010E94BF18FA
:109B900000E09C0148E253E0652D812FCCCF8091FD
:109BA0008D0B10928D0B882311F310E000E023EB56
:109BB00031E050E040E062E271E088E293E00E9430
:109BC0006ABD8091A70B882391F281CF8091920B7F
:109BD0008330B9F080916501882309F464CF11E0E6
:109BE0008091920B833009F010E0809120019091D8
:109BF00021010E94BF1800E09C0141E253E0622D68
:109C0000CCCF80918D0B10928D0B882319F310E02F
:109C100000E023EB31E050E040E060E271E081E2FF
:109C200093E00E946ABD8091A70B882399F24FCFE1
:109C300080918D0B10928D0B8823E1F120E030E0B4
:109C400048EC52E460911C0170911D0180911E014D
:109C500090911F010E94FBE120E030E0A9010E94E9
:109C60008CE80E9488E9912C812C81EEA82E80E559
:109C7000B82E6B0118EEE12E13E0F12E00E010E09B
:109C800020E030E0A9016CE171E089E193E00E94FD
:109C90003ABB8091A70B882369F019CF83E078162F
:109CA00009F494CF84E07812FECE8091920B843038
:109CB00009F4BECF80916501882309F4F4CE11E048
:109CC0008091920B843009F010E0C0901C01D0907C
:109CD0001D01E0901E01F0901F0120E030E0A9017D
:109CE000C701B6010E9495E12DEB37E346E055EB45
:109CF00087FD04C02DEB37E346E055E3C701B6010D
:109D00000E948CE869837A838B839C83CE010196C1
:109D10000E94061700E09C0149E153E0662D3DCF0B
:109D20004F925F926F927F928F929F92AF92BF926B
:109D3000CF92DF92EF92FF920F931F93CF93DF9317
:109D40000E94ADBBC091900B35E0632E6C0E43E0DA
:109D5000542ED1E0DC1B4C2E419482E0782E7C1AEC
:109D6000C1113FC08091920B8823F1F08091650171
:109D7000882359F081E09091920B911180E024E0CA
:109D800048E154E0642D0E94B4B980918002882398
:109D900009F4BEC0C23009F457C083E0CF5FC611DA
:109DA000DFCF8093910B0CC080918D0B10928D0BA7
:109DB0008823E1F20E94A0368091A70B8823B1F29C
:109DC000DF91CF911F910F91FF90EF90DF90CF9097
:109DD000BF90AF909F908F907F906F905F904F90CB
:109DE0000895C13091F68091920B8130C9F0809135
:109DF0006501882351F281E09091920B913009F036
:109E000080E09091800223E333E0911102C02FE2C1
:109E100033E001E04FE053E06D2F0E94A36CB5CF1B
:109E20008091800290918D0B10928D0B9923F9F205
:109E30008C2780938002509265010E94A01580912A
:109E4000A70B8823A1F2BCCF8091920B8230F1F056
:109E500080916501882309F4A0CF11E08091920BD5
:109E6000823009F010E060917C0270917D02809157
:109E70007E0290917F020E946E2000E09C0145E0EE
:109E800053E0672D812F0E94A36C87CF80918D0BAB
:109E900010928D0B8823E1F20E9493BA20E030E00B
:109EA0004AE754E460917C0270917D0280917E02C9
:109EB00090917F020E94FBE120E030E0A9010E9426
:109EC0008CE820E030E84BEB54E40E948BE80E94E1
:109ED00088E980EA882E85E1982E9DEEA92E90E5EE
:109EE000B92E6B0116EDE12E16E0F12E00E010E028
:109EF0002CED35E040E050E06CE772E085E093E067
:109F00000E943ABB8091A70B882309F4A1CF58CFB8
:109F100082E044CFCF92DF92EF92FF92CF93DF9314
:109F200080918D0B10928D0B882351F010928F0B26
:109F3000DF91CF91FF90EF90DF90CF900C94A036FF
:109F400081E080938F0B8091970B9091980BA0915B
:109F5000990BB0919A0B0097A105B10509F44BC07C
:109F60002AE0289FE001299FD00D11241092970B21
:109F70001092980B1092990B10929A0BBE010D2E15
:109F8000000C880B990B0E949CE12091150C3091DC
:109F9000160C4091170C5091180C0E94FBE1209177
:109FA0004D1330914E1340914F13509150130E9416
:109FB0008CE86B017C0120E030E040E151EC0E9434
:109FC0000FEA87FD18C020E030E040E151E4C7010E
:109FD000B6010E9495E1181674F0CE010E9489BF67
:109FE000C0924D13D0924E13E0924F13F092501343
:109FF00082E08093650180916501882379F08DE48A
:10A0000093E10E949FBABC0186EF92E0DF91CF916D
:10A01000FF90EF90DF90CF900C94246CDF91CF9164
:10A02000FF90EF90DF90CF9008950F931F93CF9301
:10A03000DF93FC01EB018091970B9091980BA0911D
:10A04000990BB0919A0BB7FF08C01092970B109222
:10A05000980B1092990B10929A0B80919B0B9091F8
:10A060009C0BA0919D0BB0919E0B4091970B509132
:10A07000980B6091990B70919A0B84179507A6071E
:10A08000B70744F48093970B9093980BA093990B88
:10A09000B0939A0B809165018823E1F06091970B52
:10A0A0007091980B8091990B90919A0B00919F0B56
:10A0B0001091A00B2091A10B3091A20B600F711F8A
:10A0C000821F931F0995BC018091A50B9091A60B4F
:10A0D0000E94246C80918D0B811108C08091940B9B
:10A0E0008823D1F1809165018823B1F18091A30B80
:10A0F0009091A40B0097B1F04091970B5091980B61
:10A100006091990B70919A0B00919F0B1091A00B8D
:10A110002091A10B3091A20B400F511F621F731FA2
:10A12000FE010995E091950BF091960B309741F067
:10A130008091940B811103C080918D0B8111099541
:10A1400080918D0B10928D0B882331F0DF91CF9190
:10A150001F910F910C94A036DF91CF911F910F9119
:10A1600008956BE479E184E699E10C94155061E27D
:10A170007CE18AE39CE10C94155068E07CE189E481
:10A180009CE10C94155061E77CE18AE89CE10C9419
:10A1900015506CEA7CE18FEB9CE10C94155068EC57
:10A1A0007CE183EE9CE10C94155062EF7CE18BE046
:10A1B0009DE10C94155069E97CE18AE19DE10C94E4
:10A1C000155068E57CE183E29DE10C94155062E650
:10A1D0007DE185E79DE10C94155061E87DE181EA20
:10A1E00090E20C941550CF93DF93CDB7DEB78D81FD
:10A1F00090915A02891768F080935A029E01285F55
:10A200003F4F4E815F816AE270E08AE292E00E94F5
:10A210005CE1DF91CF9108950F931F93CF93DF936C
:10A220008C016F3F19F410925A0260E020915A029B
:10A23000862F062E000C990B2817190609F04CF5ED
:10A2400060935A0260E08AE892E00E949F76C8011B
:10A250000E9491768AE00E94E575C8010E94E2E0C2
:10A26000800F911FEC01C01BD10BCB32D1053CF00C
:10A270000197FC012491207C2038D1F3F3CFDD2716
:10A28000AE01B8018AE292E00E9403E1C65DDD4FB3
:10A290001882DF91CF911F910F910895DF92EF9275
:10A2A000FF920F931F93CF93DF93CDB7DEB7C658BE
:10A2B000D1090FB6F894DEBF0FBECDBFC358DF4F34
:10A2C000188219821A821B82CD57D04080910F02CA
:10A2D00090911002A0911102B0911202CF57DF4F5E
:10A2E00088839983AA83BB83C158D04084E690E0D9
:10A2F0009093D30B8093D20B10921C1310921B13CC
:10A300001092A80464E070E0CE018F579F4F0E9426
:10A31000E8BE8091D20B9091D30B02969093D30B11
:10A320008093D20B10921C1310921B1381E0CA571A
:10A33000DF4F8883C658D040CE018A579F4F0E9476
:10A34000091E68E470E081ED91E10E94E8BE60E1E1
:10A3500070E084EE9BE00E94E8BE8AE097EDA3EAFD
:10A36000BCE3C358DF4F88839983AA83BB83CD574F
:10A37000D040CE0183589F4F0E94011E80E495E09B
:10A380000E940D1E7E018DE6E80EF11C8FEFD701B5
:10A390008C93C7010E94091E19821A821B821C829B
:10A3A0008E010F5F1F4FC8010E94011E19821A8281
:10A3B0001B821C82C8010E94011EC358DF4F1882F5
:10A3C00019821A821B82CD57D04083E0F701808327
:10A3D0008983CE0183589F4F0E94011EC7010E94AE
:10A3E000091EC8010E94091E4AE0D42EDA94DD201D
:10A3F00031F0CE0183589F4F0E94011EF7CF85E4B4
:10A4000093E10E940D1EC358DF4F188219821A82F1
:10A410001B82CD57D0403AE0D32EDA94DD2031F0C4
:10A42000CE0183589F4F0E94011EF7CF85E0D82EA2
:10A43000D982D701DC92C8010E94091EC7010E947F
:10A44000091E68E070E08DEE92E00E94E8BE68E0D0
:10A4500070E085EE92E00E94E8BE64E670E081E87C
:10A4600092E00E94E8BE19828FEFF7018083C80155
:10A470000E94051EC7010E94091E64E070E081ED84
:10A4800091E00E94E8BE80913E058983C8010E9448
:10A49000051E6CE070E087E79BE00E94E8BE198A29
:10A4A0001A8A1B8A1C8A80E090E0A0E8BFE38D87AF
:10A4B0009E87AF87B88B80910F1390911013A09156
:10A4C0001113B091121389839A83AB83BC832CEA56
:10A4D00035EC47E25EE360911313709114138091A1
:10A4E0001513909116130E940FE96D837E838F835D
:10A4F00098872CEA35EC47E25EE360911713709180
:10A5000018138091191390911A130E94FBE1698727
:10A510007A878B879C8764E170E0C8010E94E8BE5F
:10A5200084E190E09A838983C8010E94F91D80919B
:10A530006B0B90916C0BA0916D0BB0916E0B89839E
:10A540009A83AB83BC832CEA35EC47E25EE36091EF
:10A550006F0B7091700B8091710B9091720B0E9438
:10A560000FE96D837E838F8398872CEA35EC47E271
:10A570005EE36091730B7091740B8091750B9091F9
:10A58000760B0E94FBE169877A878B879C87C801DD
:10A590000E94FD1D8CE0ECE8F1E0D80101900D92E5
:10A5A0008A95E1F7C8010E94FD1D1982C8010E9429
:10A5B000091E8FE790E09A838983C8010E94F91DE4
:10A5C000E8E9F1E0D80101900D92DA94E1F765E055
:10A5D00070E0C8010E94E8BE1982C8010E94051EF1
:10A5E00080E2EDE9F1E0D80101900D928A95E1F762
:10A5F00060E270E0C8010E94E8BED7011C92C7016A
:10A600000E94051E80E892E00E94051E8CE792E001
:10A610000E94011EC358DF4F188219821A821B82C2
:10A62000CD57D040CE0183589F4F0E94011E80E23B
:10A63000F80111928A95E9F760E270E0C8010E9482
:10A64000E8BEFE01F99688E0DF011D928A95E9F7E0
:10A6500044E650E060E070E049835A836B837C837A
:10A660004D835E836F83788783E090E0A0E0B0E065
:10A6700089879A87AB87BC874D875E876F87788B82
:10A68000498B5A8B6B8B7C8B8D8B9E8BAF8BB88F52
:10A69000898F9A8FAB8FBC8F8D8F9E8FAF8FB8A312
:10A6A0008EE190E0A0E0B0E089A39AA3ABA3BCA3A5
:10A6B0008DA39EA3AFA3B8A789A79AA7ABA7BCA752
:10A6C0008DA79EA7AFA7B8AB89AB9AABABABBCAB22
:10A6D0008DAB9EABAFABB8AF60E470E0C8010E9439
:10A6E000E8BE90E1D92EF8018D2D11928A95E9F7F7
:10A6F00060E170E0C8010E94E8BED8011D92DA94C2
:10A70000E9F760E170E0C8010E94E8BEC358DF4F7E
:10A71000188219821A821B82CD57D040CE018358ED
:10A720009F4F0E94011E2CE0D22EF8018D2D119218
:10A730008A95E9F76CE070E0C8010E94E8BE8CE6FB
:10A74000D8011D928A95E9F76CE670E0C8010E9475
:10A75000E8BE8CE994E00E94FD1DF7011082118291
:10A7600012821382148215821682178268E070E0CA
:10A77000C7010E94E8BEF7011192DA94E9F7CB57BE
:10A78000DF4F1882C558D04080E090E0A0E4B0E4EC
:10A79000ED968CAF9DAFAEAFBFAFED97C7010E94F6
:10A7A0000D1ECE018B579F4F0E94091ECE01875868
:10A7B0009F4F0E94011E8091A804811124C0009126
:10A7C000D20B1091D30B80911B1390911C13D701C6
:10A7D0008D939C9384E690E09093D30B8093D20B5F
:10A7E00064E070E085ED91E00E94E8BEC7010E9440
:10A7F000F91D91E00134134009F490E08091A80420
:10A80000892B8093A8048091A804811105C060E081
:10A8100083EA9BE00E940C519091A80481E0892773
:10A82000CA57DF4F0FB6F894DEBF0FBECDBFDF9122
:10A83000CF911F910F91FF90EF90DF90089581E0ED
:10A840008093F5020E940E311092F50281110C9452
:10A850000E310E94D7310E944E510E94597C83EBE9
:10A860009BE00E94917680E008950C941F540C9414
:10A870004E512F923F924F925F926F927F928F92A2
:10A880009F92AF92BF92CF92DF92EF92FF920F937F
:10A890001F93CF93DF9300D01F92CDB7DEB70E94F6
:10A8A0009A1D782E0E94ADBB2091900B2A83122F07
:10A8B0002B5F298383E0682E611A82E0582E511A9B
:10A8C00081E0482E411A312E319427E3C22E24E52F
:10A8D000D22E3BE1A32E35E0B32E47E4842E43E392
:10A8E000942E8A81811105C18091920B882309F4ED
:10A8F000DCC080916501882359F081E09091920B32
:10A90000911180E024E042E655E0632D0E94B4B945
:10A91000711054C18A81833009F006C18091920B75
:10A92000833009F43AC180916501882309F4FCC0A1
:10A9300081E09091920B933009F080E023E049E3AD
:10A9400055E0662D0E94B4B924E02B83F12CE12C54
:10A950002A80211A2A818B81281322C0F701EE0F49
:10A96000FF1FE757F84F85919491E092B60B9093B3
:10A97000B80B8093B70B8091920B821709F425C115
:10A9800080916501882361F081E09091920B2B8189
:10A99000921380E023E04AE255E0622D0E94B4B9B0
:10A9A0000B8181E0800F8B83EA94EF2809F009C1C5
:10A9B0002A8182131FC08091920B821709F416C15D
:10A9C000809165018823B1F0DF92CF92BF92AF9260
:10A9D0008A81811B8F9381E09091920B2A8192133F
:10A9E00080E08F930E94EF1F0F900F900F900F90B9
:10A9F0000F900F9082E0800F71104EC09A818913E2
:10AA000023C08091920B891709F4FFC080916501E2
:10AA10008823D1F085E394E59F938F938DE095E0B3
:10AA20009F938F938A81811B8F9381E09091920BEA
:10AA30002A81921380E08F930E94EF1F0F900F9056
:10AA40000F900F900F900F9083E0800F9A818913E1
:10AA500021C08091920B891709F4E6C080916501AD
:10AA60008823C1F09F928F928CEF94E09F938F93F5
:10AA70008A81811B8F9381E09091920B2A8192139E
:10AA800080E08F930E94EF1F0F900F900F900F9018
:10AA90000F900F9084E0800F9A819F5F9A832981A5
:10AAA00092131FCF8093910B0EC080918D0B10924B
:10AAB0008D0B882309F41DCF0E94A0368091A70B2F
:10AAC000882309F416CF0F900F900F90DF91CF914C
:10AAD0001F910F91FF90EF90DF90CF90BF90AF90BC
:10AAE0009F908F907F906F905F904F903F902F90AE
:10AAF00008959A81913051F58091920B8130B9F08F
:10AB000080916501882309F403CF81E09091920B35
:10AB1000913009F080E023E040E555E0642D0E948B
:10AB2000B4B993E0711001C094E09B830FCF809182
:10AB30008D0B10928D0B882319F389E990E40E9404
:10AB400084368091A70B8823D9F2BDCF2A81223089
:10AB500009F0DECE8091920B823081F08091650108
:10AB6000882309F4D5CE81E09091920B923009F0C0
:10AB700080E023E041E455E0652DD1CF80918D0B3D
:10AB800010928D0B882351F38AE89FE40E9484364B
:10AB90008091A70B882311F396CF80918D0B109293
:10ABA0008D0B882309F4BFCE8CE892E40E94843692
:10ABB0008091A70B882309F4B6CE85CF83E08B83E1
:10ABC000C5CEEE24E394F12CC5CE80918D0B10926E
:10ABD0008D0B882309F4D4CE83E296E50E94843657
:10ABE0008091A70B882309F4CBCE6DCF80918D0B7C
:10ABF00010928D0B882309F4E3CE0E944E51809170
:10AC0000A70B882309F4DCCE5ECF80918D0B1092C8
:10AC10008D0B882309F4FACE0E941F548091A70B54
:10AC2000882309F4F3CE4FCF80918D0B10928D0BBA
:10AC3000882309F413CF0E94D7318091A70B882372
:10AC400009F40CCF40CF2F923F924F925F926F92B8
:10AC50007F928F929F92AF92BF92CF92DF92EF92AC
:10AC6000FF920F931F93CF93DF93CDB7DEB7289753
:10AC70000FB6F894DEBF0FBECDBF2091B60B28876C
:10AC80000E94ADBB3091900B3F83E8858E2F90E002
:10AC9000880F991F9C012757384F3C832B8336E040
:10ACA000E39FC0011124FC01E758F44FFA83E983C4
:10ACB0009C012958344F79015F8035E0432E450CC3
:10ACC00011E0312E3518252C2194FE82ED8257019A
:10ACD00034E0A30EB11C47E3C42E44E5D42E85E036
:10ACE000782E75184701E2E08E0E911C82E0682EE6
:10ACF0006518FF81F11159C01123D9F08091920B91
:10AD00001816BCF04091970B5091980B6091990BDD
:10AD100070919A0B4F5F5F4F6F4F7F4F4093970B30
:10AD20005093980B6093990B70939A0B8F5F80935D
:10AD3000920B80916501882341F0EB81FC81659144
:10AD4000749143E0822D0E9457B9F5018081809370
:10AD5000890BFF81F23009F07AC028852093B60B69
:10AD60008091920B823009F45FC080916501882345
:10AD700091F011E08091920B823009F010E0809107
:10AD8000890B0E94F41800E09C0144EE54E0662D0B
:10AD9000812F0E94A36C10E02F812F5F2F8324113D
:10ADA000A8CF86E08093910B19C02F81213069F6DE
:10ADB0008091920B813031F080916501811127C023
:10ADC00010E0C3CF80918D0B10928D0B8823A1F3DF
:10ADD0000E94A0368091A70B882371F328960FB6A6
:10ADE000F894DEBF0FBECDBFDF91CF911F910F91C1
:10ADF000FF90EF90DF90CF90BF90AF909F908F909B
:10AE00007F906F905F904F903F902F90089581E0DA
:10AE10009091920B913009F080E024E04EEE54E0E6
:10AE2000632D0E94B4B9CCCF80918D0B10928D0B05
:10AE3000882309F49ACF67E779E184EE94E00E94D1
:10AE400017BE8091A70B882309F48FCFC7CF3F810E
:10AE5000333091F58091920B8330C1F08091650180
:10AE6000882309F498CF11E08091920B833009F088
:10AE700010E0ED81FE81808191810E94BF1863E026
:10AE8000651900E09C014DED54E082CF80918D0B5F
:10AE900010928D0B882311F310E000E023EB31E0DA
:10AEA00045E050E0B7018DED94E00E946ABD8091CD
:10AEB000A70B882399F292CFFF81F43091F580910E
:10AEC000920B8430B9F080916501882309F463CF37
:10AED00011E08091920B843009F010E0F401808140
:10AEE00091810E94BF1864E0651900E09C0149ED62
:10AEF00054E04ECF80918D0B10928D0B882319F367
:10AF000010E000E02CE830E045E050E069817A8113
:10AF100089ED94E00E946ABD8091A70B882399F285
:10AF20005DCFFF81F53009F037CF8091920B8530EE
:10AF3000E1F080916501882309F42DCFDF92CF9253
:10AF40008BE195E09F938F937F9281E09091920B9C
:10AF5000953009F080E08F930E94EF1F0F900F90C3
:10AF60000F900F900F900F9016CF80918D0B109235
:10AF70008D0B8823F1F20E944E518091A70B8823FC
:10AF8000C1F22CCF0E94D7310E944E510C949236C0
:10AF9000CF9380914004811109C086ED92E0909397
:10AFA0007F0480937E0481E0809340040E945D369C
:10AFB00020E040E070E060E081E690E20E94681EE0
:10AFC000C1E0C0938F0B0E940B2210928F0B0E9446
:10AFD000A036C0938F0B8091BB0B811107C046EC4C
:10AFE00052E06DEC72E084E00E9433B660E08DE1E7
:10AFF00098E20E940C5161E080EC92E0CF910C94B9
:10B000009F762F923F924F925F926F927F928F9294
:10B010009F92AF92BF92CF92DF92EF92FF920F93E7
:10B020001F93CF93DF9300D000D01F92CDB7DEB730
:10B030002091C50B2D830E94ADBB8091900B8C831A
:10B04000582E8B5F898357EB252E56E7352E01EA64
:10B0500016E06FE3E62E66E3F62E7BEBC72E76E076
:10B06000D72E81E0482E451883E0782E751882E0AF
:10B0700085198A83E8ECAE2EE7E5BE2EF8ED8F2E1B
:10B08000F6E09F2E952D91959B832C8121113EC03A
:10B090008091920B8823B1F080916501882359F04B
:10B0A00081E09091920B911180E024E044EE56E013
:10B0B0006B810E94B4B98D81813009F0ABC024E06E
:10B0C000622EDBC080918D0B10928D0B882321F3B3
:10B0D0000E94A0368091A70B8823F1F20F900F9069
:10B0E0000F900F900F90DF91CF911F910F91FF90D4
:10B0F000EF90DF90CF90BF90AF909F908F907F9018
:10B100006F905F904F903F902F9008958D81813088
:10B1100009F080C09C81913061F58091920B813063
:10B12000D9F0809165018823A1F0BF92AF929F92E0
:10B130008F924F9281E09091920B913009F080E0D4
:10B140008F930E94EF1F0F900F900F900F900F9012
:10B150000F9094E0692EAAC080918D0B10928D0BF8
:10B160008823F9F20E94C8578091A70B8823C9F25F
:10B17000B5CF2C81223031F58091920B823099F03D
:10B1800080916501882361F081E09091920B92306B
:10B1900009F080E023E04DEC56E06A810E94B4B9EA
:10B1A00084E0682E9EC080918D0B10928D0B8823B9
:10B1B00039F38FE290E20E9484368091A70B8823B6
:10B1C000F9F28CCF8C81833009F079CF8091920B8A
:10B1D000833089F080916501882311F381E090919B
:10B1E000920B933009F080E023E048EC56E0672DA5
:10B1F0000E94B4B9AECF80918D0B10928D0B882335
:10B2000049F387EB96E30E9484368091A70B88234D
:10B2100009F364CF8091C50B823009F0AFC09C81E7
:10B2200032E0632E913009F0ABC08091920B8130F7
:10B2300009F480C08091650181118BC042E0642EC9
:10B2400081E0860D9C81891316C08091920B89172D
:10B2500009F4C6C080916501882369F06C81651985
:10B2600081E09091920B2C81921380E023E04AE9D7
:10B2700056E00E94B4B9639463948C81681216C03E
:10B280008091920B861509F4BCC0809165018823DA
:10B2900069F06C81651981E09091920B2C81921379
:10B2A00080E023E04EE856E00E94B4B981E0860DCC
:10B2B0009C81891316C08091920B891709F4B2C042
:10B2C00080916501882369F06C81651981E0909116
:10B2D000920B2C81921380E023E040E856E00E941C
:10B2E000B4B982E0860D9D819130D9F02C81821312
:10B2F00016C08091920B821709F4A5C08091650158
:10B30000882369F06C81651981E09091920B2C8102
:10B31000921380E023E04CEA56E00E94B4B983E047
:10B32000860D9C819F5F9C8329819213AECE809372
:10B33000910BD4CE80918D0B10928D0B882309F444
:10B3400079CF0E943F368091A70B882309F472CFF2
:10B35000C5CEFF92EF92DF92CF924F9281E0909113
:10B36000920B913009F080E08F930E94EF1F0F90B5
:10B370000F900F900F900F900F9060CF6624639402
:10B380002C8162125DCF8091920B8615E1F0809145
:10B390006501882309F454CF3F922F921F930F9396
:10B3A0008C8185198F9381E09091920B2C8192135F
:10B3B00080E08F930E94EF1F0F900F900F900F90DF
:10B3C0000F900F903DCF80918D0B10928D0B8823A5
:10B3D000F1F20E94B7768091A70B8823C1F27ECE4E
:10B3E00080918D0B10928D0B882309F433CF8AEF57
:10B3F0009AE30E9484368091A70B882309F42ACF10
:10B400006DCE80918D0B10928D0B882309F43DCF6A
:10B4100084E598E30E9484368091A70B882309F481
:10B4200034CF5CCE80918D0B10928D0B882309F464
:10B4300047CF89E394E50E9484368091A70B882347
:10B4400009F43ECF4BCE80918D0B10928D0B88234B
:10B4500009F454CF8EE79FE30E9484368091A70BB6
:10B46000882309F44BCF3ACE61E088E992E00E944C
:10B470009F760E9448368091BB0B811107C04DEA30
:10B4800052E065EB72E085E00E9433B660E08FE940
:10B4900092E00E940C510C9492360F931F930E94DD
:10B4A00050BF00913C0410913D0420913E04309126
:10B4B0003F04601B710B820B930B97FD0CC089B18D
:10B4C00083FB882780F991E089274A9B8260309B23
:10B4D000846080933B0480913B04817090913B0495
:10B4E00091FD826090913A04981749F0813009F1FA
:10B4F00048F0823079F0833091F080933A041F91C4
:10B500000F910895913079F09230B9F79091390404
:10B5100091500CC0992339F09330C1F3EECF9130A4
:10B52000A9F3923051F7909139049F5F90933904B9
:10B53000E4CF992359F3933001F7F5CF4F925F92FF
:10B540006F927F928F929F92AF92BF92CF92DF9233
:10B55000EF92FF920F931F93CF93DF9300D000D011
:10B56000CDB7DEB70E9450BF4B015C018091100146
:10B570008F3FF1F10E9450BFC0902904D0902A045F
:10B58000E0902B04F0902C046C197D098E099F0922
:10B5900097FD2EC080915613909157138F5F8F7037
:10B5A000891731F1E0911001E43008F0E2C024E0A5
:10B5B000E29FF0011124E354FE4F80819181A2812A
:10B5C000B38189839A83AB83BC83C12CD12C760150
:10B5D0008E010F5F1F4F20EE3BE04CED5BE068ED0E
:10B5E0007BE084ED9BE00E94C4B48FEF8093100158
:10B5F0000E944D5A80913B0482FFC4C08091380460
:10B6000081111DC091E0909338048091290289270F
:10B6100080938D0B1092290283E080936501109234
:10B620003B040E9450BF6C507E4F8F4F9F4F6093E2
:10B630003C0470933D0480933E0490933F048091BA
:10B64000340490913504A0913604B0913704A501DB
:10B650009401281B390B4A0B5B0BDA01C901B7FFB8
:10B6600005C080917804882309F4D2C1D501C401B2
:10B670008C599F4FAF4FBF4F809334049093350444
:10B68000A0933604B093370460913904062E000C61
:10B69000770B77FF03C0719561957109909139041B
:10B6A00080913304981371C0633008F06EC010921B
:10B6B00039048091390480933304643008F075C0F4
:10B6C00080918D0B8111F3C0809168139091691363
:10B6D000895D9D4541F480911101882309F4F9C0E9
:10B6E0008150809311010E942625C090080CD090B3
:10B6F000090CE0900A0CF0900B0C81110E94407331
:10B70000D701C6013AE0B695A795979587953A95E2
:10B71000D1F7009741E0A407B10520F08FEF9FEF2C
:10B72000A0E0B0E096958795209165012111E3C0D6
:10B730003091780431119AC1809168139091691306
:10B74000895D9D4509F479C180918F0B811175C187
:10B7500080912F0490913004A0913104B091320473
:10B76000881A990AAA0ABB0AB7FC75C10E949236C8
:10B7700072C18091660190916701A0916801B091BA
:10B7800069011FCF109238045ACF633009F091CF6E
:10B790008091390487FD07C081E0880F880F80936E
:10B7A000390464E086CF8FEFF8CF8091B40B21E0AD
:10B7B00030E040E050E0882309F456C0C090B00B60
:10B7C000D090B10BE090B20BF090B30BC114D10448
:10B7D000E104F104E9F170E090E080E00E949AE178
:10B7E00020E030E040E85EE30E94FBE12B013C01F9
:10B7F000C501B4016C197D098E099F090E949AE167
:10B800009B01AC01C301B2010E940FE920E030E0CE
:10B810004AE754E40E94FBE16B017C0120E030E048
:10B8200042E053E40E940FEA24E630E040E050E0BA
:10B8300087FF12C020E030E040EA52E4C701B601C1
:10B840000E940FEA2AE030E040E050E087FF04C0A9
:10B8500021E030E040E050E08092B00B9092B10BDC
:10B86000A092B20BB092B30BA09139040A2E000C37
:10B87000BB0B0E9429E824E030E040E050E00E9449
:10B88000FFE78091970B9091980BA091990BB09145
:10B890009A0B820F931FA41FB51F8093970B909351
:10B8A000980BA093990BB0939A0B10923904D50181
:10B8B000C4018856954CAF4FBF4F80932F0490938F
:10B8C0003004A0933104B093320481E08093650189
:10B8D000FBCE8CE08093110180912D0490912E0479
:10B8E000009729F0019790932E0480932D0481E016
:10B8F00080936501F8CE009741F040912D0450915E
:10B900002E044817590708F017CF80917804811149
:10B910001DC0223038F0243008F44CC0243011F41B
:10B92000109265018091A713811105C081E0809379
:10B93000A7130E94F0B380917013909171130E942D
:10B94000C9B381E08093930B8093780483E00E94D5
:10B95000DE6A81E080938E13E0916813F0916913A1
:10B9600009951092930B80917804811127C0109251
:10B970008D0B8091681390916913895D9D4509F045
:10B98000E3CE0E9450BFDC01CB0188199909AA09B6
:10B99000BB09C0902D04D0902E04F12CE12CC816C8
:10B9A000D906EA06FB0608F0C7CE90932E048093D2
:10B9B0002D04C2CE81E080936501B4CF8EE693E181
:10B9C0000E9487C291E0811101C090E090937804B9
:10B9D000882369F28091681390916913895D9D4570
:10B9E000B9F40E9450BFDC01CB0188199909AA095A
:10B9F000BB09C0902D04D0902E04F12CE12CC81668
:10BA0000D906EA06FB0620F490932E0480932D04B9
:10BA10000F900F900F900F90DF91CF911F910F918A
:10BA2000FF90EF90DF90CF90BF90AF909F908F905E
:10BA30007F906F905F904F90089548E9840E4AE39D
:10BA4000941EA11CB11C80922F0490923004A092ED
:10BA50003104B0923204809178048111D9CF809161
:10BA600065018130A9F610926501D2CF009709F4E3
:10BA70006DCF43CFCF938091FA03811154C01092C0
:10BA8000A5131092A6131092A7131092731310927D
:10BA9000721310927513109274131092771381E041
:10BAA0008093761382E28093781310927D13109224
:10BAB0007C13E1E9F3E12FE933E18FEF81932E1756
:10BAC0003F07E1F7C1E0C0938E1323E933EA3093D7
:10BAD000841320938313C0938513109286131092BE
:10BAE000871390E490938813109289132FEC32EA15
:10BAF0003093A01320939F1328E031E0309371130B
:10BB0000209370139EE19093951391E19093961377
:10BB10009CE19093931380939213809391130E94CE
:10BB2000F0B3C093FA0381E08093280287ED91E09F
:10BB30009093031380930213109205131092041331
:10BB400053985B9A52985A9A3898409A0E944D5A44
:10BB500010923904CF910895FC01A081B1811C920B
:10BB6000A281B3818C918F5F8C930280F381E02D51
:10BB700090818CE0989F800D1124EAE6F3E113AEEA
:10BB800084AF0895FC0180E09491992331F0907C7A
:10BB9000903809F08F5F3196F7CF0895FC0180E06F
:10BBA0009191992329F0907C9038D1F38F5FF8CF51
:10BBB00008954F925F926F927F928F929F92AF9271
:10BBC000BF92CF92DF92EF92FF920F931F93CF938A
:10BBD000DF9300D000D01F92CDB7DEB71092B40B28
:10BBE00080918D0B10928D0B8823E9F020E040E0CE
:10BBF00070E060E081E098E50F900F900F900F905B
:10BC00000F90DF91CF911F910F91FF90EF90DF90F8
:10BC1000CF90BF90AF909F908F907F906F905F90EC
:10BC20004F900C94681E209116013091170140919D
:10BC3000970B5091980BCA01820F931F2436310540
:10BC400009F0CEC34730510544F006978A3091057C
:10BC50000CF0D5C38AE090E0DCC306964A3F5F4F04
:10BC6000ACF38091930B882309F494C12091C60B07
:10BC70003091C70B4091C80B5091C90B6091D40B08
:10BC80007091D50B8091D60B9091D70B0E948CE8C8
:10BC90004B015C012091CA0B3091CB0B4091CC0B36
:10BCA0005091CD0B6091D80B7091D90B8091DA0B2C
:10BCB0009091DB0B0E948CE869837A838B839C8351
:10BCC0002091CE0B3091CF0B4091D00B5091D10BE6
:10BCD0006091DC0B7091DD0B8091DE0B9091DF0B9E
:10BCE0000E948CE82B013C0120E030E040E251E46E
:10BCF0000E94FBE120E030E048EC52E40E94FBE1CE
:10BD00006B017C0120E030E0A901C301B2010E9477
:10BD100095E120E030E040EA50EC87FD04C020E0EF
:10BD200030E040EA50E4C701B6010E948CE820E010
:10BD300030E040E251E40E940FE90E9481E92B01CA
:10BD40003C0180E277FE09C0709460945094409466
:10BD5000411C511C611C711C8DE28093A80B60E298
:10BD6000F0E14F16F7E25F06610471048CF0C30145
:10BD7000B20120E137E240E050E00E94FFE7CA0153
:10BD8000B9012AE030E040E050E00E94FFE7605D4A
:10BD90006093A90B60E228EE421623E0520661048C
:10BDA00071048CF0C301B20128EE33E040E050E0B2
:10BDB0000E94FFE7CA01B9012AE030E040E050E00C
:10BDC0000E94FFE7605D6093AA0BC301B20124E605
:10BDD00030E040E050E00E94FFE76AE0C62ED12C40
:10BDE000E12CF12CCA01B901A70196010E94FFE7DD
:10BDF000605D6093AB0BC301B201A70196010E9485
:10BE0000FFE76D83CA01B901A70196010E94FFE710
:10BE1000CD80CC2009F40DC38EE28093AC0B605D25
:10BE20006093AD0B2C2D205D2093AE0B68EA7BE078
:10BE300081E294E00E94ABEA20E030E0A901C50174
:10BE4000B4010E9495E120E030E040E05FEB87FD27
:10BE500004C020E030E040E05FE3C501B4010E948F
:10BE60008CE80E9481E9CB010E944018BC018CE162
:10BE700094E00E94ABEA20E030E0A90169817A8178
:10BE80008B819C810E9495E120E030E040E05FEBF7
:10BE900087FD04C020E030E040E05FE369817A8103
:10BEA0008B819C810E948CE80E9481E9CB010E94D9
:10BEB0004018BC0187E194E00E94ABEA4091550232
:10BEC0004F7749830E94CE356D83972E5C01162FE4
:10BED00080910F01C9808C15C1F0C0920F0128E438
:10BEE000C29EB001112490E080E00E949AE12AE015
:10BEF00037ED43E25CE30E94FBE10E9488E9609336
:10BF00001604C110A8C21092110480910E011817D6
:10BF100009F440C0CD80C0920E016C2D792DC50171
:10BF200020E13EE040E050E00E94DDE769015CE393
:10BF3000452E512C612C712C6D81792DC501A301E9
:10BF400092010E94DDE7CA01B901A30192010E949A
:10BF5000DDE724E6C216D10408F0A0C27F936F93F8
:10BF6000DF92CF9281EE91E09F938F9381E094E0F6
:10BF70009F938F930E942CE10FB6F894DEBF0FBE03
:10BF8000CDBF85E0982F990F990F891B880F805896
:10BF9000809300040E9450BF0091FC031091FD03A8
:10BFA0002091FE033091FF036B017C01C01AD10A7E
:10BFB000E20AF30A9701860137FD11C02091FB03C5
:10BFC00020952093FB036A547C4F8F4F9F4F6093C3
:10BFD000FC037093FD038093FE039093FF03D090C6
:10BFE000FB03D98281E00E94DE6A8091A213843132
:10BFF00058F48091A413883038F026E632E04CE003
:10C0000068E080E50E9417BA8091A2138431A0F401
:10C010008091A413823080F0E980EE2031F080918D
:10C020000C0C20E332E0811102C02AEF31E042E142
:10C0300062E088E60E9417BA8091A2138C3108F062
:10C04000E8C0E0900A13F0900B13883028F5809137
:10C050000C1390910D130E94BF18FC01808193E096
:10C06000803229F4818192E0803209F491E043E04A
:10C0700050E0491B51094E0F5F1F892F880F880F11
:10C08000981B892F67E0815F0E94616D69E070E015
:10C0900080E090E00E94EF6A8091A2138C3130F52D
:10C0A0008091A413843110F1C7010E94BF18FC01D4
:10C0B000808193E0803229F4818192E0803209F41A
:10C0C00091E043E050E0491B51094E0F5F1F892F5B
:10C0D000880F880F981B892F6CE1815F0E94616D2A
:10C0E00069E070E080E090E00E94EF6AE090660B0B
:10C0F000F090670B8091A213883028F58091680B2F
:10C100009091690B0E94BF18FC01808193E08032FE
:10C1100029F4818192E0803209F491E043E050E01B
:10C12000491B51094E0F5F1F892F880F880F981BDD
:10C13000892F67E0865A0E94616D69E070E080E0B7
:10C1400090E00E94EF6A8091A2138C3130F58091CB
:10C15000A413843110F1C7010E94BF18FC01808133
:10C1600093E0803229F4818192E0803209F491E0F9
:10C1700043E050E0491B51094E0F5F1F892F880F84
:10C18000880F981B892F6CE1865A0E94616D69E0C7
:10C1900070E080E090E00E94EF6A8091A2138C3101
:10C1A000C0F58091A4138431A0F190910C0C292F3B
:10C1B00030E02115310569F1F980F11084C18091D9
:10C1C000560187FD83C1989F90011124220F232FD0
:10C1D000221F330B31954AE24D8344E6429FC00152
:10C1E000439F900D112481589F4F6FEF70E00E9484
:10C1F0006EE8CB010E94BF18AC016CE187E60E949B
:10C20000616DCD806C2DCC0C770B880B990B0E9447
:10C21000EF6A8091A213853330F48091A4138133A7
:10C2200010F00E94F5B98091A213843368F48091D4
:10C23000A413823348F002E02091160442E367E33E
:10C240008EE693E10E94ADC08091A2138033D8F4B2
:10C250008091A4138832B8F080911104882361F092
:10C2600041E154E060E387E30E94616D65E270E0C4
:10C2700080E090E00E94EF6A41E054E060E380914A
:10C2800000040E94616D8091A213873208F055C0AE
:10C290008091A4138F3108F450C083E08093A513DC
:10C2A00026E2D22ED092A61368E570E080E090E0FE
:10C2B0000E94EF6A8BE08093A513D092A613E980C9
:10C2C000EE2009F406C18CE194E00E94206C88E223
:10C2D0008093A513F6E2F093A61369E570E080E081
:10C2E00090E00E94EF6A80E38093A51396E2C92E46
:10C2F000C092A613D980DD2009F40CC187E194E037
:10C300000E94206C8DE48093A513F6E2F093A613AF
:10C310006AE570E080E090E00E94EF6A85E5809336
:10C32000A51386E2C82EC092A613D980DD2009F499
:10C3300014C181E294E00E94206C8091A2138333A7
:10C3400038F58091A4138B3218F183E00E94DE6AE5
:10C3500083E08093A51383E38093A61366E070E0E7
:10C3600080E090E00E94EF6A81E00E94DE6A8091A6
:10C370001601909117010E94BF18AC0163E38CE095
:10C380000E94616D65E270E080E090E00E94EF6ADB
:10C390008091A213813408F009C18091A4138633DF
:10C3A00008F404C11092A5138EE38093A6138AE2C9
:10C3B00092E00E94CE5D898360E870E08AE292E0BC
:10C3C0000E94C26BF981F53108F0F0C060E270E0C4
:10C3D00080E090E00E94EF6A29812F5F2983F2CFED
:10C3E000243631054CF48536910504F58A309105E3
:10C3F00034F48AE090E009C084369105BCF0883EB0
:10C40000E3E09E0714F087EE93E02817390709F45C
:10C4100028CC90931701809316011092970B1092DD
:10C42000980B1092990B10929A0B1BCC84E690E01B
:10C43000F0CF662351F08EE28093AC0B605D609389
:10C44000AD0B80E28093AE0BF1CC80E28093AD0B1C
:10C450008093AC0BF6CF498181E3443608F480E247
:10C460008093AC0B698190E26A3040F02AE0862F1D
:10C47000622F0E9440E80E9440E8905D9093AD0BCF
:10C4800089816AE00E9440E8905D9093AE0B6CEA6F
:10C490007BE081E194E00E94ABEA37CD7F936F931C
:10C4A000DF92CF9287ED91E09F938F9381E094E0AC
:10C4B0009F938F930E942CE10FB6F894DEBF0FBEBE
:10C4C000CDBF86E05FCD65E26D8387CE85E28D834B
:10C4D00084CE87E00E94402780FF13C00CE114E067
:10C4E000F80161918F01662309F4F1CE6F320CF0EF
:10C4F0006FE3062E000C770B880B990B0E94EF6AF6
:10C50000EFCF8091B90B80FDDECE85EF91E00E94E8
:10C51000BE6BDDCE87E00E944027869580FF13C06A
:10C5200007E114E0F80161918F01662309F4EACE76
:10C530006F320CF06FE3062E000C770B880B990B13
:10C540000E94EF6AEFCF8091B90B869580FDD6CE21
:10C5500085EF91E00E94BE6BD5CE87E00E94402718
:10C560008695869580FF17C081E294E09A8389833F
:10C57000E981FA816191FA83E983662309F4DDCECA
:10C580006F320CF06FE3062E000C770B880B990BC3
:10C590000E94EF6AEDCF8091B90B8695869580FD5C
:10C5A000C8CE8DEE91E00E94BE6BC7CE0F900F906B
:10C5B0000F900F900F90DF91CF911F910F91FF90EF
:10C5C000EF90DF90CF90BF90AF909F908F907F9033
:10C5D0006F905F904F900895AF92BF92CF92DF928D
:10C5E000EF92FF920F931F93CF93DF93EC015B01C8
:10C5F0008A01FB01099587FD16C0C82ED12CF12CAC
:10C60000E12C2196F801C082D182E282F382CE0130
:10C61000DF91CF911F910F91FF90EF90DF90CF901E
:10C62000BF90AF900895982F907E903CA9F48F71A1
:10C6300090E0B0E0A0E06C017D0156E0CC0CDD1C88
:10C64000EE1CFF1C5A95D1F7CE010196F501099514
:10C650008F73C82A2296D6CF982F907F903E11F5DF
:10C660008F7090E0B0E0A0E06C017D0136E0CC0C72
:10C67000DD1CEE1CFF1C3A95D1F7CE010196F501A9
:10C6800009958F73C82A46E0CC0CDD1CEE1CFF1CFC
:10C690004A95D1F7CE010296F50109958F73C82A04
:10C6A0002396B0CF982F987F903F79F5877090E0D0
:10C6B000B0E0A0E06C017D0186E0CC0CDD1CEE1C3E
:10C6C000FF1C8A95D1F7CE010196F50109958F736C
:10C6D000C82A96E0CC0CDD1CEE1CFF1C9A95D1F705
:10C6E000CE010296F50109958F73C82A26E0CC0C7D
:10C6F000DD1CEE1CFF1C2A95D1F7CE010396F50137
:10C7000009958F73C82A24967DCF982F907C9038F6
:10C7100041F4807C803869F42196CE01F5010995B9
:10C72000F8CF8E7F8D3F28F02196CE01F501099537
:10C73000F8CFC12CD12C760165CFAF92BF92CF92AA
:10C74000DF92EF92FF920F931F93CF93DF9300D06E
:10C7500000D0CDB7DEB77C01062F6A01122F86E02C
:10C76000A82EB12C11160CF040C0AE014F5F5F4FE8
:10C770006AEA7DE1C7010E94EC627C0169817A81ED
:10C780008B819C81611571058105910571F16D3376
:10C7900071058105910509F450C06E377105810559
:10C7A000910509F44AC06A3271058105910569F560
:10C7B00007FF12C08DEC91E00E3F11F089EC91E083
:10C7C00026E01202B00111240E94606B66E070E066
:10C7D0000E946EE8161B61C065E470E080E090E0A6
:10C7E0000E94EF6A115059F510E0812F0F900F90C1
:10C7F0000F900F90DF91CF911F910F91FF90EF90CD
:10C80000DF90CF90BF90AF9008956432710581059D
:10C81000910579F4C114D10461F026E01202B0014F
:10C820001124C6010E94606BB5010E946EE8161BC0
:10C8300099CF0E94EF6A115095CF07FDBBCF61E001
:10C8400089819A81AB81BC81CD97A105B10509F49D
:10C8500060E0600F6A30ACF01150862F6AE00E94F1
:10C860004CE8092F682F880F770B605D7F4F072EEC
:10C87000000C880B990B0E94EF6A112309F4B4CFC6
:10C88000602F062E000C770B605D7F4F072E000C8B
:10C89000880B990B0E94EF6A1150112309F4A4CF61
:10C8A00086E01802B0011124C7010E94606B66E0A7
:10C8B00070E00E946EE8161B98CF0F931F93CF93E2
:10C8C000DF938C0160E088EE92E00E949F76C801C1
:10C8D0000E94EC75F80101900020E9F73197EF0113
:10C8E000C01BD10BCB32D1052CF08291807C8038DB
:10C8F000E1F3F5CFDD27AE01B8018AE292E00E94B4
:10C90000C0EAC65DDD4F1882DF91CF911F910F9174
:10C910000895EF92FF920F931F93CF93DF93CDB7BC
:10C92000DEB762970FB6F894DEBF0FBECDBF0E9490
:10C930004027882309F448C043E252E082FF02C046
:10C9400046E252E023E232E081FF02C023E132E01E
:10C9500080FD37C083E292E05F934F933F932F9324
:10C960009F938F9384E798E09F938F938E010F5F3F
:10C970001F4F1F930F930E942CE10E94597CC80106
:10C980000E94EC750FB6F894DEBF0FBECDBF80914C
:10C990005A02811103C0C8010E945D640FB6F89469
:10C9A000DEBF0FBECDBF81E062960FB6F894DEBF4A
:10C9B0000FBECDBFDF91CF911F910F91FF90EF90F0
:10C9C000089585E192E0C8CF80E0EECF1198000095
:10C9D000000087FD52C0419800000000119A00003D
:10C9E000000011980000000086FD53C0419800002F
:10C9F0000000119A0000000011980000000085FD61
:10CA000046C0419800000000119A000000001198F3
:10CA10000000000084FD39C0419800000000119A18
:10CA20000000000011980000000083FD2CC0419818
:10CA300000000000119A00000000119800000000A2
:10CA400082FD1FC0419800000000119A0000000004
:10CA500011980000000081FD12C041980000000004
:10CA6000119A000000001198000000004198000099
:10CA70000000119A000000000895419AADCF419A3C
:10CA8000EDCF419AE0CF419AD3CF419AC6CF419A98
:10CA9000B9CF419AACCF089590E080E00895282F57
:10CAA00090910705833021F495FD0FC094FD0FC0D0
:10CAB000892F90E0B0E0A0E004C0B695A7959795C7
:10CAC00087952A95D2F78170089581E0089580E0D6
:10CAD00008952F923F924F925F926F927F928F9222
:10CAE0009F92AF92BF92CF92DF92EF92FF920F93FD
:10CAF0001F93CF93DF93CDB7DEB72E970FB6F89481
:10CB0000DEBF0FBECDBFE82ED62E042F122F282F4A
:10CB100030E03C872B87462F50E05A87498765E0F5
:10CB2000F62EF29EC001F39E900D11249E878D87F4
:10CB3000FA01E80FF91FEE0FFF1FEE0FFF1FEF576F
:10CB4000FD4F60817181828193819B01AC010E94C4
:10CB50008DEA882309F434C1E00E612F6D0DFE9C2F
:10CB6000F0011124A985BA85AE0FBF1FAA0FBB1F04
:10CB7000AA0FBB1FAF57BD4FAC901196BC90119739
:10CB80001296CC9012971396DC90E00EFE9CA001BA
:10CB90001124A985BA85A40FB51FAA0FBB1FAA0F20
:10CBA000BB1FAF57BD4FEC901196FC90119712969A
:10CBB0000C91129713969C90862F90E0AD85BE85C0
:10CBC000A80FB91FAA0FBB1FAA0FBB1FAF57BD4F9E
:10CBD0008C9011967C90119712966C9012971396E8
:10CBE0005C90610F70E0AD85BE85A60FB71FAA0FE0
:10CBF000BB1FAA0FBB1FAF57BD4F4C9011963C9067
:10CC0000119712961C91129713962C90E80FF91F0A
:10CC1000EE0FFF1FEE0FFF1FEF57FD4FB081B983DF
:10CC200021812A8332813B8383818C83FA01E60F41
:10CC3000F71FEE0FFF1FEE0FFF1FEF57FD4F908105
:10CC40009D83A181AE83B281BF8323812887970111
:10CC5000402F592DB701802F992D0E948DEA8823EE
:10CC600021F0E12CF12C00E0912C9501A601B501F9
:10CC7000C6010E948DEA882319F05701C02ED92CD5
:10CC8000242D332D412F522D642D732D812F922D64
:10CC90000E948DEA882321F0412C312C10E0212CB8
:10CCA000282D372D462D552D682D772D862D952D28
:10CCB0000E948DEA882321F0842C732C612E522C43
:10CCC0002D813E814F8158856D817E818F81988530
:10CCD0000E948DEA882321F01D821E821F82188601
:10CCE00029813A814B815C8169817A818B819C8128
:10CCF0000E948DEA882341F03D8139834E814A8329
:10CD00005F815B8388858C8385E0EB85FC858E9FC6
:10CD1000D0018F9FB00D112429853A85A20FB31F32
:10CD2000AA0FBB1FAA0FBB1FAF57BD4FBA87A9875A
:10CD30009501A601B501C6010E948CE89701402F1C
:10CD4000592D0E948BE86B017C01282D372D462D33
:10CD5000552D682D772D862D952D0E948CE8242D3C
:10CD6000332D412F522D0E948BE89B01AC01C7014E
:10CD7000B6010E948CE86B017C0129813A814B81CC
:10CD80005C8169817A818B819C810E948CE82D81F4
:10CD90003E814F8158850E948BE89B01AC01C70101
:10CDA000B6010E948CE820E030E040E450E40E94AC
:10CDB0000FE9A985BA856D937D938D939C93139705
:10CDC0002E960FB6F894DEBF0FBECDBFDF91CF9188
:10CDD0001F910F91FF90EF90DF90CF90BF90AF9099
:10CDE0009F908F907F906F905F904F903F902F908B
:10CDF0000895AF92BF92CF92DF92EF92FF920F937E
:10CE00001F93CF93DF936B01E9014A3009F4B8C057
:10CE1000453109F06AC0DB011296ED91FC91F28078
:10CE2000C681D781139A88E28A950000E9F7BF2C62
:10CE3000B29420EFB22230E1A32EAF0C48E2E42EF0
:10CE400088EF0E94E6648E2D8A950000E9F7BFE125
:10CE5000BF1508F481C08F2D807780680E94E6643A
:10CE60008B2D0E94E6648E2D8A950000E9F780E8FC
:10CE70000E94E66480E00E94E6648E2D8A950000A0
:10CE8000E9F78AEF0E94E6648E2D8A950000E9F7A3
:10CE90008E01005F1F4F8881807F0E94E664899128
:10CEA0008295807F0E94E664C017D107A1F78E2D7E
:10CEB0008A950000E9F7F394E0E1BE0EFA10C0CFC6
:10CEC0001398D6011296CD91DC91CE010E9490C0AC
:10CED0008111EEC1DF91CF911F910F91FF90EF90E3
:10CEE000DF90CF90BF90AF900895FB010281138136
:10CEF000423309F498C108F49CC1463409F489C14D
:10CF0000473409F48CC14B3329F589812B81D80131
:10CF100012966C91129713964C91213009F4DFC14F
:10CF2000233009F0A9C138EF380F582F91E043178B
:10CF300008F490E041E0531708F040E031E0561764
:10CF400008F430E0592F542B352309F0BDC1942348
:10CF500009F0BAC181E0BECF80EE8F0D8068807F7E
:10CF60000E94E6648F2D8295807F0E94E6648E2D5C
:10CF70008A950000E9F780E80E94E66480E87BCFAC
:10CF80000B9A1398399A4198099A119A139A88E240
:10CF90008A950000E9F788E790E0CEE9DFE0FE013E
:10CFA0003197F1F70197D9F788EF0E94E66418E20C
:10CFB000812F8A950000E9F780E20E94E66480E014
:10CFC0000E94E664812F8A950000E9F780E00E94C4
:10CFD000E66480E80E94E664812F8A950000E9F704
:10CFE00080E00E94E66480E10E94E664812F8A95D9
:10CFF0000000E9F7CE010197F1F7CE010197F1F7B3
:10D00000CE010197F1F7CE010197F1F7CE0101971B
:10D01000F1F7CE010197F1F7CE010197F1F7CE01BB
:10D020000197F1F7CE010197F1F7CE010197F1F7E2
:10D03000CE010197F1F7CE010197F1F7CE010197EB
:10D04000F1F7CE010197F1F72197F1F780E20E9405
:10D05000E66480E40E94E664812F8A950000E9F787
:10D0600080E20E94E66480E60E94E6641A95000071
:10D07000E9F710E0D0E0C8E28D2F807780680E9449
:10D08000E664812F0E94E6648C2F8A950000E9F700
:10D0900080E80E94E66480E00E94E6648C2F8A9516
:10D0A0000000E9F78AEF0E94E6648C2F8A95000061
:10D0B000E9F780E2119800000000419800000000AC
:10D0C000119A000000001198000000004198000033
:10D0D0000000119A00000000119800000000419823
:10D0E00000000000119A00000000119800000000EC
:10D0F000419800000000119A000000001198000003
:10D100000000419800000000119A000000001198F2
:10D1100000000000419800000000119A000000008B
:10D12000119800000000419800000000119A0000D2
:10D130000000119800000000419800000000119AC2
:10D14000000000001198000000004198000000005D
:10D15000119A0000000011980000000041980000A2
:10D160000000119A00000000119800000000419892
:10D1700000000000119A000000001198000000005B
:10D18000419800000000119A000000001198000072
:10D190000000419800000000119A00000000119862
:10D1A00000000000419800000000119A00000000FB
:10D1B000119800000000419800000000119A000042
:10D1C0000000119800000000419800000000119A32
:10D1D000000000009C2F9A950000E9F7815009F0AB
:10D1E00069CF88EF0E94E6648C2F8A950000E9F7EA
:10D1F000DF5F105FD03209F03FCF80E00E94E6642D
:10D2000080EC0E94E664CA950000E9F7139881E07B
:10D2100061CED80115968C91888381E05BCEF801B0
:10D2200081818883FACFB901C8010E9471C281E06F
:10D2300051CE443171F0473109F08CCE1882F8019B
:10D2400082818983858181508A8383818B8381E078
:10D2500041CED80115964C91159750E0440F551FBB
:10D2600070E060E016968D919C910E9499EAC80149
:10D270000E94A6C081E02ECE481708F46BCE861718
:10D2800008F468CEFA80E12CD12C243070F41DC053
:10D29000BE01C8010E9471C2898198819D0D988349
:10D2A0008E0D8983FF0C09F455CEF7FEF6CFF0CF33
:10D2B0004D8150E0440F551F70E060E08E819F81EA
:10D2C0000E9499EA81E006CEFA8030E0F901E75049
:10D2D000FE4FD0802B503E4FF901E080E6CF58E062
:10D2E000580F382F23CEEF92FF920F931F93CF93B7
:10D2F000DF93EC018B017A018A859B85861797075E
:10D3000031F0888199810E94B9C21B870A87B701D1
:10D31000888199810E945FBA2E813F81820F932F6D
:10D32000911D9F838E8390E080E0DF91CF911F91CC
:10D330000F91FF90EF9008959F92AF92BF92CF927E
:10D34000DF92EF92FF920F931F93CF93DF93EC0145
:10D350008B01942EA52E8A859B858617970731F021
:10D36000888199810E94B9C21B870A87888599851F
:10D37000019649F5BC800A818E81080FC880D9804A
:10D38000D6015596ED91FC91C6010995B80EE92C90
:10D39000FA2C10E0F70121917F01211127C08E8125
:10D3A0009F81810F911D9F838E8390E080E0DF91AC
:10D3B000CF911F910F91FF90EF90DF90CF90BF9092
:10D3C000AF909F9008950E811F81692D7A2D8881DD
:10D3D00099810E945FBA800F912F911D2885398510
:10D3E0002817390738F681E090E0E1CF4B2D602F08
:10D3F000C6010E9411C3080F180FCCCFDF92EF9225
:10D40000FF920F931F93CF93DF93EC01D62E1CADA9
:10D410000BAD7C0184E0E80EF11CE98DFA8DC701AB
:10D420000995412F480F2D2D602FC7010E9411C370
:10D430009BAD890F8BAF81E090E0DF91CF911F9181
:10D440000F91FF90EF90DF900895EF92FF920F936E
:10D450001F93CF937C0100910A0510910B05C0E04A
:10D46000F701EC0FF11D6081662351F0062E000CD0
:10D47000770BC8010E94A0EA892B49F4CF5FF0CF57
:10D4800080E0CF911F910F91FF90EF90089581E080
:10D49000F8CFCF93DF9300D000D0CDB7DEB780E0D8
:10D4A00090E0A0EAB0E489839A83AB83BC8361E017
:10D4B000CE0101960E94F02B0F900F900F900F90CD
:10D4C000DF91CF9108958091FD049091FE04009723
:10D4D00031F04AE050E070E060E00C94C2DF60E0C0
:10D4E00070E0CB0108958091FD049091FE040097B7
:10D4F00031F04AE050E070E060E00C9494DE60E0CF
:10D5000070E0CB0108950E94736A97FD0CC00E94E1
:10D51000736A6F3F71058105910509F034F40E942B
:10D52000736A862F089580E008958FEF08958091A3
:10D53000FD049091FE04892B41F00E94836A91E0E2
:10D54000811101C090E0892F089591E0FCCF9CE00B
:10D55000899F802D112491E0980F909310052CE065
:10D56000280F2093B50B30E02E5F3F4F4091A21360
:10D570004217130619F014F080E008952091A413C7
:10D580009217D0F7662341F08E5F0E943EB98091DA
:10D59000B50B8E5F0E943EB98091B50B9091A2139E
:10D5A000891750F32091A41390911005291720F3A7
:10D5B0001092A5138093A61381E0089520910F0582
:10D5C000022E000C330B8217130641F080930F05D7
:10D5D00068EA76E18EE693E10C94B9C20895CF92A1
:10D5E000DF92EF92FF920F931F93CF93DF93CDB70C
:10D5F000DEB72C970FB6F894DEBF0FBECDBF6F3FDE
:10D6000071058105910509F0D0F48AE693E10E9445
:10D61000FE69E0917213F09173133196849190E05A
:10D620002C960FB6F894DEBF0FBECDBFDF91CF9121
:10D630001F910F91FF90EF90DF90CF900895F090A1
:10D64000A513E090A6132091280221110FC048E8ED
:10D6500056E16E2D8F2D0E947DC390E080E0F80E84
:10D66000F092A513E092A6139927DACFC090721317
:10D67000D09073132EE633E13A8329832F2D30E0C7
:10D680003C832B832E2D30E03E832D8318861F8212
:10D690002FEF3FEF3A8729871C861B860CE919E696
:10D6A0009E012F5F3F4FAB01BC01C6010E94C0B27B
:10D6B000B6018EE693E10E94B9C28F819885CFCFE3
:10D6C000CF92DF92EF92FF920F931F93CF93DF934E
:10D6D000CDB7DEB72C970FB6F894DEBF0FBECDBF27
:10D6E000F090A513E090A6132091280221111DC0EF
:10D6F00048E656E16E2D8F2D0E947DC390E080E0BC
:10D70000F80EF092A513E092A61399272C960FB667
:10D71000F894DEBF0FBECDBFDF91CF911F910F9167
:10D72000FF90EF90DF90CF900895C0907213D0904B
:10D7300073132EE633E13A8329832F2D30E03C83A7
:10D740002B832E2D30E03E832D8318861F827A870F
:10D7500069871C861B860CE919E69E012F5F3F4FE7
:10D760004AEA5DE1BC01C6010E9484B3B6018EE6BF
:10D7700093E10E94B9C28F819885C2CF6FEF7FEF8E
:10D780000C94606BCF92DF92EF92FF920F931F93F6
:10D79000CF93DF93CDB7DEB72C970FB6F894DEBFEB
:10D7A0000FBECDBFF090A513E090A61320912802E4
:10D7B00021111DC048E456E16E2D8F2D0E947DC3BE
:10D7C00090E080E0F80EF092A513E092A61399275E
:10D7D0002C960FB6F894DEBF0FBECDBFDF91CF9170
:10D7E0001F910F91FF90EF90DF90CF900895C09020
:10D7F0007213D09073132EE633E13A8329832F2DD1
:10D8000030E03C832B832E2D30E03E832D83188621
:10D810001F827A8769871C861B860CE919E69E01A0
:10D820002F5F3F4F4DEA5DE1BC01C6010E9484B30A
:10D83000B6018EE693E10E94B9C28F819885C2CF6E
:10D840006FEF7FEF0C94C26BAF92BF92CF92DF92DB
:10D85000EF92FF920F931F93CF93DF935C016B01C5
:10D860000E94C25DE82EC6010E94CE5DF12C03E14C
:10D8700010E0081B1109C5E20E151F050CF4CFE1DD
:10D880008C2F90E09C012E5F3F4F4091A2134217D6
:10D89000130609F0CCF509972091A413281719064F
:10D8A0009CF14091B70B5091B80B6091B60B109260
:10D8B000A513C093A61325E1C5010E949D63D1E085
:10D8C000C114D104B1F06AE370E080E090E00E94FE
:10D8D000EF6A0E151F05D4F4C45F8091A213C81718
:10D8E00040F02091A4134C2F4950550B24171506D6
:10D8F0007CF4DF91CF911F910F91FF90EF90DF901B
:10D90000CF90BF90AF900895D0E0DACFDD2389F3B8
:10D91000802F880F080F000F0093A513C093A61344
:10D9200060E270E080E090E00E94EF6AC601DF9163
:10D93000CF911F910F91FF90EF90DF90CF90BF900C
:10D94000AF900C94206C8F929F92AF92BF92CF9227
:10D95000DF92EF92FF920F931F93CF93DF93CDB798
:10D96000DEB72C970FB6F894DEBF0FBECDBF982F51
:10D97000862F5A017901D02E692F0E94A76A882329
:10D9800009F489C0C701002391F10E94C25DC82E2D
:10D99000809072139090731380912802811145C07A
:10D9A0001FEF23E12C194091B70B5091B80B6091F8
:10D9B000B60BC5010E949D63CC2009F46CC0B6E093
:10D9C0008B9F500111246AE370E080E090E00E9498
:10D9D000EF6A57E0A516B10408F444C060E270E0B5
:10D9E00080E090E00E94EF6AA81AB90AF2CF0E9484
:10D9F000CE5DC82E80907213909073138091280290
:10DA0000882371F2FE0133968AE0DF011D928A9528
:10DA1000E9F78EE693E19A83898303E719E69E018D
:10DA20002F5F3F4F4DEA5DE112C0FE0133968AE061
:10DA3000DF011D928A95E9F78EE693E19A83898347
:10DA400003E719E69E012F5F3F4F4AEA5DE1B70108
:10DA5000C4010E9484B3B4018EE693E10E94B9C26E
:10DA60001F819FCF4091B50B212F30E0A6E0CA9EC9
:10DA7000C00111242E5F3F4F281739070CF49C0179
:10DA800080E8821B8093A5134093A613C701DD2075
:10DA9000A9F00E94BE6B2C960FB6F894DEBF0FBEA5
:10DAA000CDBFDF91CF911F910F91FF90EF90DF904D
:10DAB000CF90BF90AF909F908F9008950E94206C60
:10DAC000EACFEAE6F3E183AF64AFCA010C94206CBD
:10DAD0000F931F93CF9310920905109208052FE31F
:10DAE00020930E0510920D0510920C059C01F90172
:10DAF00090812F5F3F4F9032D1F39E34C9F48181E2
:10DB000090ED980F9A3020F08D3211F08B3281F425
:10DB100032969F012F5F3F4F808180538A3008F4F7
:10DB200068C09F012F5F3F4F8081803209F463C03E
:10DB3000F093C40BE093C30B8F010F5F1F4FC081A5
:10DB40006AE270E0C8010E94A0EA009731F0FC018F
:10DB5000319780818032E1F31182CD3429F0C435D0
:10DB600019F0C73409F041C0F80180810F5F1F4FE1
:10DB70008032D1F380538A30C0F5C0930E0530E077
:10DB800020E06AE0AF014F5F5F4F629FC001639F7B
:10DB9000900D11249C01205331098081280F311DE3
:10DBA00087FD3A95FA01808180538A3058F330938B
:10DBB0000D0520930C05CA01FC01019640814032FD
:10DBC000D9F3F0930B05E0930A05CD3401F52E311E
:10DBD000310539F090F42731310519F02C31310538
:10DBE000B1F4F0930905E0930805CF911F910F91CF
:10DBF0000895F9018ECFF90194CF2537310538F01A
:10DC00002737310570F3203A83E0380751F350E0AD
:10DC100040E0CF0101966081662309F45AC0613269
:10DC200091F4CD3481F42032310569F490930905E3
:10DC30008093080563E270E00E94A0EA0097A9F2D1
:10DC4000FC011082D2CFFC01DF018D91803271F096
:10DC500090ED980F9A3008F18E3251F491819053E3
:10DC60009A30D8F041155105E1F414C0FD01ECCF14
:10DC70008D3211F08B3259F4918160ED690F6A3069
:10DC800060F09E3221F4928190539A3030F0411529
:10DC9000510519F4AF014150510981548A3108F4FA
:10DCA000B8CFDF01FD018D91882309F4B2CF90ED4B
:10DCB000980F9A30B8F393ED980F923098F38B3217
:10DCC00089F3CF0101966081603209F0A2CFFC0197
:10DCD000F8CF509309054093080587CFFC01659163
:10DCE00075918591949108958091BA0B882319F0CC
:10DCF00080E00E94493380E008954F925F926F92D6
:10DD00007F928F929F92AF92BF92CF92DF92EF92CB
:10DD1000FF92CF93DF93CDB7DEB728970FB6F89475
:10DD2000DEBF0FBECDBF5C01DB01CD90DD90ED907D
:10DD3000FC90E0915113F0915213FE83ED838481A6
:10DD40009581A681B78189839A83AB83BC839C012B
:10DD5000AD01C701B6010E948BE82B013C01F50122
:10DD600080809180A280B380AD81BE818D919D9194
:10DD70000D90BC91A02D8D839E83AF83B88727E142
:10DD800037EB41ED58EBC301B2010E940FEA87FD6A
:10DD9000D1C027E030E04CE553E4C301B2010E945A
:10DDA00095E118160CF4C6C02D813E814F8158852F
:10DDB000C501B4010E948BE82B013C0127E137EB40
:10DDC00041ED58EB0E940FEA87FDB4C023E030E03C
:10DDD00046E953E4C301B2010E9495E118160CF420
:10DDE000A9C020E030E0A9016D817E818F819885F6
:10DDF0000E948CE82B013C0120E030E040E450E43C
:10DE00000E9495E187FF05C0412C512C30E4632E20
:10DE1000762C27E137EB41ED58E3C301B2010E94B4
:10DE20008BE89B01AC01C501B4010E940FEA87FD9C
:10DE300081C020E030E046E953E46D817E818F812E
:10DE400098850E948CE82B013C0120E030E844E9F1
:10DE500053E40E940FEA18163CF4412C20E8522E9D
:10DE600024E9622E23E4722E27E137EB41ED58E3DB
:10DE7000C301B2010E948CE89B01AC01C501B40151
:10DE80000E9495E118160CF455C020E030E0A9017D
:10DE900069817A818B819C810E948CE84B015C01B5
:10DEA00020E030E040E951E40E9495E187FF06C0A0
:10DEB000812C912C90E9A92E91E4B92E27E137EB22
:10DEC00041ED58E3C501B4010E948BE89B01AC0110
:10DED000C701B6010E940FEA87FD2CC020E030E0A8
:10DEE0004CE553E469817A818B819C810E948CE8A6
:10DEF0004B015C0120E030E04AE453E40E940FEA69
:10DF0000181634F4812C912C8AE4A82E83E4B82EC0
:10DF100027E137EB41ED58E3C501B4010E948CE8DD
:10DF20009B01AC01B1E0B983C701B6010E9495E144
:10DF300018160CF41982898128960FB6F894DEBF62
:10DF40000FBECDBFDF91CF91FF90EF90DF90CF90CC
:10DF5000BF90AF909F908F907F906F905F904F9009
:10DF600008950E94736ACB0108950F931F93CF9376
:10DF70008091FD049091FE040097E9F0FC018F016F
:10DF8000C1912C2F2F7D81F0C53411F0C536B9F722
:10DF9000F801108270E060E00E9436DDF801C08375
:10DFA000CF911F910F91089570E060E0CF911F9184
:10DFB0000F910C9436DD60E070E0CB01F1CF682F5B
:10DFC000880F770B80910A0590910B050E94A0EABB
:10DFD000FC0181E0309709F480E0309781F0918175
:10DFE00020ED290F2A3030F09E3251F49281905367
:10DFF0009A3098F43196F093FE04E093FD0408956E
:10E000009D3211F09B3249F4928120ED290F2A3084
:10E0100088F39E3211F49381EACFF0E0E0E0EBCF99
:10E020000E94DF6F882341F081E02091FD04309150
:10E03000FE04232B09F480E00895CF93DF93EB01D6
:10E040000E941070882321F0DF91CF910C94B16F62
:10E05000CE01DF91CF910895CF93C62F0E9410700B
:10E06000882319F0CF910C94836A8C2FCF91089557
:10E07000CF92DF92EF92FF926A017B010E941070B3
:10E08000882331F0FF90EF90DF90CF900C94B56F24
:10E09000C701B601FF90EF90DF90CF900895CF9326
:10E0A000DF93C82FD62F0E941070882321F0DF91B4
:10E0B000CF910C94976A8C2F0E94DF6F811101C061
:10E0C0008D2FDF91CF9108954F925F926F927F9243
:10E0D0008F929F92AF92BF92CF92DF92EF92FF9278
:10E0E0000F931F93CF93DF93EC012091E5023091C2
:10E0F000E6024091E7025091E802688179818A81C5
:10E100009B810E948BE86B017C012091E902309198
:10E11000EA024091EB025091EC026C817D818E818C
:10E120009F810E948BE84B015C01A70196016091E1
:10E1300042017091430180914401909145010E94F8
:10E1400095E1882309F450C0C0924201D092430166
:10E15000E0924401F09245012091F5043091F604DB
:10E160004091F7045091F804C701B6010E94FBE109
:10E170002B013C010E94B7E96B017C0120E030E0FB
:10E18000A9010E9495E187FD70C020E030E040E4E5
:10E1900050E4C701B6010E940FEA18162CF4C12CF6
:10E1A000D12CC0E4EC2EFE2CA7019601C301B201D4
:10E1B0000E948BE86093ED047093EE048093EF046B
:10E1C0009093F004C701B6010E9481E96093EB04CB
:10E1D000062E000C770B6F5F7F4F6430710514F0D3
:10E1E00064E070E06093E904D09140011091EB0489
:10E1F000A501940160914601709147018091480109
:10E20000909149010E9495E1811133C0D11381C0E1
:10E210002091D1043091D2044091D3045091D40480
:10E220006091ED047091EE048091EF049091F00400
:10E230000E94FBE12091D5043091D6044091D7048F
:10E240005091D8040E948CE8DF91CF911F910F91DB
:10E25000FF90EF90DF90CF90BF90AF909F908F9006
:10E260007F906F905F904F900895C12CD12C7601D4
:10E270009BCF8092460190924701A0924801B092B4
:10E2800049012091F9043091FA044091FB04509126
:10E29000FC04C501B4010E94FBE14B015C010E943A
:10E2A000B7E96B017C0120E030E0A9010E9495E113
:10E2B00087FDF3C020E030E040E450E4C701B60140
:10E2C0000E940FEA18162CF4C12CD12CB0E4EB2ECE
:10E2D000FE2CA7019601C501B4010E948BE8609352
:10E2E000F1047093F2048093F3049093F404C70153
:10E2F000B6010E9481E96093EC04062E000C770BB6
:10E300006F5F7F4F6430710514F064E070E06093DC
:10E31000EA04C091EC04D11305C0809141018C172F
:10E3200009F470C08091EB049091EC04909341014A
:10E33000809340010C2E000CDD0B25E01203C00180
:10E340001124FC01EC0FFD1FEE0FFF1FEE0FFF1F4E
:10E35000EF57FD4F20813181428153812093E504A5
:10E360003093E6044093E7045093E8040091EA04F4
:10E37000002E000C110BFC01E00FF11FEE0FFF1F30
:10E38000EE0FFF1FEF57FD4F6081718182819381F6
:10E390000E948BE86093E1047093E2048093E304AD
:10E3A0009093E4042091E90435E02303F001112463
:10E3B000CE0FDF1FCC0FDD1FCC0FDD1FCF57DD4F82
:10E3C000288139814A815B812093DD043093DE040A
:10E3D0004093DF045093E004E00FF11FEE0FFF1FA6
:10E3E000EE0FFF1FEF57FD4F608171818281938196
:10E3F0000E948BE86093D9047093DA048093DB0465
:10E400009093DC048090F1049090F204A090F304C7
:10E41000B090F4042091E1043091E2044091E304CF
:10E420005091E404C501B4010E94FBE12091E50490
:10E430003091E6044091E7045091E8040E948CE892
:10E440006B017C01C092D504D092D604E092D7042F
:10E45000F092D8042091D9043091DA044091DB0481
:10E460005091DC04C501B4010E94FBE12091DD0460
:10E470003091DE044091DF045091E0040E948CE86A
:10E48000A70196010E948BE86093D1047093D20497
:10E490008093D3049093D404BBCEC12CD12C7601AD
:10E4A00018CF1F93CF93DF93CDB7DEB72C970FB65E
:10E4B000F894DEBF0FBECDBF182F882379F020E07F
:10E4C00030E0A9016091ED027091EE028091EF02BF
:10E4D0009091F0020E9495E18823F9F080917B02EF
:10E4E0008117D9F00E940B228CE0E9EDF1E0DE010A
:10E4F000119601900D928A95E1F7CE0101960E9446
:10E50000647080917B02882391F084ED9BE00E94EF
:10E51000442210927B020E94C82C2C960FB6F894CD
:10E52000DEBF0FBECDBFDF91CF911F91089581E077
:10E5300080937B0284ED9BE00E942C22ECCF80E054
:10E540000E9451721092E9021092EA021092EB02BC
:10E550001092EC021092E5021092E6021092E7028D
:10E560001092E8021092F1021092F2021092F3025D
:10E570001092F4021092ED021092EE021092EF024D
:10E580001092F002E1E8F2E025EE32E080E090E067
:10E59000A0ECBFE780839183A283B38384839583B8
:10E5A000A683B78380879187A287B387848795875F
:10E5B000A687B787808B918BA28BB38B74962E170F
:10E5C0003F0741F708958F929F92AF92BF92CF92EB
:10E5D000DF92EF92FF92C090ED02D090EE02E090B9
:10E5E000EF02F090F00220E030E0A901C701B6018F
:10E5F0000E9495E18823E1F1A701960160E070E0B7
:10E6000080E89FE30E940FE96B017C018090F1029A
:10E610009090F202A090F302B090F40220E030E07B
:10E62000A901C501B4010E9495E1882329F1A50142
:10E63000940160E070E080E89FE30E940FE9C092DF
:10E64000F504D092F604E092F704F092F804609397
:10E65000F9047093FA048093FB049093FC04FF90F8
:10E66000EF90DF90CF90BF90AF909F908F900895E4
:10E67000C12CD12C7601CACF60E070E0CB01DFCF96
:10E68000EFE6F0E080818260808308958091C00B86
:10E690009091C10B892B79F48091C00B9091C10BA3
:10E6A000892B49F42091C00B3091C10B81E0232BC1
:10E6B00019F480E0089581E00895CF92DF92EF92FF
:10E6C000FF926B017C0183E3C816D104E104F104DD
:10E6D00070F082E3C81AD108E108F10862E370E043
:10E6E00080E090E00E94B5BE0E94EEC7ECCFC7016B
:10E6F000B6010E94B5BEFF90EF90DF90CF900C94D2
:10E70000EEC75E9A8091B90B8E7F8093B90B5E9AAB
:10E710008091B90B8D7F8093B90B159A8091B90BBD
:10E720008B7F8093B90B5E9A089581E00895DC0198
:10E73000EC918E2F90E0FC01EE0FFF1FE80FF91F08
:10E74000E35EFC4E80818F77808308951092900065
:10E7500082E0809391001092950010929400C19AEB
:10E76000E1E7F0E080818260808308957F928F925C
:10E770009F92AF92BF92CF92DF92EF92FF920F9350
:10E780001F93CF93DF93EC017B0188818C3008F0DD
:10E79000C4C090E0FC01EE0FFF1FE80FF91FE35E1D
:10E7A000FC4E80818F770E9464B419821A8288811E
:10E7B0002CE0622F0E9440E8829FB001112430E0DB
:10E7C00020E0AB01420F531FFA01EE0FFF1FE40FD1
:10E7D000F51FE35EFC4E908197FD09C02F5F3F4F10
:10E7E0002C30310571F7811102C00E94A673788028
:10E7F000072D10E06801CC0CDD1CF601E00FF11FC5
:10E80000E35EFC4E80818068808377FC86C080E276
:10E81000E81682E0F8060CF03FC08A8128E532E075
:10E82000281B310987FD3395220F331F220F331F19
:10E83000032E000C440B550B898178E8872E912C10
:10E84000881A910887FD9394880C991C880C991C50
:10E85000092C000CAA08BB0860E070E0CB01F7FCB3
:10E860000AC0B701653B710514F064EB70E0072E38
:10E87000000C880B990B281939094A095B090E9479
:10E88000CDE724EB30E040E050E00E94FFE7820E4D
:10E89000931EA41EB51E74018BE08715D8F0298144
:10E8A00088E890E0821B910927FD9395880F991FB6
:10E8B000880F991FE816F90604F502972FB7F89408
:10E8C000E601C00FD11FC35EDC4E880F991F9A83EB
:10E8D00089832FBF62E370E080E090E0DF91CF9109
:10E8E0001F910F91FF90EF90DF90CF90BF90AF906E
:10E8F0009F908F907F900C945D732A8188E592E0C1
:10E90000821B910927FD9395880F991F880F991FE6
:10E91000E816F90694F6C701D0CFDF91CF911F9189
:10E920000F91FF90EF90DF90CF90BF90AF909F90AE
:10E930008F907F900895CF93DF93EB01682F70E065
:10E9400082E493E10E94B673688179818A819B8118
:10E95000643F21E072078105910520F464EF71E0C6
:10E9600080E090E00E945D7386B182958170DF91B6
:10E97000CF910895CF93DF9300D000D0CDB7DEB70D
:10E980008EEE92E0A0E0B0E089839A83AB83BC83F3
:10E99000BE016F5F7F4F8AE50E949B740F900F90BE
:10E9A0000F900F90DF91CF910895CF93DF9300D018
:10E9B00000D0CDB7DEB78EEE92E0A0E0B0E0898364
:10E9C0009A83AB83BC83BE016F5F7F4F8AE00E9456
:10E9D0009B740F900F900F900F90DF91CF9108953F
:10E9E000CF93DF9300D000D0CDB7DEB784EF91E0B6
:10E9F000A0E0B0E089839A83AB83BC83BE016F5FE4
:10EA00007F4F8CE30E949B740F900F900F900F909C
:10EA1000DF91CF910895CF93DF9300D000D0CDB791
:10EA2000DEB784EF91E0A0E0B0E089839A83AB8306
:10EA3000BC83BE016F5F7F4F80EA0E949B740F9082
:10EA40000F900F900F90DF91CF9108951F920F922A
:10EA50000FB60F9211240BB60F922F933F934F9343
:10EA60005F936F937F938F939F93AF93BF93EF9336
:10EA7000FF938091BB0487FF27C0109295001092EE
:10EA800094008091BB048F5F8093BB048091BB0492
:10EA9000082E000C990B209141132817190629F014
:10EAA00024F08091BB048C30DCF180919400909133
:10EAB0009500049680349C4908F47DC080919400B0
:10EAC00090919500049679C08091BB04082E000CAB
:10EAD000990B209141132817190699F294F2E091AD
:10EAE000BB048E2FEE0F990BFC01EE0FFF1FE80FFA
:10EAF000F91FE35EFC4E808187FFC3CFE091BB042A
:10EB00008E2FEE0F990BFC01EE0FFF1FE80FF91F80
:10EB1000E35EFC4E808160E08F770E9459BEB1CFEA
:10EB20002091940030919500E091BB048E2FEE0F60
:10EB3000990BFC01EE0FFF1FE80FF91FE35EFC4E7F
:10EB400081819281820F931F909399008093980006
:10EB5000E091BB048E2FEE0F990BFC01EE0FFF1F0F
:10EB6000E80FF91FE35EFC4E808187FF11C0E09142
:10EB7000BB048E2FEE0F990BFC01EE0FFF1FE80F69
:10EB8000F91FE35EFC4E808161E08F770E9459BEE1
:10EB9000FF91EF91BF91AF919F918F917F916F9175
:10EBA0005F914F913F912F910F900BBE0F900FBE31
:10EBB0000F901F90189580E49CE9909399008093A2
:10EBC00098008FEF8093BB04E3CF9091C00095FF36
:10EBD000FCCF8093C6000895CF93DF93EC01899119
:10EBE000882319F00E94E575FACF8DE00E94E57543
:10EBF0008AE0DF91CF910C94E575CF92DF92EF928E
:10EC0000FF920F931F93CF93DF93CDB7DEB7A097FB
:10EC10000FB6F894DEBF0FBECDBF442309F445C044
:10EC2000611571058105910579F100E0C42ED12CA3
:10EC3000F12CE12CA70196010E94DDE711E0100FF5
:10EC4000E1E0F0E0EC0FFD1FE00FF11D07FDFA958C
:10EC50006083B901CA01012F611571058105910514
:10EC600049F7115010F1E1E0F0E0EC0FFD1FE10F6A
:10EC7000F11D17FDFA95908187E39A3008F480E33F
:10EC8000890F0E94E575EDCF80E3A0960FB6F8944A
:10EC9000DEBF0FBECDBFDF91CF911F910F91FF90CF
:10ECA000EF90DF90CF900C94E575A0960FB6F89496
:10ECB000DEBF0FBECDBFDF91CF911F910F91FF90AF
:10ECC000EF90DF90CF900895CF92DF92EF92FF9276
:10ECD000CF936B017C01C42F4A3069F4F7FE0BC05F
:10ECE000F094E094D094C094C11CD11CE11CF11CA0
:10ECF0008DE20E94E5754C2FC701B601CF91FF90C0
:10ED0000EF90DF90CF900C94FD75CF93DF93EC01E3
:10ED10008991882319F00E94E575FACFDF91CF9190
:10ED20000895CF93DF93EC01FE018491219688230F
:10ED300019F00E94E575F8CFDF91CF9108950F93F8
:10ED40001F93CF938C01C62F89E19FE00E9491769B
:10ED5000C8010E949176CC2331F08AE0CF911F91B7
:10ED60000F910C94E575CF911F910F91089561E07B
:10ED700083E29FE00C949F76AF92BF92CF92DF9296
:10ED8000EF92FF920F931F93CF93DF9386E89EE05D
:10ED90000E949176C0E0D7E0D15021F080E20E943D
:10EDA000E575FACF8C2F0E9456B4CF5FC53099F726
:10EDB0008AE00E94E57501E812E0C0E080E20E946E
:10EDC000E5758C2F0E9456B45801D5E080E20E9470
:10EDD000E575F501C080D180E280F380A70196013E
:10EDE000C701B6010E948DEA882369F180E20E9482
:10EDF000E5758DE30E94E5758DE30E94E5758DE371
:10EE00000E94E5758DE30E94E5758DE30E94E5752E
:10EE1000D150F4E1AF0EB11CD111D8CF8AE00E94DD
:10EE2000E575CF5F0C5F1F4FC53041F68AE0DF917B
:10EE3000CF911F910F91FF90EF90DF90CF90BF90F7
:10EE4000AF900C94E57520E030E0A901C701B60150
:10EE50000E940FEA87FD03C08BE20E94E57543E044
:10EE6000C701B6010E94A4C3D3CFCF92DF92EF9225
:10EE7000FF926A017B010E94917642E0C701B601D0
:10EE8000FF90EF90DF90CF900C94A4C3CF92DF92CD
:10EE9000EF92FF926A017B010E9491764AE0C701DE
:10EEA000B601FF90EF90DF90CF900C9464762F9294
:10EEB0003F924F925F926F927F928F929F92AF920A
:10EEC000BF92CF92DF92EF92FF920F931F93CF9357
:10EED000DF93CDB7DEB7C654D1090FB6F894DEBFC5
:10EEE0000FBECDBF70E060E085E40E941D70182F5A
:10EEF0008F3F09F483C08823E9F084E296E1CA5B7E
:10EF0000DF4F0FB6F894DEBF0FBECDBFDF91CF91BC
:10EF10001F910F91FF90EF90DF90CF90BF90AF9037
:10EF20009F908F907F906F905F904F903F902F9029
:10EF30000C94917624EB30E03A83298383E50E9498
:10EF40001070882321F00E94B16F9A83898365E055
:10EF500070E083E40E941D708AA760E085E50E944E
:10EF60004F7025968FAF259760E087E196E10E946C
:10EF70000C51A981BA81BD01BB0F880B990B0E946E
:10EF80009CE16D837E838F8327969FAF27970E9496
:10EF900050BF688B798B8A8B9B8B1F3F09F045C4D0
:10EFA00020E030E04CE053E46D817E818F81279634
:10EFB0009FAD27970E940FEA18160CF0AAC18CEE9D
:10EFC00095E10E949176CA5BDF4F0FB6F894DEBFE1
:10EFD0000FBECDBFDF91CF911F910F91FF90EF90AA
:10EFE000DF90CF90BF90AF909F908F907F906F9069
:10EFF0005F904F903F902F900C9407B646E450E0FE
:10F000005A8349839BCF1FAEAFC12496EEADFFADAF
:10F010002497808383C2FBEE4F2E512C612C712CE0
:10F0200004C384E190E0A0E0B0E08C8B9D8BAE8BBC
:10F03000BF8BE4E14E2E512C612C712C04C34C8A01
:10F040005D8A6E8A7F8AFFC22496EEADFFAD24975B
:10F050008083D4C389819A81AB81BC8129A93AA9D3
:10F060004BA95CA9821B930BA40BB50BB7FD59C030
:10F070008FAD0E9448C48AE00E94E57589819A811B
:10F08000AB81BC818053984FAF4FBF4F89AB9AABD8
:10F09000ABABBCAB9DA9911177C02EA93FA948ADE0
:10F0A00059ADB101802F26969FAD26970E940FEA99
:10F0B00018160CF053C020E030E040E050E4B101FD
:10F0C000802F26969FAD26970E948CE86EAB7FAB73
:10F0D00088AF99AF2CA53DA54EA55FA589819A81E2
:10F0E000AB81BC81280F391F4A1F5B1F2AAF3BAF82
:10F0F0004CAF5DAF20E030E040EC50E46D817E81AC
:10F100008F8127969FAD27970E948BE89101402F12
:10F1100026965FAD26970E9495E1881F8827881F55
:10F120008DAB88899989AA89BB89C816D906EA0650
:10F13000FB0610F4D701C60129813A814B815C811D
:10F14000281B390B4A0B5B0BDA01C90181389F443C
:10F15000A241B105A8F188E395E10EC289819A81A7
:10F16000AB81BC812AAD3BAD4CAD5DAD821B930B39
:10F17000A40BB50B47E254E266E374E2B7FDD1CFCE
:10F18000812F0E943DC5CDCF20E030E040EF51E41B
:10F190006D817E818F8127969FAD27970E948BE896
:10F1A0009B01AC01B101802F26969FAD26970E944E
:10F1B00095E187FFB6CF43ED54E263EE74E2E0CF12
:10F1C0004AA55BA5888D998D481759070CF09EC0FC
:10F1D00003970CF49BC08BED94E10E9491761F3F46
:10F1E00009F076C0ABECB4E1BA83A9838AEB94E171
:10F1F0000E94917689819A810E94917648855985ED
:10F200006A857B8587ED94E10E9435778AE00E94CC
:10F21000E5758AEB94E10E94917689819A810E943A
:10F22000917649A15AA16BA17CA183ED94E10E9442
:10F2300035778AE00E94E5758AEB94E10E94917629
:10F2400089819A810E949176B501A4018FEC94E1A5
:10F250000E9435778AE00E94E5752596FFAD2597D7
:10F26000FF2391F12CEA35EC47E25EE369A17AA134
:10F270008BA19CA10E94FBE16B017C012CEA35EC87
:10F2800047E25EE3C501B4010E940FE92885398594
:10F290004A855B851F3F09F520936B0B30936C0B00
:10F2A00040936D0B50936E0BC0926F0BD092700B0E
:10F2B000E092710BF092720B6093730B7093740B6E
:10F2C0008093750B9093760B81E0809357017BCEF2
:10F2D000E6E4F7E2FA83E98389CF20930F133093B2
:10F2E00010134093111350931213C0921313D09222
:10F2F0001413E0921513F092161360931713709382
:10F3000018138093191390931A13DECF0E949E5AFC
:10F3100080C088ED95E10E9491760E940EC58FE72E
:10F3200080936A0B24EB30E0A8EEB3E00E9431E852
:10F330006CA77DA78EA79FA7288939894A895B89F1
:10F34000260F371F481F591F2AAF3BAF4CAF5DAF89
:10F350001092570181E08093500132E0310F3EAFAF
:10F36000323008F450CE1FAFC888D988EA88FB88AD
:10F37000C9AADAAAEBAAFCAA812C912C540189A271
:10F380009AA2ABA2BCA288869986AA86BB868FE782
:10F3900090E0A0E0B0E08C8B9D8BAE8BBF8B1C8689
:10F3A00090E49A8FACE1AB8FB6E4BC8F1D8E1E8EBD
:10F3B0001F8E18A23FE7432E512C612C712C1DAAE1
:10F3C0008EAA9FAAA8AEB9AE1EA21FA218A619A601
:10F3D000E1E0EDA3198E188E212C312C00E0269649
:10F3E0001FAE2697F5E11F02C00111249C012A5F80
:10F3F0003C4E22963FAF2EAF2297285F3F4F249678
:10F400003FAF2EAF24974AA5042E000C550B5BA7E7
:10F410004AA780915001882309F4B0C00E9450BFD0
:10F4200069837A838B839C835091390558AB55232C
:10F4300009F48BC00E9425C56091660B7091670B23
:10F440001F3F39F02296AEADBFAD229714966D9155
:10F450007C91072E000C880B990B0E949CE11B01EC
:10F46000082F26969FAF26972D8D3E8D4F8D58A144
:10F4700026969FAD26970E940FEA18163CF42D8E13
:10F480003E8E0F8F2696BFAD2697B8A32C853A8D5A
:10F490004B8D5C8DB101802F26969FAD26970E94E3
:10F4A00095E187FF07C02C863A8E0B8F2696EFAD2D
:10F4B0002697EC8FFDA19101402F26965FAD2697F0
:10F4C0006D817E818F8127969FAD2797FF2309F459
:10F4D0005AC00E9495E187FF38C049815A816B81EB
:10F4E0007C814C195D096E097F09DB01CA018858CE
:10F4F0009341A109B109B7FD28C08C899D89AE89C6
:10F50000BF8984199509A609B709B595A795979557
:10F5100087951F3F09F079CD80936A0B4EA35FA3B7
:10F5200068A779A7FD81FD8F2E812E8F3F813F8FA8
:10F5300027964FAD279748A389819A81AB81BC81DB
:10F54000888B998BAA8BBB8B1DA220E030E040EF0B
:10F5500051E46D817E818F8127969FAD27970E9410
:10F560008CE89101402F26965FAD26970E9495E189
:10F5700087FF70CD86E595E10E949176109250014B
:10F580000E940EC5A1CE0E940FEA1816F4F68981DA
:10F590009A81AB81BC81288939894A895B89821B20
:10F5A000930BA40BB50BAC01BD0148585341610945
:10F5B000710977FDCACF488D598D452B09F40DC1CE
:10F5C000CEA0DFA0E8A4F9A4C80ED91EEA1EFB1E37
:10F5D0002EA13FA148A559A5281B390B4A0B5B0B4F
:10F5E000C301B2010E94CDE7A70196010E94FFE787
:10F5F0004C885D886E887F88420E531E641E751E7F
:10F6000054E145165104610471040CF40ACD8CEEEA
:10F6100048165104610471040CF0FDCC90E84916C1
:10F620005104610471040CF40ACD4C8A5D8A6E8A1F
:10F630007F8A2EEF30E040E050E02419350946097A
:10F64000570929013A014C895D896E897F8980EDCE
:10F6500095E10E944677B301A2018BEC95E10E94EF
:10F6600046774C855A8D6B8D7C8D84EC95E10E949C
:10F6700035774D8D5E8D6F8D78A18DEB95E10E9474
:10F680003577A88DB98D13970CF4A7C0C301B201CB
:10F690000E949CE120E030E040E850E40E94FBE161
:10F6A0004B015C012C853A8D4B8D5C8D6D8D7E8D73
:10F6B0008F8D98A10E948BE82BED3FE049E450E448
:10F6C0000E94FBE120E030E040E05FE30E94FBE1CC
:10F6D0009B01AC01C501B4010E940FE96C877D87D5
:10F6E0008E879F87C701B6010E949CE12FE632E119
:10F6F00043E85AE30E94FBE16B017C011E3F59F095
:10F700002AE939E949E15FE3812C912CA12C6EE3D0
:10F71000B62E1F3F59F42DEC3CEC4CE45EE37BEA43
:10F72000872E7AEA972EA92C7EE3B72E6C857D85ED
:10F730008E859F850E94FBE1688779878A879B87F2
:10F740009B01AC010E948CE8A70196010E940FE981
:10F7500069A37AA38BA39CA3288539854A855B85F9
:10F76000C701B6010E94FBE1A50194010E94FBE1E3
:10F770004B015C014C855D856E857F8587EB95E14E
:10F780000E943577B701A60181EB95E10E9435779C
:10F790008AE00E94E575BEAD82EA95E1B23010F0D4
:10F7A00083E995E10E949176488559856A857B8534
:10F7B0008DE895E10E94357749A15AA16BA17CA102
:10F7C00087E895E10E943577B501A40181E895E1CC
:10F7D0000E9435778AE00E94E5758C899D89AE8903
:10F7E000BF89840D951DA61DB71DB595A795979545
:10F7F00087951F3F09F028CC80936A0B288D398D9F
:10F800002F5F3F4F398F288F3D813C874E814A8F34
:10F810005F815B8F27968FAD27978C8FC980DA80A9
:10F82000EB80FC8098A99DA390CEE12E012E000CC8
:10F83000FF08F70183E0EE0FFF1F8A95E1F7E35A17
:10F84000FE4F668177816F507109072E000C880B7F
:10F85000990B0E949CE19B01AC016D817E818F819F
:10F8600027969FAD27970E940FEA18160CF4A7CB96
:10F8700088ED95E10E9491760E940EC585E18E9DEE
:10F88000F0018F9DF00D1124EA5FFC4E8FE7808719
:10F8900022E330E049CDCF93DF93EB010E949176D4
:10F8A000CE01DF91CF910C945DB48FE79EE00C9474
:10F8B000917689E79EE00C949176CF9384E50E943F
:10F8C0001070C0E08823D9F00E94836AC82F1816F0
:10F8D000B4F40E94597C8DE40E94E57580910C057A
:10F8E00090910D050E9418B66C2FCC0F770B89ED07
:10F8F0009FE00E944B7C8AE00E94E575CFEF8C2F41
:10F90000CF9108950E940EC50E94483680913F0510
:10F910008130A1F40E94557C82E09EE00E949176A5
:10F9200060E088EF9DE00E940C516EE571E080E0A0
:10F9300090E00E945D7388E080933F050895CF9228
:10F94000DF92EF92FF921F93CF93DF9300D000D00E
:10F95000CDB7DEB78EEEC82E82E0D82EE12CF12C8A
:10F96000C982DA82EB82FC82BE016F5F7F4F8AE53B
:10F970000E949B7481110EC010E0812F0F900F9098
:10F980000F900F90DF91CF911F91FF90EF90DF903C
:10F99000CF9008950E940B75C982DA82EB82FC82B7
:10F9A000BE016F5F7F4F8AE50E949B74182F8823EA
:10F9B00019F30E94557C8CED9EE00E9491760E9486
:10F9C000827CDBCFCF92DF92EF92FF921F93CF9397
:10F9D000DF9300D000D0CDB7DEB78EEEC82E82E028
:10F9E000D82EE12CF12CC982DA82EB82FC82BE0196
:10F9F0006F5F7F4F8AE00E949B7481110EC010E000
:10FA0000812F0F900F900F900F90DF91CF911F914A
:10FA1000FF90EF90DF90CF9008950E940B750E94A9
:10FA2000BA740E94D5740E94BA74C982DA82EB82D9
:10FA3000FC82BE016F5F7F4F8AE00E949B74182F8B
:10FA40008823E9F20E94557C8FE99EE00E9491761E
:10FA50000E94827CD5CFEC018B01F42E0E940EC552
:10FA60000E94557C88ED9DE00E949176011511055C
:10FA700011F406E417E2209711F4CFECDDE00E94C8
:10FA80003A5D1F930F93DF93CF938FEB9DE09F938E
:10FA90008F93D1E0DF930E94F3500E949236C09181
:10FAA0006F13C695C6958DB79EB707960FB6F89497
:10FAB0009EBF0FBE8DBF8091A713811104C0D0934C
:10FAC000A7130E94F0B380917013909171130E945C
:10FAD000C9B3DC2FDD0F1D2F1C0F83E00E94DE6AEF
:10FAE0004AE252E06C2F80E00E94616D1092A513F3
:10FAF000D093A61380EB9DE00E94BE6B1092A513DD
:10FB00001093A61383EA9DE00E94BE6B8EE693E1FC
:10FB10000E9487C28111E1CF61E086EC9DE00E94E6
:10FB20009F7689EE93E030E6019729F0232F2A95FE
:10FB30000000E9F7F9CFF89489EE93E038EE0197E9
:10FB400029F0232F2A950000E9F7F9CF0E940EC56E
:10FB5000FF2021F00E948173A895FECF5E9AFCCF12
:10FB60008091191290911A122FEF3FEF981751F0D0
:10FB7000E92FF0E0E75EFD4E228130E09F5F9F7746
:10FB800090931A12C90108952F923F924F925F925B
:10FB90006F927F928F929F92AF92BF92CF92DF929D
:10FBA000EF92FF920F931F93CF93DF9300D000D07B
:10FBB00000D0CDB7DEB780914E05803108F051C13D
:10FBC0000E9450BF6B017C0180914E05811108C0DD
:10FBD0008091191290911A12891B8F7709F491C4A0
:10FBE00011E601E013C08A3019F08D3009F0FCC035
:10FBF0001092011380919F129091A012FC01E55682
:10FC0000FD4E1682892BF1F40E94EEC780914E05BD
:10FC1000803108F026C18091191290911A12891B27
:10FC20008F7709F41EC10E94B07D97FFDCCF0E9440
:10FC3000557C85E89DE00E94917680911912809311
:10FC40001A12E4CF1092A01210929F1221EA32E110
:10FC50003D832C83EC81FD818191803209F44BC07E
:10FC60008E3409F06DC060E87DE08C819D810E943A
:10FC700012E15C01892B49F06EE470E08C819D817A
:10FC800004960E94A0EA009711F48C819D814AE0BD
:10FC900050E070E060E001960E9494DE2B013C0190
:10FCA00080919B1290919C12A0919D12B0919E12F6
:10FCB0000196A11DB11D481659066A067B0629F05A
:10FCC00060E08DE49DE0AB2861F16AE270E08C8138
:10FCD0009D810E94CFEA009739F1282F3C81231B98
:10FCE000B12C222359F02150EC81FD81E20FF11D4E
:10FCF0003081B326F6CFFD83EC83ACCF4AE050E0F1
:10FD000070E060E001960E9494DE8B2C912CB12C67
:10FD1000A12C681579058A059B0551F060E08EE2FB
:10FD20009DE00E94A0B472CF60E084E09DE0F9CF36
:10FD300040929B1250929C1260929D1270929E1261
:10FD400080913F058130E9F067E470E08C819D810E
:10FD50000E94A0EA0097A9F04AE050E070E060E05D
:10FD600001960E9494DE623071058105910548F488
:10FD70008DE89CE00E94917660E083E89CE00E9420
:10FD80000C51C0920305D0920405E0920505F09253
:10FD900006058091A1128B3309F438CF80914E056E
:10FDA000803108F033CF80915005819FC00111242C
:10FDB00061EA72E18F5A9A4F0E94ABEA8091500536
:10FDC000189FF0011124EF54FA4F10828F5F803199
:10FDD00040F48093500580914E058F5F80934E05CF
:10FDE00015CF10925005F7CF90910113913009F47F
:10FDF0000DCF9430B0F09450909301138830C9F433
:10FE000080919F129091A012009709F4FFCE019764
:10FE10009093A01280939F1285569D4EFC011682EE
:10FE2000F5CE8C35C9F49C5F90930113943009F49E
:10FE3000EDCE20919F123091A012A9014F5F5F4F2C
:10FE40005093A01240939F1225563D4EF901868390
:10FE50004F3551051CF4DACE8B3381F60093011334
:10FE6000D5CE0E9450BF6B017C018091FF04909120
:10FE70000005A0910105B09102050097A105B1050B
:10FE800081F14091BC0B5091BD0B6091BE0B709104
:10FE9000BF0B840F951FA61FB71FA7019601281B34
:10FEA000390B4A0B5B0BDA01C901B7FD1AC00E947E
:10FEB000557C4091C30B5091C40B5D834C8386E409
:10FEC0009CE00E9491768C819D810E9485768AE0DB
:10FED0000E94E57540E070E060E090E080E00E9404
:10FEE0002B7D80914A0190914B01A0914C01B091E2
:10FEF0004D01892B8A2B8B2B79F090915613809191
:10FF00005713981709F405C1C092BC0BD092BD0BD2
:10FF1000E092BE0BF092BF0B0E9450BF4B015C0100
:10FF200080912902811108C0209156139091571396
:10FF300081E0291301C080E020910A1330910B1356
:10FF400091E089272A3A31050CF480E091E0409154
:10FF5000C8045091C9046091CA047091CB04452B28
:10FF6000462B472B09F490E0981789F0882309F471
:10FF70000AC1D501C40180569444A24FBF4F80935B
:10FF8000C8049093C904A093CA04B093CB044090D2
:10FF9000E00B5090E10B6090E20B7090E30B20912E
:10FFA000C4043091C5044091C6045091C704C301F4
:10FFB000B2010E9495E1882319F18091C8049091C3
:10FFC000C904A091CA04B091CB044092C4045092D9
:10FFD000C5046092C6047092C704892B8A2B8B2BB0
:10FFE00009F449C0D501C40180569444A24FBF4FC3
:10FFF0008093C8049093C904A093CA04B093CB041F
:020000021000EC
:100000008091C8049091C904A091CA04B091CB0416
:100010000097A105B10579F1881A990AAA0ABB0AC5
:10002000B7FC29C01092C8041092C9041092CA04E7
:100030001092CB0481E39CE00E94917660E08DE118
:100040009CE00E940C5180910C1390910D13181696
:10005000190624F490E080E00E947D218091680BD5
:100060009091690B1816190634F41092690B1092CE
:10007000680B0E94CFBF8091CC049091CD04A091D9
:10008000CE04B091CF04A7019601281B390B4A0B6F
:100090005B0BDA01C901B7FD14C220915613909190
:1000A000571380915601291709F471C0E091571335
:1000B0003BE5E39FF0011124EA58F34F9081899FBB
:1000C000C0011124880F892F881F990B9195182F33
:1000D0000E9450BF112309F4F6C08090BC04909098
:1000E000BD04A090BE04B090BF0481149104A1048B
:1000F000B10409F04FC06C597F4F8F4F9F4F6093F1
:10010000BC047093BD048093BE049093BF041FEFA2
:1001100047C00E9450BF0091BC0B1091BD0B2091B5
:10012000BE0B3091BF0B80904A0190904B01A09084
:100130004C01B0904D01080D191D2A1D3B1D601B7F
:10014000710B820B930B97FF03C01092D004E4CE87
:100150008091D0048111E0CE81E08093D0045E9A3A
:100160008091B90B8E7F8093B90B5E9A8091B90B09
:100170008D7F8093B90B159A8091B90B8B7F8093FB
:10018000B90B5E9AC9CE80E090E0DC01F8CE909188
:100190000C0C95CF681979098A099B0997FDB7CF8F
:1001A000412F50E05D834C8384E00E9464B41111C0
:1001B00093C060E084E00E9459BE80913805882396
:1001C00009F472C10091220110912301C801029724
:1001D00020910C1330910D13281739070CF464C1CA
:1001E00030905713212C19821A821B82809156134A
:1001F000831509F4DFC0832D90E02BE5289FF001E3
:10020000299FF00D1124E05EF34F458956896789D7
:10021000708D452B462B472B89F4418D528D638D74
:10022000748D452B462B472B49F4458D568D678D94
:1002300070A1452B462B472B09F440C0EBE5E89F06
:10024000A001E99F500D1124405E534F5D834C8304
:10025000FA0161817281838194810E944DEA4B0190
:100260005C01EC81FD8161A172A183A194A10E9436
:100270009AE12B013C01EC81FD8165A176A187A16A
:1002800090A50E949AE19B01AC01C301B2010E94BA
:100290000FE9A50194010E94FBE15B018E839C8321
:1002A000222D39814A815B810E940FEA181634F4AD
:1002B0002A2CB982FE81FA832C812B833394332D2F
:1002C0003F70332E93CF1092BC041092BD04109255
:1002D000BE041092BF0464CF8C819D818F3F910535
:1002E00011F461E067CFEAE2F7E2E491E150EA302D
:1002F00008F059C0F0E0E158FE470C9482E889818B
:100300008E8193819F81D381D381AB81B381BB8166
:10031000C78184B5806884BD17BD4FCF84B5806226
:1003200084BD18BD4ACF8091800080688093800092
:10033000EC81FD81F0938900E09388003ECF8091AD
:1003400080008062809380002C813D8130938B00FF
:1003500020938A0032CF8091B00080688093B000F3
:100360001093B3002ACF8091B00080628093B000D8
:100370001093B40022CF8091900080688093900009
:100380004C815D81509399004093980016CF8091E5
:1003900090008062809390008C819D8190939B005F
:1003A00080939A000ACFEC81FD81E038F1050CF0D2
:1003B00098CFFFCEB801110F880B990B0E949CE1DA
:1003C0008B018E839C8320911C0130911D014091F3
:1003D0001E0150911F01622D79818A819B810E94AB
:1003E000FBE198014E815C810E948CE83B014C014D
:1003F000A0902001B09021019B01AC01B8018E8139
:100400009C810E940FEA1816A4F0B501BB0C880B62
:10041000990B0E949CE18B018E839C839B01AC0114
:10042000B301C4010E940FEA18161CF083018E82EA
:100430009C828090C0049090C104A090C204B090AF
:10044000C30498014E815C81C501B4010E940FEA8A
:100450001816C4F428E431EE4AE75FE3C501B4019D
:100460000E94FBE120E037ED43EA5CE30E948CE868
:100470009B01AC01B8018E819C810E94FBE18B0144
:100480008E839C83C801AE81BC818093C00490930D
:10049000C104A093C204B093C304B801CD010E946B
:1004A00081E9CB010E947D2144E6C40ED11CE11CF0
:1004B000F11CC092CC04D092CD04E092CE04F09214
:1004C000CF040E94EEC780913F058823E9F126966C
:1004D0000FB6F894DEBF0FBECDBFDF91CF911F9155
:1004E0000F91FF90EF90DF90CF90BF90AF909F90D3
:1004F0008F907F906F905F904F903F902F900C94D3
:100500009E5A8091030590910405A0910505B09134
:100510000605A7019601281B390B4A0B5B0BDA0174
:10052000C901885E9340A109B109B7FD59CB8DE996
:100530009DE00E949176C0920305D0920405E0925E
:100540000505F09206054CCB26960FB6F894DEBF53
:100550000FBECDBFDF91CF911F910F91FF90EF9014
:10056000DF90CF90BF90AF909F908F907F906F90D3
:100570005F904F903F902F9008952F923F924F920F
:100580005F926F927F928F929F92AF92BF92CF9223
:10059000DF92EF92FF920F931F93CF93DF93CDB72C
:1005A000DEB763970FB6F894DEBF0FBECDBF809164
:1005B000D01183FDA3C189E40E941070882309F43F
:1005C0008FC10E94836A90E01816190614F481E026
:1005D00090E026E0289FF001299FF00D1124E958B2
:1005E000F44F828193811A828C38910514F08CE843
:1005F00090E09093690B8093680B0E94CFBF60E0FE
:1006000081E00E94F5C42091680B3091690B8091C4
:10061000660B9091670B821793070CF422C18CE94B
:1006200094E160E00E940C5181E0809350011B82B4
:100630001C821D821E8219861A861B861C861E86B7
:100640002CE32F873CE1388B46E4498B312C212C5D
:1006500050E859838FEB8A8B1B8A91E09D87812C10
:10066000912C54010091680B1091690BB801012E77
:10067000000C880B990B0E949CE16B017C01232DDF
:10068000322D49815A890E9495E1882389F0809111
:10069000660B9091670BAA81A111E6C0B1E0BB8BFC
:1006A000081719070CF01B8A3C2C2D2CE982FA8ABA
:1006B0000E9450BF6B017C01DC01CB0129853A858A
:1006C0004B855C85821B930BA40BB50BB7FD2FC02C
:1006D000D701C60188519C4FAF4FBF4F89879A877A
:1006E000AB87BC8780E00E9448C488E994E10E94FF
:1006F000917681149104A104B10409F4DFC0C5010D
:10070000B40168577C4E8F4F9F4F6C197D098E093D
:100710009F0928EE33E040E050E00E94DDE7CA0187
:10072000B9014AE00E9464768AE00E94E5750E9461
:10073000C47D0E9450BF6093BC0B7093BD0B80932F
:10074000BE0B9093BF0B6091660B7091670B072EE9
:10075000000C880B990B0E949CE16F8378878C01B9
:100760009B01AC01632D722D89819A890E948BE8CF
:100770002B013C0120E030E0A9010E940FEA87FF35
:1007800004C077FA709477F8709481149104A104EE
:10079000B10409F097C020E030E040E85FE3C30116
:1007A000B2010E9495E187FF10C09D85812C912C9C
:1007B0005401992331F082E8882E86E0982EA12CEE
:1007C000B12C8C0C9D1CAE1CBF1CAB89AA2391F1D3
:1007D0002B813C814D815E812115310541055105FB
:1007E00041F0D701C601821B930BA40BB50BB7FDDB
:1007F00021C02F813885A8016E857F8588899989D8
:100800000E948BE820E030E040E85FE30E9495E141
:1008100087FD2DC0D701C601805A9541AF4FBF4F0C
:100820008B839C83AD83BE839F819E87A885AF8782
:10083000088B198B809150018823C9F08114910491
:10084000A104B10461F0B8E8CB1AB3E1DB0AE10816
:10085000F108C818D908EA08FB08F7FE08C01D8689
:1008600001CF8BEA94E1DDCE081719070CF58091D2
:100870005001882309F442C01092500163960FB6CC
:10088000F894DEBF0FBECDBFDF91CF911F910F91C6
:10089000FF90EF90DF90CF90BF90AF909F908F90A0
:1008A0007F906F905F904F903F902F900C9407B681
:1008B0003C2C2D2CE982FA8A1B8AFACE8FE30E9407
:1008C000E57532CF20E030E040E450E4C301B201EE
:1008D0000E940FEA18160CF078CF4601570175CF29
:1008E00083E50E9410708A83811105C082E50E9411
:1008F0001070882319F00E94B16F76CE63960FB600
:10090000F894DEBF0FBECDBFDF91CF911F910F9145
:10091000FF90EF90DF90CF90BF90AF909F908F901F
:100920007F906F905F904F903F902F9008952F92FF
:100930003F924F925F926F927F928F929F92AF926F
:10094000BF92CF92DF92EF92FF920F931F93CF93BC
:10095000DF93CDB7DEB765970FB6F894DEBF0FBE55
:10096000CDBF8091D01183FD82C10E945D7C8A87BA
:1009700087FD7DC189E40E941070882309F4A8C115
:100980000E94836A90E01816190614F481E090E042
:1009900026E0289FF001299FF00D1124E958F44F1B
:1009A000808191811D8A0E947D2161E081E00E9409
:1009B000F5C420910C1330910D1380910A1390917E
:1009C0000B13821793070CF038C188E894E19F93CA
:1009D0008F9383E994E19F938F931F920E94F3502A
:1009E0000F900F900F900F900F9031E03C8B0E9472
:1009F0005C228C89882309F43AC1909138059B8B3D
:100A00001092380581E0809350011C821D821E8265
:100A10001F821B861C861D861E861F86ACE3A88B44
:100A2000BCE1B98B26E42A8B312C212C30E83A83A7
:100A30004FEB4B831982812C912C540100910C13A4
:100A400010910D13B801012E000C880B990B0E9418
:100A50009CE16B017C01232D322D4A815B810E9438
:100A600095E1882389F080910A1390910B135D8999
:100A70005111EFC0A1E0A983081719070CF01982E2
:100A80003C2C2D2CEA82FB820E9450BF6B017C0122
:100A9000DC01CB012B853C854D855E85821B930B4C
:100AA000A40BB50BB7FD2FC0D701C60188519C4FD1
:100AB000AF4FBF4F8B879C87AD87BE878A850E94CB
:100AC00048C489E794E10E94917681149104A104BD
:100AD000B10409F4EBC0C501B4016053784F8F4FE6
:100AE0009F4F6C197D098E099F0928EE33E040E085
:100AF00050E00E94DDE7CA01B9014AE00E94647635
:100B00008AE00E94E5750E94C47D0E9450BF6093F8
:100B1000BC0B7093BD0B8093BE0B9093BF0B609189
:100B20000A1370910B13072E000C880B990B0E946F
:100B30009CE1688779878C019B01AC01632D722D44
:100B40008A819B810E948BE82B013C0120E030E0F0
:100B5000A9010E940FEA87FF04C077FA709477F822
:100B6000709481149104A104B10409F0A3C020E0A1
:100B700030E040E85FE3C301B2010E9495E187FFE6
:100B800010C09C89812C912C5401992331F08AE961
:100B9000882E82E0982EA12CB12C8C0C9D1CAE1CB2
:100BA000BF1CA981AA2391F12C813D814E815F81D7
:100BB000211531054105510541F0D701C601821BC0
:100BC000930BA40BB50BB7FD21C028853985A8016F
:100BD0006F85788989899A890E948BE820E030E0C6
:100BE00040EC5FE30E9495E187FD36C0D701C60166
:100BF000805A9541AF4FBF4F8C839D83AE83BF8397
:100C000098859F87A985A88B098B1A8B80915001A5
:100C1000882311F181149104A104B10461F0B0EDB5
:100C2000CB1AB7E0DB0AE108F108C818D908EA08CE
:100C3000FB08F7FE11C01C8A01CF2D898DE794E1D6
:100C4000222309F4C4CE5D895C8BD1CE4C894D8BB7
:100C5000CECE0817190724F580915001882321F082
:100C6000109250010E9407B62B8920933805659693
:100C70000FB6F894DEBF0FBECDBFDF91CF911F91AD
:100C80000F91FF90EF90DF90CF90BF90AF909F902B
:100C90008F907F906F905F904F903F902F9008952E
:100CA0003C2C2D2CEA82FB821982EECE8FE30E942F
:100CB000E57526CF20E030E040E450E4C301B20106
:100CC0000E940FEA18160CF06CCF4601570169CF4D
:100CD00083E50E9410708D8B811107C082E50E9410
:100CE00010708C8B882309F4B1CF0E94B16F5BCE5A
:100CF0002F923F924F925F926F927F928F929F922C
:100D0000AF92BF92CF92DF92EF92FF920F931F9319
:100D1000CF93DF93CDB7DEB7EF970FB6F894DEBF72
:100D20000FBECDBF80917B02888B87E50E94DF6F6D
:100D3000882309F41BC120E030E0A9016091ED0295
:100D40007091EE028091EF029091F0020E9495E185
:100D5000811107C00E94557C87EC9FE00E9491762C
:100D600018C18AE50E941070882339F10E94B56F7E
:100D70002091CE0B3091CF0B4091D00B5091D10BE5
:100D80000E948BE86B017C0120E030E040E251ECF6
:100D9000C701B6010E940FEA87FD0AC020E030E0DB
:100DA00040E251E4C701B6010E9495E1181674F4BF
:100DB0000E94557C8AEB9FE0D1CFC090DC0BD09095
:100DC000DD0BE090DE0BF090DF0BDECF40E050E07B
:100DD00060EC7FE788E50E9438702091C60B309167
:100DE000C70B4091C80B5091C90B0E948BE82B0197
:100DF0003C0140E050E060EC7FE789E50E943870FC
:100E00002091CA0B3091CB0B4091CC0B5091CD0B64
:100E10000E948BE84B015C016FEF89E40E942C700B
:100E2000182F6FEF8AE40E942C70082FA301920103
:100E3000C301B2010E948DEA81116EC0A501940127
:100E4000C501B4010E948DEA811166C08BA19CA1ED
:100E5000ADA1BEA18BAB9CABADABBEAB2091E5020F
:100E60003091E6024091E7025091E802C301B201DD
:100E70000E948BE82B013C0120E030E040E05FE382
:100E80006BA97CA98DA99EA90E94FBE19B01AC01E5
:100E9000C301B2010E948CE82BA93CA94DA95EA90F
:100EA0000E940FE90E9481E9162F4FA058A469A45F
:100EB0007AA42091E9023091EA024091EB0250912C
:100EC000EC02C501B4010E948BE84B015C0120E0FB
:100ED00030E040E05FE3C301B2010E94FBE19B010F
:100EE000AC01C501B4010E948CE8A30192010E94EB
:100EF0000FE90E9481E9062F812F012E000C990B2A
:100F000097FD2CC0059764F5802F002E000C990BDF
:100F100097FD28C0059744F51530D8F50530C8F57C
:100F200080E00E94517295E01902F0011124E00F57
:100F3000F11D07FDFA95EE0FFF1FEE0FFF1FEF5794
:100F4000FD4FC082D182E282F38288890E94517271
:100F500088898823F1F00E94E42C1BC010E0D4CFD4
:100F600014E0D2CF00E0D8CF04E0D6CF8AE40E94CC
:100F7000DF6F81110CC070E060E086E50E941D709B
:100F80009A8389830597F0F085E99FE0E7CE0E9478
:100F90009F72EF960FB6F894DEBF0FBECDBFDF9104
:100FA000CF911F910F91FF90EF90DF90CF90BF9066
:100FB000AF909F908F907F906F905F904F903F90F9
:100FC0002F90089560E084E40E944F708F8740E086
:100FD00050E0BA018AE50E9438706BA77CA78DA704
:100FE0009EA740E050E86BE376E483E50E9438700A
:100FF00020E030E040E752E40E940FE96093660190
:101000007093670180936801909369010091511377
:1010100010915213D801CD90DD90ED90FC9020E01E
:1010200030E0A901C701B6010E948CE8962E872EF8
:10103000382E292E20E030E040E450E40E9495E173
:1010400087FF06C0912C812CB0E43B2E80E4282E33
:1010500020E030E046E953E4C701B6010E948CE885
:101060006BAB7FAB88AF99AF20E030E844E953E445
:101070000E940FEA18163CF41BAAB0E8BFABE4E9E3
:10108000E8AFF3E4F9AFD80114964D905D906D9000
:101090007C90179720E030E0A901C301B2010E94C3
:1010A0008CE85B016C0120E030E040E951E40E94F3
:1010B00095E187FF06C0A12CB12CF0E9CF2EA1E469
:1010C000DA2E20E030E04CE553E4C301B2010E9487
:1010D0008CE87B018C0120E030E04AE453E40E947C
:1010E0000FEA181624F4E12CF12C0AE413E488E446
:1010F0000E94DF6F882309F413C20E94B56F0E941B
:1011000081E92B0177FF02C06F5F7F4F759567956F
:10111000EE27FF27E61BF70BFFAFEEAFBF016259CB
:101120007F4F072E000C880B990B0E949CE16AAF41
:101130007BAF8CAF9DAF9501A6010E940FEA1816F8
:1011400024F0AAAEBBAECCAEDDAE6EAD7FAD6A56BE
:101150007F4F072E000C880B990B0E949CE15B01CE
:101160006C01292D382D432D522D0E940FEA18169F
:1011700024F0A92CB82CC32CD22CC501D6018B8B02
:101180009C8BAD8BBE8B8AAD9BADACADBDAD8F8B5B
:10119000988FA98FBA8FB201550C880B990B0E94BA
:1011A0009CE12B013C01AC019B016AAD7BAD8CAD98
:1011B0009DAD0E948CE81B014C019701A8010E9483
:1011C00095E187FF02C071018401A3019201B5017D
:1011D000C6010E948CE85B016C012BA93FA948ADB8
:1011E00059AD0E9495E187FF04C0ABAABFAAC8AE63
:1011F000D9AE8BA99FA9A8ADB9AD8B8F9C8FAD8FB0
:10120000BE8FC701D8018F8F98A3A9A3BAA3BE012F
:10121000695E7F4FCE0143960E947D6E882309F45C
:10122000ACC1BE01615E7F4FCE014B960E947D6EC8
:10123000E82E882309F4A1C12F89388D498D5A8D54
:101240006F8D78A189A19AA10E948BE820E030E0FF
:1012500040E85EE30E94FBE14B015C012B893C8985
:101260004D895E896B8D7C8D8D8D9E8D0E948BE866
:1012700020E030E040E85EE30E94FBE16BA37CA34A
:101280008DA39EA38FA298A6A9A6BAA689819A81AA
:101290001816190674F483E69FE00E9491768F85F4
:1012A000882321F089E59FE00E9491768AE00E94E0
:1012B000E5750E940B220E94D42A80E00E945172A0
:1012C00080E090E0A0E2B1E48FA798ABA9ABBAAB05
:1012D00060E0CE018F960E94F02B2091ED023091BC
:1012E000EE024091EF025091F0026BA17CA18DA122
:1012F0009EA10E9495E1811130C02091F1023091B0
:10130000F2024091F3025091F4026FA178A589A5F1
:101310009AA50E9495E1811120C02091E5023091AB
:10132000E6024091E7025091E8026B897C898D8941
:101330009E890E9495E1811110C02091E9023091AF
:10134000EA024091EB025091EC026F89788D898D11
:101350009A8D0E9495E18823A9F00E949F7288E0EF
:10136000FE01B396ADEEB2E001900D928A95E1F7E1
:1013700088E0FE017396A5EEB2E001900D928A9589
:10138000E1F7188A60E085E40E944F708824839416
:10139000811102C062E0862E1B861C861D861E8679
:1013A0001A8A9E2C49E2C42E4FE0D42E57E3A52E74
:1013B0005FE0B52E1A8915300CF0E9C06B857C858D
:1013C0008D859E859B01AC010E948DEA8111DFC055
:1013D0003324339435E0232E911005C033243A94FE
:1013E00022242A9484E091E09926F12EFF0CFF0C30
:1013F000F10EF394898B19896A89121509F4C3C017
:10140000062E000C770B880B990B0E949CE12FA1F4
:1014100038A549A55AA50E94FBE12F89388D498D31
:101420005A8D0E948CE82B013C01612F110F770B24
:10143000880B990B0E949CE12BA13CA14DA15EA1C0
:101440000E94FBE12B893C894D895E890E948CE8D2
:101450006B837C838D839E834F82588669867A86D0
:1014600089819A81892B89F085E49FE00E94917699
:101470008F2D0E9456B469E170E083E49FE00E94E2
:101480004B7C80E49FE00E9491761F92F9E1FF93EC
:101490001F92FF92DF92CF92BF92AF921F920E9453
:1014A000F3502981482DBE01695F7F4FCE0103961D
:1014B0000E9480B62B013C014B865C866D867E8641
:1014C0000FB6F894DEBF0FBECDBFAC019B010E94EA
:1014D0008DEA811155C009898A8925E002038001BE
:1014E0001124080F111D87FD1A95000F111F000F01
:1014F000111F0F571D4FA30192016BA57CA58DA550
:101500009EA50E948CE8D8016D937D938D939C934A
:101510001397188A0E94C47DF3948989830D6ACF3A
:10152000A501B60186E40E9438702B013C01492DCB
:10153000582D632D722D8CE40E9438706B8B7C8B40
:101540008D8B9E8B4F8A588E698E7A8EA701B8013B
:1015500082E40E9438706B017C014BA95FA968ADE1
:1015600079AD82E50E9438706B8F7C8F8D8F9E8F56
:10157000CF8ED8A2E9A2FAA24ACE89E79FE0EECBAD
:1015800088890E9451728A898F5F8A8B13CF0E944B
:1015900007B60E94746E882359F088890E945172A0
:1015A00080E090E0A0ECBFE78B879C87AD87BE878B
:1015B0006B857C858D859E859B01AC010E948DEAA3
:1015C00081114DC08F85811126C082E0F82E02E086
:1015D00094E0C92E12E0DC2CD11A21E041E0612F09
:1015E000802F0E94696521E04FEF612F8F2D0E94AF
:1015F00069652FEF41E06D2D802F0E9469652FEF07
:101600004FEF6D2D8F2D0E946965115020F701500D
:10161000F3940F3FF9F60E94BC760E94E3728F8527
:10162000811118C084ED9BE00E9464709B01AC01A5
:101630006091DC0B7091DD0B8091DE0B9091DF0BE4
:101640000E948BE86093DC0B7093DD0B8093DE0BC4
:101650009093DF0B8F858111E888E0927B020E94D6
:10166000BB2A80917B0281110E94C82C0E94496A8A
:1016700072CC2F923F924F925F926F927F928F9295
:101680009F92AF92BF92CF92DF92EF92FF920F9311
:101690001F93CF93DF93CDB7DEB7C254D1090FB6F6
:1016A000F894DEBF0FBECDBF21968FAF21972DB727
:1016B0003EB723963FAF2EAF239780910E058D3412
:1016C00009F4E0C4843511F40C949C9F873491F4A0
:1016D00080910C0590910D058C31910509F465C23E
:1016E00008F06DC08430910509F4EAC130F4029726
:1016F00008F4FBC00E941EB67AC18531910509F439
:1017000076C14B97B9F787E00E94896481116FC158
:101710008CE0E5EEF1E0DE01119601900D928A95E4
:10172000E1F780E50E94107060E081110E94736A09
:1017300080E090E0A8E4B2E48F8F98A3A9A3BAA3B5
:1017400080E090E0A0EAB0E48B8F9C8FAD8FBE8FDD
:10175000613009F4EEC1623009F4FFC120E030E0ED
:1017600040E050E46091DC0B7091DD0B8091DE0B6A
:101770009091DF0B0E948CE87B018C0120E030E02F
:1017800046E953E40E940FEA181624F4E12CF12CE8
:1017900006E913E4A984BA84CB84DC849701A80108
:1017A000B501C6010E940FEA181614F475018601EE
:1017B000C701D8018F8B988FA98FBA8FF0C18A3259
:1017C000910509F4C7C208F081C08D31910509F473
:1017D00052C24E9709F08ECF0091511310915213BF
:1017E000D8012D913D914D915C916091D40B7091F8
:1017F000D50B8091D60B9091D70B0E948CE8AB0152
:10180000BC0188E50E94387069837A838B839C834E
:10181000F80124813581468157816091D80B709100
:10182000D90B8091DA0B9091DB0B0E948CE8AB0115
:10183000BC0189E50E9438706D837E838F83988711
:10184000BE016B5F7F4FCE0101960E947D6E8823A3
:1018500009F4CDC080E00E9451720E94D42A61E058
:1018600085E40E944F70182F21E0482FBE016B5F66
:101870007F4FCE0101960E9480B66B017C01AC01C6
:101880009B010E948DEA811119C049815A816B81A7
:101890007C8188E290E10E9435774D815E816F8185
:1018A000788583E290E10E943577B701A6018EE149
:1018B00090E10E9435778AE00E94E5750E94BB2A7C
:1018C00011110E94496A0E94E42C91C08B35910548
:1018D00009F463C38C35910509F463C38A35910516
:1018E00009F008CF1092070582C080913F05813032
:1018F00009F07DC0EBE5CE2EE2E0DE2EF4EDEF2E1A
:10190000FBE0FF2EA6ECAA2EABE0BA2E10E088E595
:10191000810F0E941070882309F4B6C00E94B56F31
:101920002B013C01812F0E944F65882309F4A2C03E
:10193000D7012D913D914D915C91C301B2010E945F
:101940008CE8D6016D937D938D939C9313971F5FC5
:10195000F4E0CF0ED11C24E0E20EF11C34E0A30E23
:10196000B11C1330A1F685E40E941070882309F49D
:1019700096C00E94B56F6B017C0183E00E944F65A9
:10198000882371F02091E00B3091E10B4091E20B44
:101990005091E30BC701B6010E948CE86B017C01FA
:1019A000C0926702D0926802E0926902F0926A02E5
:1019B00040E050E0BA0186E40E94387020E030E058
:1019C000A9010E940FEA181684F40E94B56F20E066
:1019D00030E040E752E40E940FE9609318017093F1
:1019E000190180931A0190931B010E94562721969A
:1019F0002FAD219721110C94FE950E9450BF60934A
:101A000003057093040580930505909306050091E6
:101A10004F0511E6109FF0011124EF54FA4F808119
:101A200081110C94FE9586E794E10E949176019FC6
:101A3000800111240F5A1A4FD8018C918E3411F065
:101A40000C94BD9F80E20E94E5758EE40E94E575CE
:101A50000F5F1F4FF80181918F0190ED980F9A3021
:101A600030F08D3221F08B3211F00C94BD9F0E942A
:101A7000E575F0CFF5012081318142815381C301A9
:101A8000B2010E948BE85DCFF70180819181A28134
:101A9000B381F60180839183A283B38358CF809171
:101AA000E00B9091E10BA091E20BB091E30B8093DE
:101AB000670290936802A0936902B0936A0278CF9C
:101AC00080E50E941070C12CD12C7601882321F072
:101AD0000E94636A6B017C0183E50E941070882379
:101AE00061F00E94B56F20E030E04AE754E40E94C4
:101AF000FBE10E9488E96B017C010E940B2280912E
:101B00002A02811105C060E08CEE9FE00E940C511A
:101B10000E9450BFC60ED71EE81EF91E0E9450BF7D
:101B20006C197D098E099F0997FF61CF0E94C47DC2
:101B3000F5CFBE01655E7F4FCE0109960E94D12B85
:101B4000AE01415E5F4FBE016B5F7F4FCE010196DC
:101B50000E94AF2B0E94E42C4ACF29853A854B8501
:101B60005C856091DC0B7091DD0B8091DE0B9091B8
:101B7000DF0B0E948CE86B017C0120E030E046E93D
:101B800053E40E9495E187FD06C0C12CD12C76E973
:101B9000E72E73E4F72ECF8AD88EE98EFA8EBE0137
:101BA000655E7F4FCE014796C9CF87E00E944027F0
:101BB000811106C060E08FE40E944F70811117CF41
:101BC0000E940B221092270160917B028CE40E94FC
:101BD0004F70E82E80E00E9451720E9450BF6093C7
:101BE000BC0B7093BD0B8093BE0B9093BF0B0E94F8
:101BF000D42A81E080933C050E94C8318AE50E9486
:101C0000DF6FF82E882369F081E00E944027182FAB
